:100000000C948C130C94B6130C94B6130C94B61376
:100010000C94B6130C94B6130C94B6130C94B6133C
:100020000C94B6130C94B6130C94B6130C94B6132C
:100030000C94B6130C9498250C94B6130C94B61328
:100040000C94B6130C9477230C9451C20C94B613F1
:100050000C94547E0C944A7E0C94B6130C94B613F4
:100060000C94B6130C94B6130C94B6130C94B613EC
:100070000C94B6130C94B6130C94B6130C94B613DC
:100080000C94A4790C94B6130C94B6134E414E49BB
:100090004E495459494E46CDCCCC3D0AD7233C1746
:1000A000B7D13877CC2B329595E6241FB14F0A0093
:1000B0000020410000C84200401C4620BCBE4CCA83
:1000C0001B0E5AAEC59D7400407A10F35A00A07200
:1000D0004E18090010A5D4E80000E8764817000083
:1000E000E40B54020000CA9A3B000000E1F5050051
:1000F0000080969800000040420F000000A086019A
:10010000000000102700000000E803000000006469
:1001100000000000000A00000000000100000000D4
:10012000002C76D888DC674F0823DFC1DFAE59E1A9
:10013000B1B796E5E3E453C63AE651997696E8E618
:10014000C28426EB898C9B62ED407C6FFCEFBC9CEB
:100150009F40F2BAA56FA5F490055A2AF75C936BFD
:100160006CF9676DC11BFCE0E40D47FEF520E6B5B8
:1001700000D0ED902E0300943577050080841E0892
:100180000000204E0A000000C80C333333330F98B0
:100190006E12831141EF8D2114893BE65516CFFE77
:1001A000E6DB18D1844B381BF77C1D901DA4BBE403
:1001B00024203284725E228100C9F124ECA1E53D45
:1001C0002741425300504C410042656400456E6334
:1001D0006C6F73757265002568753A2530326875E5
:1001E0000025303268753A253032687500202020AD
:1001F000202020200020202020003FFFF038007029
:1002000030FC3020FC102078102030102C00D02E34
:1002100031D02F7BD02F7BD02E31D02C00D020306E
:100220001020781020FC1030FC303800703FFFF0B8
:100230003FFFF03800703186302387102787902FDA
:1002400087D02F03D0203010207810207810203055
:10025000102F03D02F87D027879023871031863027
:100260003800703FFFF0041040020820020820040C
:100270001040082080104100104100082080041028
:10028000400000001FFFF81FFFF863616E63656C9C
:10029000005072696E742041626F72746564004D23
:1002A00032350050617573696E672E2E2E007265AF
:1002B00073756D65004D32340050726F6265205A5F
:1002C000204F66667365740046696C2E2044696130
:1002D0002E004F6666004F6E004520696E206D6DE2
:1002E0005E3300452073746570732F6D6D005A2066
:1002F00053746570732F6D6D00592053746570735E
:100300002F6D6D00582053746570732F6D6D004113
:100310006476616E6365642053657474696E677397
:100320000046696C616D656E740053746570732F5F
:100330006D6D00436F6E66696775726174696F6E8B
:100340000053746F77004465706C6F790053572DBC
:100350004D6F64650053656C662D5465737400526F
:100360006573657400436F6E666967757261746961
:100370006F6E00526573746F7265204465666175B7
:100380006C7473004C6F61642053657474696E679C
:10039000730053746F72652053657474696E67736C
:1003A00000424C546F7563680050726F6265205A4A
:1003B000204F666673657400416476616E636564A0
:1003C0002053657474696E6773004D61696E004DEA
:1003D0003139305335350A4732380A4732390A4DF8
:1003E0003430300A4D313034533231350A473238E7
:1003F0000A4D313039533231350A4D3432305331B0
:100400000A4731583130305931303046353030308C
:100410000A47315A300A4D3530300A4D31313720D4
:10042000536574205A204F6666736574004D3130F1
:1004300036533132380A4D33303343385332313545
:100440004530550A4D3530300A4D3131372050494D
:10045000442054756E6520446F6E65004D3139300F
:100460005335350A4D313034533231350A4732383D
:100470000A4732394C310A4731205831303059312E
:10048000303046353030300A47315A30004D353043
:10049000300A4D3131372053657474696E677320AB
:1004A00053746F726564005072657020666F7220BD
:1004B0005A2041646A7573740053746F72652053D7
:1004C000657474696E6773005049442054756E6595
:1004D000005365747570004D61696E003F004261A4
:1004E000636B0053746F70004D3231005072696E4F
:1004F000742066726F6D204D656469610052656C91
:1005000065617365204D65646961004D3232004C50
:100510006576656C696E6720546F6F6C7300436F0E
:100520006E66696775726174696F6E0054656D708F
:1005300065726174757265004D6F74696F6E0052FB
:100540006573756D65205072696E740041747461D5
:100550006368204D656469610054756E650053746D
:100560006F70205072696E74005061757365205011
:1005700072696E7400496E666F2053637265656EB2
:100580000043616E6E6F7420656E746572207375C2
:10059000626469723A2000022E2E00015265667272
:1005A000657368004D61696E002100486F74656E67
:1005B0006420746F6F20636F6C64004261636B0032
:1005C00050726F63656564004D6F74696F6E0044AF
:1005D000697361626C652053746570706572730035
:1005E0004D3834004175746F20486F6D6500473297
:1005F00038004D61696E0050726568656174202431
:1006000020456E6400507265686561742024204244
:1006100065640054656D706572617475726500C5BE
:1006200001C101436F6F6C646F776E005072656833
:1006300065617420240046616E2053706565640016
:10064000426564004E6F7A7A6C65004D61696E0098
:1006500050726F6265205A204F666673657400465B
:100660006C6F770046616E2053706565640042656B
:1006700064004E6F7A7A6C65005370656564004D56
:1006800061696E00486F6D696E67204661696C65CF
:1006900064006F70656E00545249474745524544A7
:1006A000003A20007A5F6D696E00795F6D696E00B7
:1006B000785F6D696E005265706F7274696E672045
:1006C000656E6473746F70207374617475730A005F
:1006D00020746F6F206C6F6E67206578747275730D
:1006E000696F6E2070726576656E7465640A0020AD
:1006F000636F6C6420657874727573696F6E2070B7
:10070000726576656E7465640A00486F6D652025B4
:100710007325732573204669727374005761726E76
:10072000696E673A20486F6D696E672042756D701B
:100730002044697669736F72203C20310A000202FE
:100740000400000000000000000000000000007A2B
:100750004300007A4300007A43000000410000009B
:10076000410000004000007A4300007A4300007A14
:10077000430000000000000000000000005365740A
:1007800074696E67732053746F72656400454550D9
:10079000524F4D20496E697469616C697A65640ACB
:1007A0000000803B4400803B440000204100009654
:1007B000420000A0420000A0420000C8430000BE6A
:1007C00042D0070000D0070000640000004B00008A
:1007D0000024F4D43050C38E20C2A24017828B7004
:1007E00011127A910D816CD90AA861E108C7586687
:1007F00007615143061E4B5D05C145A7041A41110F
:1008000004093D9803713931034036DB02653391A9
:1008100002D4305402802E1D02632CEE01752AC5CD
:1008200001B028A001102781018F2564012B244BE2
:1008300001E0223401AC211F018D200D01801FFC3D
:1008400000841EED00971DDF00B81CD200E61BC619
:1008500000201BBC00641AB200B219A8000A19A03B
:10086000006A189900D117910040178B00B51684C3
:100870000031167E00B31579003A157300C7146F66
:100880000058146A00EE1366008813630025135E97
:1008900000C7125B006C12570015125400C11151B1
:1008A0000070114F0021114B00D61049008D1047E8
:1008B000004610440002104200C00F4000800F3E6E
:1008C00000420F3C00060F3B00CB0E3800930E3762
:1008D000005C0E3500270E3400F30D3200C10D31DF
:1008E00000900D3000600D2E00320D2D00050D2CF6
:1008F00000D90C2B00AE0C2900850C29005C0C27BC
:1009000000350C27000E0C2600E80B2400C40B2435
:1009100000A00B23007D0B23005A0B2100390B2173
:1009200000180B2000F80A1F00D90A1E00BB0A1E7F
:10093000009D0A1D00800A1D00630A1C00470A1B57
:10094000002C0A1B00110A1A00F7091A00DD091908
:1009500000C4091900AB091900920917007B091896
:1009600000630917004C0916003609160020091605
:10097000000A091500F5081500E0081400CC081459
:1009800000B8081400A4081400900813007D081291
:10099000006B0813005808120046081200340811B2
:1009A00000230811001208110001081100F00710BF
:1009B00000E0071000D0071000C0071000B0070FBC
:1009C00000A107100091070E0083070F0074070FA6
:1009D0000065070E0057070E0049070E003B070D84
:1009E000002E070E0020070D0013070D0006070D4F
:1009F00000F9060C00ED060D00E0060C00D4060C14
:100A000000C8060C00BC060C00B0060C00A4060BC7
:100A10000099060C008D060B0082060B0077060B72
:100A2000006C060B0061060A0057060B004C060A14
:100A30000042060A0038060A002E060A0024060AAA
:100A4000001A060A001006090007060A00FD05093B
:100A500000F4050900EB050900E2050900D90509C4
:100A600000D0050900C7050900BE050900B5050845
:100A700000AD050800A50509009C050800940508BF
:100A8000008C050800840508007C05080074050832
:100A9000006C050700650508005D050700560508A0
:100AA000004E050700470507004005080038050708
:100AB00000310507002A050700230507001C05066D
:100AC00000160507000F05070008050600020507C8
:100AD00000FB040600F5040700EE040600E8040627
:100AE00000E2040700DB040600D5040600CF04067C
:100AF00000C9040600C3040600BD040600B70406CE
:100B000000B1040500AC040600A6040600A004051C
:100B1000009B04060095040500900406008A040565
:100B20000085040500800406007A040500750405AC
:100B300000700405006B04050066040500610405EF
:100B4000005C04050057040500520405004D04052F
:100B50000048040500430405003E0404003A04056F
:100B60000035040500300404002C040500270404AB
:100B700000230405001E0404001A040400160405E2
:100B800000110404000D0404000904050004040419
:100B90000000040400FC030400F8030400F4030450
:100BA00000F0030400EC030400E8030400E4030481
:100BB00000E0030400DC030400D8030400D40304B1
:100BC00000D0030400CC030400C8030300C50303E2
:100BD0000024F404D9201BC40C5C0E9804C4095FE3
:100BE0000265077101F405F900FB04B300480487AE
:100BF00000C10369005803550003034500BE023AD3
:100C0000008402310053022A002902250004022038
:100C100000E4011C00C8011900AF0117009801147D
:100C20000084011300710110006101100051010ED8
:100C30000043010D0036010B002B010B0020010BBE
:100C400000150109000C01090003010800FB000860
:100C500000F3000800EB000700E4000600DE0006D9
:100C600000D8000600D2000600CC000500C7000531
:100C700000C2000500BD000400B9000400B5000476
:100C800000B1000400AD000400A9000400A50003A9
:100C900000A20003009F0004009B000300980003D3
:100CA000009500020093000300900003008D0002F5
:100CB000008B00030088000200860002008400030D
:100CC00000810002007F0002007D0002007B000224
:100CD0000079000200770001007600020074000233
:100CE0000072000100710002006F0002006D00013F
:100CF000006C0002006A0001006900020067000148
:100D0000006600010065000100640002006200014D
:100D10000061000100600001005F0002005D000151
:100D2000005C0001005B0001005A00010059000155
:100D30000058000100570001005600010055000155
:100D40000054000100530000005300010052000154
:100D50000051000100500001004F0001004E000052
:100D6000004E0001004D0001004C0001004B00004E
:100D7000004B0001004A000100490001004800004A
:100D80000048000100470001004600000046000145
:100D90000045000000450001004400010043000040
:100DA0000043000100420000004200010041000039
:100DB0000041000100400001003F0000003F000131
:100DC000003E0000003E0001003D0000003D00012B
:100DD000003C0000003C0000003C0001003B000023
:100DE000003B0001003A0000003A00010039000019
:100DF0000039000100380000003800000038000110
:100E00000037000000370001003600000036000007
:100E100000360001003500000035000000350001FB
:100E200000340000003400000034000100330000F2
:100E300000330000003300010032000000320000E7
:100E400000320001003100000031000000310001DB
:100E5000003000000030000000300001002F0000D2
:100E6000002F0000002F0000002F0001002E0000C6
:100E7000002E0000002E0001002D0000002D0000BB
:100E8000002D0000002D0001002C0000002C0000AF
:100E9000002C0000002C0001002B0000002B0000A3
:100EA000002B0000002B0001002A0000002A000097
:100EB000002A0000002A000100290000002900008B
:100EC000002900000029000000290001002800007E
:100ED0000028000000280000002800000028000171
:100EE0000027000000270000002700000027000066
:100EF0000027000100260000002600000026000058
:100F0000002600000026000100250000002500004A
:100F1000002500000025000000250000002500013C
:100F20000024000000240000002400000024000031
:100F30000024000100230000002300000023000023
:100F40000023000000230000002300000023000114
:100F50000022000000220000002200000022000009
:100F600000220000002200010021000000210000FA
:100F700000210000002100000021000000210000ED
:100F800000210001002000000020000000200000DF
:100F900000200000002000000020000000200000D1
:100FA00000200001001F0000001F0000001F0000C3
:100FB000001F0000001F0000001F0000001F0001B4
:100FC000001E0000001E0000001E0000001E0000A9
:100FD00000043700001E290000511B0000581000BB
:100FE0000010090000CC040000780200004101005C
:100FF0000020436F756E7420583A004265640045C6
:101000003100626564002C2073797374656D207300
:10101000746F7070656421204865617465725F4902
:10102000443A200048656174696E67204661696CC6
:1010300065640048656174696E67206661696C6506
:1010400064004D3131322053687574646F776E00DF
:101050001000C90210012C01400122017001180189
:10106000B0010E01F00104015002FA00B002F000DC
:101070003003E600D003DC009004D2007005C80005
:10108000A006BE000008B400B009AA00D00BA00062
:10109000600E960060118C00001582002019780007
:1010A000C01D6E00A0226400B0275A00902C500092
:1010B00000314600E0343C0010383200903A2800FD
:1010C000603C1E00A03D1400803E0A00203F00004E
:1010D000544845524D414C2052554E4157415900BC
:1010E000546865726D616C2052756E61776179002C
:1010F0004572723A204D415854454D50004D41586B
:1011000054454D5020747269676765726564004587
:1011100072723A204D494E54454D50004D494E543F
:10112000454D502074726967676572656400202FB1
:10113000002042403A0020403A007C3C3E5E2B3D7D
:101140003F2F5B5D3B2C2A225C00434F4D4D554E9B
:1011500049434154494F4E0044525952554E00455F
:1011600052524F525300494E464F004543484F009C
:10117000486F74656E642049646C652054696D65C0
:101180006F757400486F74656E642049646C6520E7
:1011900054696D656F75740A002121204B494C4CD0
:1011A0002063617573656420627920746F6F206DB0
:1011B00075636820696E6163746976652074696D12
:1011C00065202D2063757272656E7420636F6D6D7E
:1011D000616E643A200053544F505045442E200015
:1011E0005072696E7465722073746F7070656420DC
:1011F00064756520746F206572726F72732E20465D
:10120000697820746865206572726F7220616E64FF
:1012100020757365204D39393920746F20726573DC
:10122000746172742E202854656D706572617475D6
:1012300072652069732072657365742E205365741E
:1012400020697420616674657220726573746172BE
:1012500074696E67290A004E6F20436865636B737B
:10126000756D2077697468206C696E65206E756D88
:101270006265722C204C617374204C696E653A2053
:10128000004E6F20436865636B73756D20776974DA
:1012900068206C696E65206E756D6265722C204CDD
:1012A000617374204C696E653A2000636865636BF6
:1012B00073756D206D69736D617463682C204C616A
:1012C0007374204C696E653A20004C696E65204E3F
:1012D000756D626572206973206E6F74204C617346
:1012E00074204C696E65204E756D6265722B312CD1
:1012F000204C617374204C696E653A20004D313189
:10130000300053657269616C207374617475732069
:101310006D69736D617463680A005344207265617E
:1013200064206572726F720A004D656469612049BC
:101330006E73657274656400506C656173652052EC
:1013400065736574005052494E5445522048414CD3
:101350005445440025533A20255300706F77657239
:101360006F6666004B494C4C45442E200050726914
:101370006E7465722068616C7465642E206B696C94
:101380006C28292063616C6C6564210A0053544FFA
:10139000505045442E20005072696E74657220735F
:1013A000746F707065642064756520746F20657259
:1013B000726F72732E20466978207468652065729A
:1013C000726F7220616E6420757365204D393939F2
:1013D00020746F20726573746172742E20285465B6
:1013E0006D706572617475726520697320726573C2
:1013F00065742E205365742069742061667465726B
:101400002072657374617274696E67290A0065637E
:10141000686F3A004572726F723A0042696C696E89
:10142000656172204C6576656C696E6720477269EC
:10143000643A0A0021212053544F502063616C6CA0
:1014400065642062656361757365206F6620424C38
:10145000546F756368206572726F72202D207265FB
:1014600073746172742077697468204D3939390A50
:101470000021212053544F502063616C6C6564201F
:1014800062656361757365206F6620424C546F75A9
:101490006368206572726F72202D207265737461AB
:1014A00072742077697468204D3939390A004265B1
:1014B00064204C6576656C696E6720004661696CD6
:1014C000656420746F20656E61626C65204265649E
:1014D000204C6576656C696E670A00496E76616CB2
:1014E0006964206D6573682E0A0050726F62696EC0
:1014F0006720506F696E740025532025692F256978
:10150000002E0A002F0050726F62696E67206D65B1
:10151000736820706F696E742000202844525952FD
:10152000554E2900473239204175746F2042656459
:10153000204C6576656C696E67003F20284C2C5204
:101540002C462C4229206F7574206F6620626F75BF
:101550006E64732E0A003F2856296572626F7365A8
:10156000206C6576656C20696D706C61757369625D
:101570006C652028302D34292E0A00426164205ADF
:101580002076616C75650A004E6F2062696C696E29
:1015900065617220677269640A0020496E76616C29
:1015A00069642065787472756465722000536C6597
:1015B00065702E2E2E005A2050726F626520506189
:1015C0007374204265640A005A2050726F6265206D
:1015D0005061737420426564004732384C300020FB
:1015E0005A3A200020593A200042656420583A2097
:1015F000004D65736820706F696E74206F7574207C
:101600006F662072616E67650A00436C69636B20C8
:10161000746F20526573756D652E2E2E004E6F20EF
:101620004D6F76652E00456E642066696C65206C92
:101630006973740A00426567696E2066696C65208B
:101640006C6973740A004E6F206D656469610A00ED
:10165000706175736500286E6F2066696C6529007E
:1016600043757272656E742066696C653A2000532A
:1016700044207072696E74696E67206279746520A7
:10168000004E6F74205344207072696E74696E67E7
:101690000A002E0A0044656C6574696F6E206661ED
:1016A000696C65642C2046696C653A200046696C5B
:1016B000652064656C657465643A0025697300256E
:1016C000696D20256973002569682025696D2025CD
:1016D000697300256964202569682025696D2025C6
:1016E00069730025697920256964202569682025AA
:1016F000696D20256973005072696E742074696D7C
:10170000653A20006F6B006F6666006B1166115FB3
:101710001158114A1144454255473A00544D33443B
:1017200020456E64657233204F46462E00204500EA
:10173000204D39322058004649524D574152455F9D
:101740004E414D453A4D61726C696E20322E302EFD
:10175000375F4457372E3320544D3344204533539D
:101760004D444242202841707220323420323032BF
:10177000312032303A31373A33332920534F5552E2
:1017800043455F434F44455F55524C3A687474700B
:10179000733A2F2F6769746875622E636F6D2F49D6
:1017A0006E73616E6974794175746F6D6174696F80
:1017B0006E2F4D61726C696E2F747265652F437266
:1017C00065616C6974794477696E5F322E302050A0
:1017D000524F544F434F4C5F56455253494F4E3A28
:1017E000312E30204D414348494E455F54595045B4
:1017F0003A544D334420456E646572332045585445
:1018000052554445525F434F554E543A3120555539
:1018100049443A63656465326132662D3431613220
:101820002D343734382D396231322D6335356336F6
:10183000326633363766660A002F2F004D31343555
:1018400020533C696E6465783E206F7574206F6626
:101850002072616E67652028302D31290A002054DE
:1018600000205200416363656C65726174696F6E3C
:101870003A2050005741524E494E4721204C6F7735
:10188000205A204A65726B206D6179206C65616415
:1018900020746F20756E77616E7465642070617559
:1018A0007365732E0A004D3230362058004F46467D
:1018B000004F4E0020580020204D61783A20002033
:1018C0000020204D696E3A2000536F667420656ECB
:1018D0006473746F70733A200046523A0020466C6D
:1018E0006F773A20003A200020536572766F20000F
:1018F000206F7574206F662072616E67650A0053F1
:101900006572766F200050726F6265204F66667355
:101910006574205A0050726F6265204F6666736569
:1019200074205A0020643A0020693A0020703A007E
:10193000496E76616C69642065787472756465724D
:101940000A0064697300656E0043290A0061626CD5
:10195000656420286D696E2074656D702000436F8A
:101960006C6420657874727564657320617265209B
:10197000004D34323120696E636F7272656374207A
:10198000706172616D657465722075736167650A57
:10199000004D65736820706F696E74206F757420D8
:1019A0006F662072616E67650A004F6666736574C4
:1019B00073204170706C696564004572723A2054FE
:1019C0006F6F206661722100546F6F206661722014
:1019D00066726F6D207265666572656E63652070F4
:1019E0006F696E740A00454550524F4D204F4B0AA7
:1019F00000290A0020746F20003F5A206F75742060
:101A00006F662072616E6765202800290A002074C5
:101A10006F20003F59206F7574206F662072616ED1
:101A2000676520282D00290A0020746F20003F5888
:101A3000206F7574206F662072616E676520282D97
:101A400000205A0020590050726F6265204F666670
:101A50007365742058004D383400446F6E652070F3
:101A600072696E74696E672066696C650A004D372D
:101A700037004D333100496E76616C6964206578BA
:101A80007472756465720A0020573A00436F6F6C78
:101A9000696E672E2E2E0048656174696E672E2E62
:101AA0002E00452025530020573A0042656420430C
:101AB0006F6F6C696E672E2E2E004265642048653C
:101AC0006174696E672E2E2E0023646566696E65EB
:101AD0002044454641554C545F004B6420004B69FF
:101AE00020004B702000504944204175746F74757C
:101AF0006E652066696E697368656421205075742F
:101B000020746865206C617374204B702C204B69C5
:101B100020616E64204B6420636F6E7374616E7419
:101B2000732066726F6D2062656C6F7720696E74CA
:101B30006F20436F6E66696775726174696F6E2E90
:101B4000680A00504944204175746F74756E6520B1
:101B50006661696C6564212074696D656F75740ACE
:101B600000504944204175746F74756E652066613C
:101B7000696C6564212054656D706572617475725D
:101B80006520746F6F20686967680A00204B643AAB
:101B90002000204B693A2000204B703A200020435F
:101BA0006C617373696320504944200A00205475A6
:101BB0003A2000204B753A2000206D61783A2000D1
:101BC000206D696E3A200020643A2000206269612D
:101BD000733A2000504944204175746F74756E65E6
:101BE0002073746172740A00504944204175746F07
:101BF00074756E65206661696C6564212054656D3D
:101C0000706572617475726520746F6F20686967A2
:101C1000680A00504944204175746F74756E6520E0
:101C20006661696C65642120426164206865617445
:101C300065722069640A00504944204175746F74CC
:101C4000756E65004572723A207574663820666F4D
:101C50006E74206E6F7420696E697469616C697A44
:101C600065642E004572723A207574663820666F7E
:101C70006E74206E6F7420696E697469616C697A24
:101C800065642E004572723A207574663820666F5E
:101C90006E74206E6F7420696E697469616C697A04
:101CA00065642E00000C0F00FE07022503BB017FB8
:101CB000FE08FE08FE05080806000040F0C88888F7
:101CC000987810050808060000C0F8888888888879
:101CD000F80505050600012030F830200508080643
:101CE00000002070F820202020E00509090600FFF0
:101CF0002070A8A8B888887020070505070001D8BB
:101D00006C366CD80509090600FFF8A88888888811
:101D100088A8F8050A0A0600FE205050505088A8EE
:101D2000A8887003030306000340A040FFFFFFFFE5
:101D3000FFFFFFFFFFFFFFFFFFFFFFFFFFFFFFFFB3
:101D4000FFFF0000000605FF010707060200808074
:101D50008080800080030303060105A0A0A0050683
:101D60000606000050F85050F8500509090600FF1B
:101D70002070A8A07028A87020050707060000C8DA
:101D8000C8102040989805070706000040A0A04012
:101D9000A8906801030306020580808003090906F4
:101DA00001FF204040808080404020030909060157
:101DB000FF804040202020404080050707060000AB
:101DC00020A8702070A8200505050600012020F835
:101DD00020200203030601FFC04080050101060028
:101DE00003F8020202060100C0C005070706000052
:101DF00008101020404080050707060000708898F2
:101E0000A8C8887003070706010040C04040404052
:101E1000E0050707060000708808102040F8050755
:101E200007060000F808103008887005070706004C
:101E30000010305090F81010050707060000F880D9
:101E4000F008088870050707060000304080F08819
:101E50008870050707060000F808101020202005EC
:101E600007070600007088887088887005070706D5
:101E7000000070888878081060020505060100C01F
:101E8000C000C0C00206060601FFC0C000C04080FE
:101E900003050506010120408040200503030600DC
:101EA00002F800F803050506010180402040800586
:101EB000070706000070881020200020050707068D
:101EC00000007088B8A8B880700507070600007089
:101ED0008888F8888888050707060000F048487059
:101EE0004848F005070706000070888080808870E9
:101EF000050707060000F04848484848F00507076E
:101F0000060000F88080F08080F8050707060000D2
:101F1000F88080F0808080050707060000708880C8
:101F200080988870050707060000888888F88888E8
:101F300088030707060100E04040404040E00507F5
:101F40000706000038101010109060050707060003
:101F5000008890A0C0A09088050707060000808038
:101F600080808080F805070706000088D8A8888848
:101F700088880507070600008888C8A8988888050B
:101F8000070706000070888888888870050707069C
:101F90000000F08888F08080800507070600007048
:101FA000888888A89068050707060000F08888F0F0
:101FB000A090880507070600007088807008887068
:101FC000050707060000F82020202020200507072D
:101FD0000600008888888888887005070706000042
:101FE0008888888850502005070706000088888860
:101FF00088A8A85005070706000088885020508848
:102000008805070706000088885020202020050743
:1020100007060000F80810204080F80309090601AF
:10202000FFE080808080808080E005070706000058
:10203000804040201010080309090601FFE020201D
:102040002020202020E005030306000520508805FD
:1020500001010600FEF80303030601058040200588
:102060000505060000700878887805070706000057
:102070008080F0888888F005050506000070808063
:1020800088700507070600000808788888887805A2
:1020900005050600007088F080700507070600003F
:1020A000304840E04040400507070600FE70888841
:1020B000887808700507070600008080F088888807
:1020C000880307070601004000C0404040E00409C3
:1020D000090601FE1000301010101090600507076F
:1020E00006000080808890E09088030707060100C2
:1020F000C04040404040E0050505060000D0A8A8CB
:10210000A8A8050505060000B0C88888880505054B
:1021100006000070888888700507070600FEF088B2
:102120008888F080800507070600FE788888887810
:102130000808050505060000B0C880808005050573
:1021400006000078807008F00507070600002020D0
:10215000F820202018050505060000888888986862
:10216000050505060000888888502005050506003D
:10217000008888A8A8500505050600008850205052
:10218000880507070600FE888888502040800505DE
:1021900005060000F8102040F80309090601FF2099
:1021A00040404080404040200109090602FF8080F5
:1021B000808080808080800309090601FF80404084
:1021C00040204040408005030306000248A890FFDD
:1021D00043616E6E6F74206F70656E2073756264FC
:1021E0006972200053442063617264206F6B0A009F
:1021F0006F70656E526F6F74206661696C65640AFA
:1022000000766F6C756D652E696E69742066616904
:102210006C65640A004E6F20534420636172640A47
:10222000000A4D3234004D3233202573002E0A004F
:102230006F70656E206661696C65642C2046696C00
:10224000653A200046696C652073656C656374654A
:10225000640A002053697A653A200046696C65205B
:102260006F70656E65643A2000454E4420535542B8
:10227000524F5554494E450A002220706F73002278
:1022800020706172656E743A2200535542524F5568
:1022900054494E452043414C4C207461726765742B
:1022A0003A220053756263616C6C204F76657266EA
:1022B0006C6F77004578636565646564206D61784F
:1022C00020535542524F5554494E45206465707411
:1022D000683A0057726974696E6720746F20666986
:1022E0006C653A2000667265736800646F696E679A
:1022F000002066696C653A20004E6F7720002F61E0
:1023000075746F25632E670070012C019001270101
:10231000B0012201C0011D01F001180110021301DA
:1023200030020E016002090190020401C002FF00A8
:102330000003FA004003F5008003F000D003EB0037
:102340002004E6007004E100E004DC004005D70052
:10235000C005D2004006CD00D006C8008007C300EB
:102360003008BE00F008B900C009B400B00AAF00E0
:10237000B00BAA00D00CA500000EA000500F9B00CF
:10238000C01096005012910000148C00C0158700F8
:10239000B0178200B0197D00D01B7800001E7300BA
:1023A00040206E0090226900F024640040275F0006
:1023B00090295A00E02B5500102E500020304B0081
:1023C00010324600E033410090353C0010373700B2
:1023D00070383200A0392D00B03A2800A03B23000D
:1023E000603C1E00103D1900903D1400103E0F008F
:1023F000703E0A00C03E0500003F0000403FFBFF6A
:10240000803FF6FFC03FF1FF2020506C616E6E658B
:102410007242756666657242797465733A2000206F
:1024200046726565204D656D6F72793A2000436F85
:102430006D70696C65643A204170722032342032CC
:102440003032310A00204C6173742055706461741D
:1024500065643A20323032312D30342D3138207CD1
:1024600020417574686F723A2054696E794D6163CA
:1024700068696E657333440A00322E302E375F442C
:1024800057372E330A004D61726C696E0020536F0E
:102490006674776172652052657365740A0020570F
:1024A00061746368646F672052657365740A002005
:1024B00042726F776E206F75742052657365740A6F
:1024C000002045787465726E616C20526573657486
:1024D0000A00506F77657255700A007374617274E8
:1024E0000A004732385859004D31303031006F6B97
:1024F000006572726F722077726974696E672074FA
:102500006F2066696C650A00446F6E6520736176A2
:10251000696E672066696C652E0A004D3239004588
:102520006E6473746F7073002553202563202563D8
:1025300020256320256300205A3A0020593A0020C4
:10254000583A00656E6473746F7073206869743AEA
:102550002000000000010200090A0000000004033E
:10256000080700000000000000000000000000005C
:102570000000004D6F76652025736D6D004D6F7600
:102580006520302E316D6D004D6F766520316D6D9B
:10259000004D6F76652031306D6D004D6F76652092
:1025A00041786973004578747275646572004D6F87
:1025B0007665205A004D6F76652059004D6F76651F
:1025C0002058005072696E742066726F6D204D65E0
:1025D00064696100FFFFFF50726F62696E67204699
:1025E00061696C65640A0050726F62696E672046AB
:1025F00061696C656400205A3A200020593A200035
:1026000042656420583A2000220A00556E6B6E6FB6
:10261000776E20636F6D6D616E643A202200544DB9
:10262000334420456E646572332052656164792EAF
:10263000005072696E74696E672E2E2E005072699A
:102640006E74205061757365640020453A00205A0D
:102650003A0020593A00583A004572726F7220775A
:10266000726974696E6720746F20454550524F4DF2
:10267000210A0020746F6F206C6F6E67206578747C
:10268000727573696F6E2070726576656E746564BD
:102690000A0020636F6C6420657874727573696FCB
:1026A0006E2070726576656E7465640A005265739B
:1026B000656E643A200000002200250028002B00EF
:1026C00000002100240027002A0002020202020268
:1026D00002020404040404040404030303030303C4
:1026E000030301010101010101010102040810209D
:1026F00040800102040810204080010204081020DC
:10270000408080402010080402012F2F616374690B
:102710006F6E3A00ECD40BDC11241FBECFEFD0E477
:10272000DEBFCDBF12E0A0E0B1E0E6E7F4ED01E0EE
:102730000BBF02C007900D92A034B107D9F728E172
:10274000A0E4B2E001C01D92A630B207E1F713E1A8
:10275000CBE8D3E104C02197FE010E949AE7CA3872
:10276000D107C9F70E94DBD50C942EEA0C94000027
:102770000F931F93CF93DF93CDB7DEB760970FB65C
:10278000F894DEBF0FBECDBF8C01DC01ED91FC9152
:102790000280F381E02DBE016F5F7F4F0995882392
:1027A00009F464C08981807CC9F56F81637070E031
:1027B000762F6627770F770F8885B4E08B9FC0014F
:1027C0001124682B792B898582958695869583704F
:1027D000682B6F5F7F4F90E080E02A852370220F87
:1027E0003B8537FB332730F9232B3E813F70230F86
:1027F0003327331F2750310904C0660F771F881F06
:10280000991F2A95D2F760960FB6F894DEBF0FBED7
:10281000CDBFDF91CF911F910F910895803419F5AD
:1028200068856695669570E090E080E0CB0177273B
:1028300066272A85622B098510E0102F0027012EBC
:10284000000C220B330B602B712B822B932B6F5FB1
:102850007F4F8F4F9F4F4AE0660F771F881F991F4A
:102860004A95D1F7D0CF8BE0F801848360E070E027
:10287000CB01C9CF0895FC0182810895CF92DF92E8
:10288000EF92FF9280917002882309F457C0C090A4
:102890006C02D0906D02E0906E02F0906F0220E02A
:1028A00030E0A901C701B6010E94ADE0882309F418
:1028B00045C020E030E040E05FE3C701B6010E9480
:1028C00013E19B01AC010E9413E12BED3FE049E4D1
:1028D00050E40E9413E19B01AC0160E070E080E8ED
:1028E0009FE30E9427E86B017C01C0926702D092AF
:1028F0006802E0926902F0926A0260911C01709194
:102900001D01072E000C880B990B0E94B4E02AE0F1
:1029100037ED43E25CE30E9413E1A70196010E94B8
:1029200013E1609364017093650180936601909355
:102930006701FF90EF90DF90CF900895C12CD12CCC
:1029400080E8E82E8FE3F82ED0CF8F929F92AF923F
:10295000BF92CF92DF92EF92FF92FC01C080D180B4
:10296000E280F38020E030E040E251E4C701B601AC
:102970000E9413E120E030E040E251E40E9413E1C4
:102980004B015C0120E030E0A901C701B6010E94C3
:10299000ADE020E030E040EA50E487FF04C020E0F2
:1029A00030E040EA50ECC501B4010E94A4E720E009
:1029B00030E040E251E40E9427E80E9499E89B0140
:1029C0008BE237FF05C022273327261B370B8DE20A
:1029D00080933506C90168EE73E00E9486E7CB015B
:1029E000EAE0F0E0BF010E9486E7805D8093360652
:1029F000C90164E670E00E9486E7CB01BF010E9436
:102A000086E7805D80933706C901BF010E9486E793
:102A1000282FCB01BF010E9486E7805D8093380696
:102A20008EE280933906205D20933A0685E396E096
:102A3000FF90EF90DF90CF90BF90AF909F908F90DE
:102A400008959C0197FF26C0EE27FF27E81BF90B8E
:102A50002D398FEF38070CF05DC08DE2809337067B
:102A6000CF0164E670E00E9486E7CB012AE030E007
:102A7000B9010E9486E7805D80933806CF01B901D5
:102A80000E9486E7CB01B9010E9486E7805D8093B2
:102A900039062AC0283E83E03807B4F1C90168EE40
:102AA00073E00E9486E7CB01EAE0F0E0BF010E94FC
:102AB00086E7805D80933706C90164E670E00E9476
:102AC00086E7CB01BF010E9486E7805D80933806D0
:102AD000C901BF010E9486E7CB01BF010E9486E7C2
:102AE000805D80933906F901CF016AE070E00E94B1
:102AF00086E7805D80933A0687E396E008958DE24D
:102B000037FDC5CF80E2C3CFF90180E2243631051D
:102B10000CF0A4CF80E28093370680933806EA3029
:102B2000F1056CF38DE237FF80E280933806CF0128
:102B30006AE070E00E9486E7605D60933906D4CF5A
:102B40009C0197FD2DC080E2243631055CF0C9015F
:102B500064E670E00E9486E7CB016AE070E00E94C4
:102B600086E7805D8093380680E22A3031055CF08C
:102B7000EAE0F0E0C901BF010E9486E7CB01BF0196
:102B80000E9486E7805D80933906C9016AE070E0A3
:102B90000E9486E7805D80933A0688E396E0089578
:102BA0003195219531098DE2DDCF282F81E324363F
:102BB00009F080E28093370690E22A3040F03AE054
:102BC000822F632F0E9458E70E9458E7905D9093F0
:102BD0003806822F6AE00E9458E7905D909339068C
:102BE00085E280933A0687E396E0089560911C01A0
:102BF00070911D01072E000C880B990B0E94B4E008
:102C00002AE037ED43E25CE30E9413E12091670282
:102C1000309168024091690250916A020E9413E16A
:102C200060936401709365018093660190936701DE
:102C30000895CF93DF93EC01CB01BA010E94B4E079
:102C400029EC38EC48EC5EE30E9427E820E030E015
:102C500040E05FE30E94A4E70E94A0E86883DF9160
:102C6000CF9108950E94B4E029EC38EC48EC5EE383
:102C70000E9427E820E030E040E05FE30E94A4E704
:102C80000E94A0E824E6629FC001112481589F4F52
:102C90006FEF70E00E9486E7862F0C94D515CF93D6
:102CA000DF93EC01CB01BA010E94B4E020E030E0F8
:102CB000A9010E94A4E70E9499E879836883DF91C3
:102CC000CF9108950E94B4E020E030E0A9010E9475
:102CD000A4E70E9499E8CB010C94A01580914206CC
:102CE000811104C08091FA058093A4060895809113
:102CF00019178823C1F0815080931917E2E5F5E197
:102D0000882351F08150990B2BE1289FF001299FD6
:102D1000F00D1124E55FF94E8BE1A7E3B5E10190D9
:102D20000D928A95E1F720911917211105C0809124
:102D3000241780628093241781E090E0A0E0B0E047
:102D4000211103C080E090E0DC0180933006909375
:102D50003106A0933206B093330610922B0681E021
:102D600080932D0683E080935B0108958F929F925C
:102D7000AF92BF92CF92DF92EF92FF92CF936B010F
:102D80007C0120E030E0A9010E94ADE087FDAAC0EF
:102D90006DEB77E386E095E3A70196010E94A4E737
:102DA0006B017C0120E030E0A9010E94ADE087FFCB
:102DB0009EC0C701B601905820E030E040E251E4E7
:102DC0000E9413E120E030E040E251E40E9413E170
:102DD00020E030E040EA50E40E94A4E720E030E048
:102DE00040E251E40E9427E80E9499E86B017C01CF
:102DF00080E28093340660E280E1C81687E2D8065C
:102E0000E104F1048CF0C701B60120E137E240E0B3
:102E100050E00E9417E7CA01B9012AE030E040E023
:102E200050E00E9417E7605D6093350660E288EE2F
:102E3000C81683E0D806E104F1048CF0C701B6019E
:102E400028EE33E040E050E00E9417E7CA01B901E4
:102E50002AE030E040E050E00E9417E7605D6093B8
:102E6000360660E284E6C816D104E104F1048CF071
:102E7000C701B60124E630E040E050E00E9417E7C9
:102E8000CA01B9012AE030E040E050E00E9417E7B3
:102E9000605D609337068AE0882E912CA12CB12CBE
:102EA000C701B601A50194010E9417E7C62FCA0108
:102EB000B901A50194010E9417E7605D609338068F
:102EC0008EE280933906C05DC0933A0684E396E0B3
:102ED000CF91FF90EF90DF90CF90BF90AF909F90F9
:102EE0008F9008956DEB77E386E095EB55CF20E06A
:102EF00030E040E251E4C701B60162CFCF93DF93E7
:102F0000EC01CB01BA010E94B4E020E030E040E2E5
:102F100051E40E9427E820E030E0A9010E94A4E7E4
:102F2000688379838A839B83DF91CF9108950E9480
:102F3000B4E020E030E040E251E40E9427E820E0E5
:102F400030E0A9010E94A4E70C94B616CF93DF935A
:102F5000EC01CB01BA010E94B4E020E030E04AE786
:102F600054E40E9427E820E030E0A9010E94A4E791
:102F7000688379838A839B83DF91CF9108958091C1
:102F8000B8159091B915891B8F7051F480915D0629
:102F9000813031F08091241782FB882780F90895D1
:102FA00081E00895FC0184910895FC0180810895D9
:102FB000209104063091050621153105E9F0809134
:102FC0000206909103060296245031098217930756
:102FD0009CF490931A05809319050E94B0C1605E1D
:102FE00070448D4F9F4F60931B0570931C05809319
:102FF0001D0590931E05089510921B0510921C0547
:1030000010921D0510921E0508958F929F92AF9207
:10301000BF92EF92FF920F931F93CF93DF93EC0138
:103020008B01E42EF22E8091CA159091CB158C174E
:103030009D0709F43EC02091460227FD10924602EA
:103040002CE5C534D20709F03FC08F52924671F487
:103050000E94B0C16E517B4F8F4F9F4F60936404AD
:10306000709365048093660490936704D093CB15A6
:10307000C093CA1530E020E000933006109331066B
:103080002093320630933306E0922B06F0922C0602
:10309000CF52D24621F410922A061092630482E0A5
:1030A00080935B0181E080932D0610926A04109258
:1030B0002906DF91CF911F910F91FF90EF90BF9064
:1030C000AF909F908F90089522E6CF32D20771F68D
:1030D00085549C4519F0CFE2D2E6C8CF0E94B0C11A
:1030E0008090640490906504A0906604B09067049A
:1030F000681979098A099B0997FFEDCF80914506E8
:103100008770873041F7C6E1D6E5B0CF20E040E0D8
:1031100070E060E082EC9DE10C9405188091B506AA
:10312000811114C0809168019091690101972091EB
:10313000091530910A152817390744F420E040E0BA
:1031400070E060E087EC9DE10C9405180C94861803
:1031500021E020932A06FC0180819181A281B38124
:103160008093120190931301A0931401B093150161
:1031700020E040E070E060E0809117069091180632
:103180000C940518CF93DF9300D000D0CDB7DEB7F5
:103190008DEC9CECACECBCE389839A83AB83BC8361
:1031A000CE0101960E94A8180F900F900F900F90DB
:1031B000DF91CF910895CF93DF9300D000D0CDB7AA
:1031C000DEB78DEC9CECACECBDE389839A83AB83DA
:1031D000BC83CE0101960E94A8180F900F900F900B
:1031E0000F90DF91CF910895CF93DF9300D000D05F
:1031F000CDB7DEB780E090E0A0E8BFE389839A8393
:10320000AB83BC83CE0101960E94A8180F900F904B
:103210000F900F90DF91CF910895CF93DF9300D05F
:1032200000D0CDB7DEB780E090E0A0E2B1E48983C2
:103230009A83AB83BC83CE0101960E94A8180F909D
:103240000F900F900F90DF91CF9108950F931F93E0
:103250000E94B0C1009127041091280420912904F4
:1032600030912A04601B710B820B930B97FD0CC0ED
:1032700089B183FB882780F991E089274A9B826086
:10328000309B846080932604809126048170909105
:10329000260491FD826090912504981749F08130B1
:1032A00009F148F0823079F0833091F08093250461
:1032B0001F910F910895913079F09230B9F7909164
:1032C000240491500CC0992339F09330C1F3EECF10
:1032D0009130A9F3923051F7909124049F5F90931D
:1032E0002404E4CF992359F3933001F7F5CFCF921B
:1032F000DF92EF92FF92CF93C82F0E94B0C16B0173
:103300007C0124EA30E74DE75FE3609112017091A0
:10331000130180911401909115010E94ADE087FD89
:1033200018C08AEF90E0A0E0B0E08C0D9D1DAE1DAE
:10333000BF1D8093180490931904A0931A04B093AE
:103340001B04C0931001CF91FF90EF90DF90CF90BE
:10335000089580E090E0DC01E8CFCF93DF93EC01AB
:103360008D810E940B7F60E08B81DF91CF910C9467
:10337000B9C0DF92EF92FF920F931F93CF93DF9329
:103380008C01C62FD22FF32EE42ED52E0E94AD191C
:103390000E942FC28C2F80640E94FF7E8D2D0E9480
:1033A000FF7E8E2D0E94FF7E8F2D0E94FF7E8D2F2F
:1033B0000E94FF7E87E8C11101C085E90E94FF7E5F
:1033C000CC3011F40E94047FC0E00E94047FF80119
:1033D000868387FF04C0CF3F11F0CF5FF6CFDF9128
:1033E000CF911F910F91FF90EF90DF90089561E0D2
:1033F000FC0183810E94B9C08FEF0C94FF7E0F9374
:103400001F93CF938C010E94AD190E942FC2C82F29
:10341000882371F08DEF0E94FF7E0E942FC2C82F7B
:10342000C8010E94F7198C2FCF911F910F91089519
:1034300082E1F8018483F4CF8F929F92AF92BF9282
:10344000CF92DF92EF92FF920F931F93CF93DF9370
:10345000EC016A017B01590120E030E0A90167E33A
:103460000E94B919A501980167E1CE010E94B9191E
:10347000811127C08F81833039F089E0CC0CDD1CAD
:10348000EE1CFF1C8A95D1F7A701960169E1CE01D8
:103490000E94B91911E0882319F010E087E08C83AD
:1034A000CE010E94F719812FDF91CF911F910F91CB
:1034B000FF90EF90DF90CF90BF90AF909F908F9054
:1034C000089589E08C8310E0EBCFCF93DF93EC017C
:1034D0006EBDFA01CA019E5F0DB407FEFDCF2081CB
:1034E0002EBD0DB407FEFDCF21812EBD3296E8170B
:1034F000F90791F70DB407FEFDCF8FEF0E94FF7E15
:103500008FEF0E94FF7E0E94047F8E838F71853033
:1035100049F083E18C83CE010E94F71980E0DF91AE
:10352000CF91089581E0FBCF0F931F93CF93DF934B
:10353000EC018B010E94AD190E942FC281110CC0B9
:1035400085E18C8310E0CE010E94F719812FDF9175
:10355000CF911F910F910895A8016CEFCE010E94A9
:10356000651A182F882361F3EECF0F931F93CF9323
:10357000DF93EC0189018F81833039F089E0440FBA
:10358000551F661F771F8A95D1F79A01AB0168E135
:10359000CE010E94B91981112AC0A8016EEFCE0197
:1035A0000E94651A182F8823B1F00E942FC2182F8D
:1035B0008823D1F020E030E0A9016DE0CE010E9427
:1035C000B919882321F086E18C8310E004C00E94A1
:1035D000047F8111F8CFCE010E94F719812FDF916E
:1035E000CF911F910F91089587E18C83F4CF86E0EE
:1035F000EBCF1F93CF93DF93EC010E94AD1920E036
:1036000030E0A9016CE0CE010E94B91911E08823D5
:1036100019F010E083E08C83CE010E94F719812F0E
:10362000DF91CF911F9108951F93CF93DF93EC010A
:103630008F81833039F089E0440F551F661F771F53
:103640008A95D1F79A01AB0162E1CE010E94B919C6
:1036500011E0882319F010E085E08C83CE010E94F0
:10366000F719812FDF91CF911F9108958F929F922B
:10367000AF92BF92EF92FF920F931F93CF93DF937E
:103680008C01EB017A010E94B0C14B015C012CE27C
:10369000820E21E0921EA11CB11C0E94047FF80141
:1036A00086838F3F69F40E94B0C1681979098A093D
:1036B0009B0997FDF2CF81E1F8018483C0E021C02E
:1036C0008E3F71F5F1E0EF1AF1088FEF8EBDFE012C
:1036D0002FEF0DB407FEFDCF8EB581932EBDCF0128
:1036E0008C1B9D0B8E159F05A0F30DB407FEFDCF1F
:1036F0008EB5CE0DDF1D88830E94047F0E94047F5B
:10370000C1E0C8010E94F7198C2FDF91CF911F9162
:103710000F91FF90EF90BF90AF909F908F90089582
:103720008FE0CACF0F931F93CF93DF93EC018B01F0
:103730000E94AD1940E052E0B801CE01DF91CF9177
:103740001F910F910C94361B0F931F93CF93DF9310
:10375000EC0189018F81833039F089E0440F551FD6
:10376000661F771F8A95D1F79A01AB0161E1CE01FF
:103770000E94B91981110AC040E052E0B801CE019F
:10378000DF91CF911F910F910C94361B84E08C83B5
:10379000CE010E94F71980E0DF91CF911F910F9128
:1037A00008958F929F92AF92BF92CF92DF92EF9245
:1037B000FF920F931F93CF93DF93EC01162F1F827D
:1037C0001C824B830E94B0C16B017C0120EDC20EB4
:1037D00027E0D21EE11CF11CA89561E08B810E94BC
:1037E000B9C08B810E9420B8249A2C9A279A2698D7
:1037F000259A81E00E940B7F85E08D830E940B7FDC
:103800000AE08FEF0E94FF7E0150D9F7A89520E0D3
:1038100030E0A90160E0CE010E94B9198E838130A9
:1038200081F00E94B0C16C197D098E099F0997FD36
:10383000EECF81E08C83CE010E94F7191A8280E0DE
:103840006AC0A8952AEA31E040E050E068E0CE0185
:103850000E94B919853041F581E08F83A8958F8149
:10386000812C912C5401823029F4812C912CA12C93
:1038700080E4B82E20E030E0A90167E3CE010E9489
:10388000B919A501940169E2CE010E94B9198E838C
:103890008823F1F00E94B0C16C197D098E099F093F
:1038A00097FDE8CF8AE0C6CF04E00E94047F8E83B4
:1038B0000150D9F78A3A11F482E0CFCF0E94B0C10B
:1038C0006C197D098E099F0997FDBCCF82E0B2CFAC
:1038D0008F818230C1F420E030E0A9016AE3CE019B
:1038E0000E94B919882311F088E0A4CF0E94047FB8
:1038F000807C803C11F483E08F830E94047F0E94CF
:10390000047F0E94047FCE010E94F71981E08A8320
:10391000173070F41D83DF91CF911F910F91FF90AD
:10392000EF90DF90CF90BF90AF909F908F900895D1
:1039300088E18C8384CF0F931F93CF93DF93EC01A7
:103940008B0120E030E0A90169E00E94B9198111E2
:103950000AC040E150E0B801CE01DF91CF911F9144
:103960000F910C94361B80E18C83CE010E94F719D5
:1039700080E0DF91CF911F910F910895CF93C82FD1
:10398000CB010E947B7A81EA96E00E947B7A82E9F1
:1039900096E0CC2311F087E996E00E947B7A8AE0DA
:1039A000CF910C94637A0C94BCC10C94BCC140912F
:1039B000E50221E042276CE070E00C9462B940918E
:1039C000E50221E0422764E070E00C9462B9409186
:1039D000E50221E0422761E070E00C9462B9409179
:1039E000E50221E0422762E070E00C9462B9409168
:1039F000E50221E0422761E070E00C9462B9409159
:103A0000E50221E0422768E070E00C9462B9409141
:103A1000E50221E042276CE070E00C9462B941E0DD
:103A200061E070E00C9462B94091E50221E0422728
:103A30000C9462B962E070E00C9448C16CE070E0F4
:103A40000C9448C164E070E00C9448C161E070E0FF
:103A50000C9448C161E070E00C9448C16CE070E0E7
:103A60000C9448C1CF93DF938091B8159091B9150C
:103A7000891B80958F7019F40E944083F5CF809147
:103A8000B8158F5F8F70A091B8159BE4A99FD001E6
:103A90001124FD01E854F94FEF0119929A95E9F7C5
:103AA00098E09083A353B94F90E1EAEBF5E10190E0
:103AB0000D929A95E1F72091B8159091B9152913B7
:103AC00003C094E69093B5158093B815DF91CF911C
:103AD0000C94A477CF92DF92EF92FF920F931F93F3
:103AE000C12CD12C76018C0128E736E044E756E062
:103AF00060E776E08CE696E00E94BAB81F910F91DD
:103B0000FF90EF90DF90CF900895CF93DF9300D098
:103B100000D0CDB7DEB784EF91E0A0E0B0E08983BC
:103B20009A83AB83BC83BE016F5F7F4F88E70E949F
:103B300019790F900F900F900F90DF91CF9108950A
:103B4000CF93DF93CDB7DEB720E24F8158856E81EA
:103B50008D810E9433BDDF91CF9108956FEF8091E9
:103B6000FA050C944CBF61E37EE482E00C94D3D25E
:103B700066E37EE481E00C94D3D26BE37EE480E0E4
:103B80000C94D3D260E47EE483E00C94D3D20F9300
:103B90001F9309EA15E02BEA35E046E858E16BEBA4
:103BA00075E080EC95E00E94CEC41F910F910895BE
:103BB0000F931F930CED14E02EE535E040EE5EE52B
:103BC0006EED74E083EE94E00E94CEC41F910F91DD
:103BD0000895CF92DF92EF92FF92CF93DF9300D0C0
:103BE00000D0CDB7DEB70E94B4E020E030E04AE775
:103BF00054E40E9427E820E030E0A9010E94A4E7F5
:103C00006B017C0120E030E0A9010E94ADE02DEBCA
:103C100037E346E055E387FF04C02DEB37E346E08A
:103C200055EBC701B6010E94A4E769837A838B83B1
:103C30009C83CE0101960E94ECBD0F900F900F90D7
:103C40000F90DF91CF91FF90EF90DF90CF9008958C
:103C500080915B01882341F0609168047091690450
:103C600041E081E00C94D6BC0895CF93DF93EC0142
:103C70000E94F6CB1B82DF91CF910895CF93DF9303
:103C8000EC01462F41706C857D858E859F850E9455
:103C9000C3C8882351F0888920E2829FC001112483
:103CA0008C509D4EDF91CF91089590E080E0FACF47
:103CB000CF93DF93EB01FC012381211104C080E04D
:103CC000DF91CF9108952250223028F48FE288832B
:103CD000198281E0F5CF60E00E943E1E009779F3E3
:103CE000DC0160E080E09EE22D91203299F0883086
:103CF00031F49E01260F311DF90190836F5F9E0103
:103D0000260F311DAD0141505109FA014081F901E1
:103D100040836F5F8F5F8B3039F7FE01E60FF11D37
:103D20001082D7CF3F924F925F926F927F928F9285
:103D30009F92AF92BF92CF92DF92EF92FF920F933A
:103D40001F93CF93DF93CDB7DEB72C970FB6F894C0
:103D5000DEBF0FBECDBF5C01DC0159968D909C90FB
:103D6000F40181859285A385B4859C01AD012F5F07
:103D70003F4F4F4F5F4F29873A874B875C87D5016D
:103D800014964D905D906D907C901797411451045E
:103D90006104710409F459C0BFEF4B1A5B0A6B0A46
:103DA0007B0A312C730162011D821E821F821886DC
:103DB000F40181859285A385B4852D813E814F8153
:103DC0005885281739074A075B0708F056C08985C8
:103DD0009A85AB85BC858C159D05AE05BF0550F455
:103DE00082E0C82ED12CE12CF12C92E0492E512CEE
:103DF000612C712C9E012F5F3F4FB701A601C401BA
:103E00000E94FDCA8823C9F189819A81AB81BC8156
:103E1000892B8A2B8B2B01F1260137019FEF491A41
:103E2000590A690A790A2D813E814F8158852F5F91
:103E30003F4F4F4F5F4F2D833E834F8358873FEF58
:103E4000C31AD30AE30AF30AB3CF408051806280D9
:103E5000738033243394A6CFC414D504E604F70446
:103E600011F70FEF1FEF2FEF3FE0B701A601C401DD
:103E70000E946BCA782E81111AC0712C872D2C9646
:103E80000FB6F894DEBF0FBECDBFDF91CF911F916B
:103E90000F91FF90EF90DF90CF90BF90AF909F90E9
:103EA0008F907F906F905F904F903F900895F501B5
:103EB0004481558166817781411551056105710500
:103EC00039F097018601C4010E946BCA8823A9F2C8
:103ED000D5011496CD92DD92ED92FC921797332086
:103EE00051F0D701C6010196A11DB11DF4018083D7
:103EF0009183A283B383F50185899689A789B08DC3
:103F0000892B8A2B8B2B09F0B9CFC58AD68AE78AF1
:103F1000F08E818180688183B1CF40E050E0BA01AA
:103F20000C9445CC4F925F926F927F92AF92BF926A
:103F3000CF92DF92EF92FF920F931F93CF93DF9375
:103F40001F92CDB7DEB78C017B015A01C22EDB0177
:103F500059968D919C91F801928F818FCB010E948F
:103F60008D1F712CF70180859185A285B3854189CC
:103F700052896389748984179507A607B70708F0E3
:103F800052C055E0B695A795979587955A95D1F764
:103F9000F82FFF70DF2ED70113968C91823010F42A
:103FA00080E0DBC041E050E0BE016F5F7F4FC701A2
:103FB0000E946DCD0197A1F7F70180859185A285BB
:103FC000B3854F96A11DB11D80879187A287B387C6
:103FD000F0E2DF9EB00111246C507D4E6115710539
:103FE000F9F2DB018C91882341F0853E09F04CC049
:103FF000772029F077247394B5CF71100EC080918B
:10400000F4149091F514A091F614B091F714F801FE
:1040100084879587A687B787D08ADB018C91811129
:10402000E9CF772473948C2D8274823409F0B8CF51
:10403000772009F4A2C0F801D08861E0C8010E948D
:104040003E1E009709F4ACCF20E2DC011D922A95B8
:10405000E9F72BE0F501DC0101900D922A95E1F7DB
:1040600021E238E2FC01318B208B40E058E0578799
:104070004687338B228B318F208F578B468B0E9444
:104080007AC8811109C08CCF4BE050E0C5010E9475
:10409000B9E9892B09F066CFF0E2DF9ED001112447
:1040A0009D012C503D4EF9018385817121F08C2DAD
:1040B000827109F001C1F801818D928D4091F41453
:1040C0005091F5146091F6147091F7144487558758
:1040D00066877787D08AFD01EC50FD4E448855886D
:1040E000712C612C320155244424D80155964D92EF
:1040F0005D926D927C925897428D538D70E060E096
:10410000442955296629772955964D935D936D93DA
:104110007C935897D9011B962C91287109F0BEC049
:10412000848D958DA68DB78DF801818B928BA38B95
:10413000B48B81E083838C2D8F70F801818314828E
:10414000158216821782108611861286138681E0E8
:10415000C4FE03C0C8010E94D9CC0F90DF91CF915B
:104160001F910F91FF90EF90DF90CF90BF90AF9095
:104170007F906F905F904F900895D70113968C9128
:104180001397823009F40CCF51968D919D910D902B
:10419000BC91A02D803E9F4FAF41B10508F000CFEC
:1041A000C7010E94921E882309F4FACE0E947AC8A1
:1041B000882309F4F5CED7015996ED91FC915A97D1
:1041C00014964D905D906D907C901797B2E04B1ACD
:1041D000510861087108858504C0440C551C661C93
:1041E000771C8A95D2F786859785A089B189480E74
:1041F000591E6A1E7B1E81E08093F8144092F414CD
:104200005092F5146092F6147092F714E4EFF2E114
:1042100080E092E0DF019C011D9221503040E1F7E7
:10422000DD24D394D7015996ED91FC918481D81661
:10423000C0F48091F9149091FA14DC01ED91FC9195
:104240000288F389E02D24EF32E1B301A2014D0D84
:10425000511D611D711D0995882309F4A1CED394C8
:10426000E1CF258580E092E0A0E0B0E004C0880FB7
:10427000991FAA1FBB1F2A95D2F7F70141895289BE
:1042800063897489840F951FA61FB71F818B928B3A
:10429000A38BB48B84EF92E1D12CD6CE203161F484
:1042A00098012F5E3F4F0E9480CB882329F084E045
:1042B000D80113968C933FCFD80113961C9270CEE1
:1042C000FC01238121110C94351E08952F923F92F9
:1042D0004F925F926F927F928F929F92AF92BF9216
:1042E000CF92DF92EF92FF920F931F93CF93DF93C2
:1042F000CDB7DEB7C354D1090FB6F894DEBF0FBEF9
:10430000CDBF4C015B016A01222E19821C821C8EDA
:104310001F8E6115710521F510E0CE014C960E94AB
:104320006021CE0101960E946021812FCD5BDF4F7D
:104330000FB6F894DEBF0FBECDBFDF91CF911F91B6
:104340000F91FF90EF90DF90CF90BF90AF909F9034
:104350008F907F906F905F904F903F902F90089537
:10436000FC0183818111D8CFFA0180818F32A1F1C4
:104370008B01CE0101967C013C0180E2382E2E019A
:104380009CE1490E511C2396EFAE23972496FFAE75
:10439000249722963FAE229721963FAE21973FAEBB
:1043A0003EAE3DAE3CAE3BAE3AAE39AE38AE3FAAC5
:1043B000960190E047E0D9018D91882309F447C028
:1043C0008F3209F444C08E3209F54A3009F4A4CF83
:1043D00098E04AE09D01EFCFFB01838182508B0181
:1043E000823060F0618D728DCE014C960E94B5D105
:1043F0008E01045E1F4F882309F48ECFC6016C0125
:104400000196F60120812F32D1F3B3CFEAE3F1E137
:104410002491222321F031968213FACF7DCF4917C0
:1044200008F47ACF813208F477CF8F3709F474CF4C
:104430003FE9380F3A3108F420EEE7E3F0E0EC0F03
:10444000FD1FE90FF11D820F80839F5FC3CF8FA9EE
:10445000803209F461CF6901F90180812F5F3F4FFC
:104460008F32C9F3882301F121E0AE01495C5F4F2F
:10447000B801C7010E94921F882309F44DCF0A1585
:104480001B0519F0C8010E94351E942D852D6E1450
:104490007F0431F023969FAD239724968FAD249708
:1044A0008701E92EF82E75CF222DAE01495C5F4FB2
:1044B000B801C4010E94921F182F2FCF8F929F9294
:1044C000AF92BF92CF92DF92EF92FF92CF936B01A8
:1044D0007C01B42E20E030E0A9010E94ADE087FF0E
:1044E00007C08DE20E94637AF7FAF094F7F8F0942F
:1044F000C0E060E070E080E09FE3CB1541F02DEC80
:104500003CEC4CEC5DE30E9413E1CF5FF6CFA701DA
:1045100096010E94A4E76B017C010E94A0E84B0178
:104520005C014AE00E9460C7CC2379F1C501B40167
:104530000E94B2E09B01AC01C701B6010E94A3E753
:104540006B017C018EE20E94637AC150F0F020E0A2
:1045500030E040E251E4C701B6010E9413E16B0173
:104560007C010E94A0E84B015C014AE00E9460C708
:10457000C501B4010E94B2E09B01AC01C701B601C4
:104580000E94A3E76B017C01E0CFCF91FF90EF90F9
:10459000DF90CF90BF90AF909F908F900895EF9253
:1045A000FF920F931F93CF937C018B01C2E44F3F87
:1045B00009F0C4E580E20E94637A8C2F0E94637A3E
:1045C0008AE30E94637AF70160817181828193811D
:1045D00042E00E945E228EE291E10E947B7AF80125
:1045E000608171818281938142E00E945E2262E05B
:1045F00070E080E090E0CF911F910F91FF90EF90DD
:104600000C9415C11F93CF93DF93CDB7DEB72897D6
:104610000FB6F894DEBF0FBECDBF182F60910B15FB
:1046200070910C15072E000C880B990B0E94B4E0BA
:104630006D837E838F8398876091091570910A1529
:10464000072E000C880B990B0E94B4E069837A83D3
:104650008B839C834AEFBE016B5F7F4FCE01019637
:104660000E94CF226091040670910506072E000C6F
:10467000880B990B0E94B4E06D837E838F839887AB
:104680006091020670910306072E000C880B990BAF
:104690000E94B4E069837A838B839C834FEFBE01D1
:1046A0006B5F7F4FCE0101960E94CF22609106067C
:1046B0001F3F39F085E11802F0011124EB5FFA4E3B
:1046C000608570E086E391E10E94267B609106069A
:1046D00070E081E391E10E94267B28960FB6F89462
:1046E000DEBF0FBECDBFDF91CF911F9108950F9315
:1046F0000FB70F9300916E000B7F00936E007894BC
:104700000F930BB70F930CB70F921F922F933F93FA
:104710004F935F936F937F938F939F93AF93BF93C9
:10472000EF93FF9311240E946129FF91EF91BF91B4
:10473000AF919F918F917F916F915F914F913F9139
:104740002F911F900F900CBF0F910BBF0F91046022
:10475000F89400936E000F910FBF0F911895CF93AF
:10476000DF93C5E0D5E11F821E820E94BCC118867E
:104770005D98CEEFD5E01F821E820E94D817188662
:104780005C98DF91CF9108954F925F926F927F92E4
:104790008F929F92AF92BF92EF92FF920F931F93CF
:1047A000CF93DF93B0E2A0E06A2F70E0AB014B0F34
:1047B000511D55954795411117C0E2E5F0E18591EE
:1047C0009491282F822FDF91CF911F910F91FF900D
:1047D000EF90BF90AF909F908F907F906F905F9081
:1047E0004F900895B42FE2CFA41711F0B41303C073
:1047F000EEECF0E1E4CF9A0121503109220F331F92
:10480000220F331FF901E05BFF4EE590F490F901B0
:10481000EC5AFF4E059114918E159F051CF3A42FA1
:10482000081719070CF4C0CFBC01F901EE5AFF4E6E
:10483000C591D491F901EA5AFF4EA590B4906E1932
:104840007F09072E000C880B990B0E94B4E02B0106
:104850003C01B5016C1B7D0B072E000C880B990BDE
:104860000E94B4E09B01AC01C301B2010E9413E1BC
:104870004B015C01B8016E197F09072E000C880BF3
:10488000990B0E94B4E09B01AC01C501B4010E94E8
:1048900027E84B015C01BE01DD0F880B990B0E94DC
:1048A000B4E09B01AC01C501B4010E94A4E70E94E1
:1048B00099E8262F972F86CFCF93DF93C5E0D5E1D8
:1048C0008A819B810E947EB69D838C83CEEFD5E04A
:1048D0008A819B810E94C4239D838C83A89510921A
:1048E000E802DF91CF910895EF92FF920F931F930B
:1048F000CF93C82F7B018A018091F9058130A1F403
:104900000E94307BC7010E947B7A86E090E10E9482
:104910007B7AC7FD20C08C2F0C2E000C990B0E94B7
:1049200016B78AE00E94637A0E94AF23A89580910F
:10493000FF04811115C081E08093FF0480E880931B
:10494000F9056BEF7FE0CF3F11F06FEF7FE040E0C4
:10495000C8010E94B27D82E090E10E947B7AE1CFA3
:10496000CF911F910F91FF90EF9008954F925F921A
:104970006F927F928F929F92AF92BF92CF92DF926F
:10498000EF92FF920F931F93CF93DF93EC016B0194
:104990004A01B22EFA014080518062807380A301E7
:1049A00092016D817E818F8198850E94ADE0882380
:1049B000A1F04D825E826F827886AA24A39420E0C3
:1049C00030E0A901F40160817181828193810E94AC
:1049D00027E918160CF0A12CAC828C818230A1F052
:1049E000833009F45AC08130C9F52D813E814F8151
:1049F0005885F60160817181828193810E94ADE0CA
:104A000087FD2CC082E08C83B701FF0C880B990BCB
:104A10000E94B4E09B01AC016D817E818F819885FD
:104A20000E94A3E79B01AC01F60160817181828144
:104A300093810E9427E987FD22C00E94B0C16B01CB
:104A40007C019801A8EEB3E00E9449E7C60ED71E8C
:104A5000E81EF91EC882D982EA82FB82DF91CF91DB
:104A60001F910F91FF90EF90DF90CF90BF90AF908C
:104A70009F908F907F906F905F904F9008950E94CD
:104A8000B0C1088119812A813B81601B710B820BA7
:104A9000930B97FDE3CF83E08C8340ED50E160EE14
:104AA00070E18B2DDF91CF911F910F91FF90EF90CF
:104AB000DF90CF90BF90AF909F908F907F906F903E
:104AC0005F904F900C947424CF93DF93EC01488156
:104AD00059816A817B8181EF9FE00E943D7F4C81FB
:104AE0005D816E817F8182E596E20E943D7F4885EF
:104AF00059856A857B858EE496E20E943D7F8AE037
:104B0000DF91CF910C94637ABC012091E004309145
:104B1000E1044091E0045091E1042417350731F499
:104B200081E02617370709F080E008959A01F1CF58
:104B30000F930FB70F9300916E000F930B7F0093AD
:104B40006E0000916F000D7F00936F000F930BB705
:104B50000F930CB70F921F922F933F934F935F9336
:104B60006F937F938F939F93AF93BF93EF93FF9335
:104B700011240E94EF2AFF91EF91BF91AF919F9175
:104B80008F917F916F915F914F913F912F911F90E6
:104B90000F900CBF0F910BBF0F910260F894009320
:104BA0006F000F9100936E000F910FBF0F9118953A
:104BB00000000000000000008091E80580FF27C091
:104BC000459A8FEF809396048091E805869580FF43
:104BD00021C0479A8FEF809397048091E8058695CE
:104BE000869580FF1AC02A988FEF80939804809151
:104BF000E80586958695869580FF12C0289A8FEFE6
:104C0000809399040000000000000000089545987A
:104C100081E0D8CF479881E0DECF2A9A81E0E5CFC6
:104C2000289881E0EDCFAF92BF92CF92DF92EF92C2
:104C3000FF920F931F93CF93DF93C9E6DBE00CE85D
:104C400016E089E7A82E8BE0B82EC12CD12C760176
:104C5000C39469917991899199910E94B2E02889D0
:104C600039894A895B890E9413E10E94A0E8F80112
:104C700061937193819391938F01C616D706E806CD
:104C8000F90610F46B017C01AC16BD0611F76FEF4D
:104C90007FEFCB01A70196010E94F5E620939C06C9
:104CA00030939D0640939E0650939F06DF91CF91CF
:104CB0001F910F91FF90EF90DF90CF90BF90AF903A
:104CC00008950F931F93CF93DF930DE71BE0C5EA81
:104CD000D6E0F80121913191419151918F0160E02D
:104CE00070E080E89FE30E9427E8699379938993B5
:104CF0009993F6E0C53BDF0761F70E941CB9DF918D
:104D0000CF911F910F910C9413260C9461260C9453
:104D100061260C9461260C9461269091B8158091BF
:104D2000B915981306C08091B6069091B706892BE5
:104D300019F00E944083F1CF08959091B8158091A9
:104D4000B915981308C08091B6069091B706892BC3
:104D500011F40C94E5770E944083EFCFCF93DF935B
:104D600020916B02222379F0EC010E94C8749B0110
:104D7000AC01688579858A859B850E94A3E7688751
:104D800079878A879B87DF91CF910895CF93DF93AF
:104D900020916B02222379F0EC010E94C8749B01E0
:104DA000AC01688579858A859B850E94A4E7688720
:104DB00079878A879B87DF91CF9108954F925F9281
:104DC0006F927F928F929F92AF92BF92CF92DF921B
:104DD000EF92FF920F931F93CF93DF93CDB7DEB780
:104DE0006A970FB6F894DEBF0FBECDBF9A8F898F3A
:104DF0005B018A01DC01D6966D917D918D919C912C
:104E0000D9970E94B2E06B017C01F50120813181CC
:104E1000428153810E9413E10E9410E82B013C0162
:104E2000D8012D913D914D915C91C701B6010E9431
:104E300013E10E9410E84B015C01C301B2010E9422
:104E4000A0E8698B7A8B8B8B9C8B68377105810509
:104E5000910540F428E730E040E050E0298B3A8BA0
:104E60004B8B5C8BC501B4010E94A0E86D877E87E7
:104E70008F87988B683771058105910540F488E725
:104E800090E0A0E0B0E08D879E87AF87B88BE98D7A
:104E9000FA8DEE5BFF4F208131814281538129835E
:104EA0003A834B835C83CA01B9010E94B4E02B01B1
:104EB0003C0169897A898B899C890E94B2E0698763
:104EC0007A878B879C8720E030E0A901C301B2017B
:104ED0000E94ADE0882309F43BC1A7019601C701F8
:104EE000B6010E9413E14B015C0129853A854B858F
:104EF0005C85CA01B9010E9413E19B01AC01C501A7
:104F0000B4010E94A3E74B015C01A3019201C3011C
:104F1000B2010E94A4E79B01AC01C501B4010E944B
:104F200027E80E9410E80E94A0E86D837E838F83AB
:104F3000988769817A818B819C8190958095709505
:104F400061957F4F8F4F9F4F0E94B4E04B015C01F2
:104F50006D857E858F8598890E94B2E069837A830A
:104F60008B839C8320E030E0A901C501B4010E943D
:104F7000ADE0882309F4F0C029813A814B815C813E
:104F8000CA01B9010E9413E16D8B7E8B8F8B988FC4
:104F9000A7019601C701B6010E9413E19B01AC0174
:104FA0006D897E898F89988D0E94A3E76B017C01B2
:104FB000A5019401C501B4010E94A4E79B01AC01C5
:104FC000C701B6010E9427E80E94CFE8A98DBA8DDB
:104FD00095968D909D90AD90BC90989775016401C9
:104FE0002D813E814F815885C21AD30AE40AF50A01
:104FF0000E94A0E8C61AD70AE80AF90AF7FE6EC0AE
:1050000020E030E0A901C301B2010E94ADE0882395
:1050100009F4A6C0C501B4010E94B2E06B017C0195
:10502000A3019201C301B2010E94A4E79B01AC015C
:10503000C701B6010E9413E16B017C0129853A8505
:105040004B855C85CA01B9010E9413E19B01AC014B
:10505000C701B6010E94A3E76B017C0129813A8157
:105060004B815C81CA01B9010E9413E19B01AC0133
:10507000C701B6010E94A4E76B017C0120E030E08B
:1050800040E850E4C301B2010E9413E19B01AC016E
:10509000C701B6010E9427E80E9410E86B017C015D
:1050A00020E030E0A9010E9427E918161CF0C12C6D
:1050B000D12C7601C701B6010E94A0E86D837E83E2
:1050C0008F83988786169706A806B90620F48D82E6
:1050D0009E82AF82B886C12CD12C76018D819E81B3
:1050E000AF81B885E98DFA8D81A792A7A3A7B4A750
:1050F000C80ED91EEA1EFB1EC5A6D6A6E7A6F0AAB4
:1051000029893A894B895C8922AF33AF44AF55AFC7
:10511000FE962D853E854F855889208331834283B5
:1051200053836A960FB6F894DEBF0FBECDBFDF91F2
:10513000CF911F910F91FF90EF90DF90CF90BF9094
:10514000AF909F908F907F906F905F904F90089559
:1051500060E070E0CB01E5CE60E070E0CB0134CFE1
:1051600060E070E0CB0198CF90916F0081E091FDFD
:1051700002C080E0089590916F009D7F90936F0032
:105180000895CF93C82F0E94B42894E0C99F90013E
:105190001124F901ED51FB4F21513B4FD9014D91A4
:1051A0005D916D917C91408351836283738391E023
:1051B0009093E204882319F0CF910C94A477CF91B7
:1051C0000895CF92DF92EF92FF928091E7058111CF
:1051D00005C080914606882309F46EC0809175044D
:1051E000329B64C081608093750480917504339B09
:1051F0005FC082608093750480917504349B5AC0AF
:10520000846080937504C090D304C0FE10C0809168
:10521000E80580FF0CC08091750480FF08C0809174
:10522000F80581608093F80580E00E94C128D12CA8
:10523000F12CE12CD701C601B695A79597958795D6
:1052400080FF11C08091E805869580FF0CC0809199
:10525000750481FF08C08091F80582608093F8058D
:1052600081E00E94C12882E0F694E794D794C79425
:105270008A95D1F7C0FE20C08091E8058695869575
:1052800080FF1AC0809146068823B1F08091750492
:1052900082FF12C08091F80584608093F80582E057
:1052A000FF90EF90DF90CF900C94C1288E7F9BCF22
:1052B0008D7FA0CF8B7FA5CFFF90EF90DF90CF9019
:1052C00008950F931F93CF93DF9380913E018F3703
:1052D00008F441C08F5790910D15909322059923A2
:1052E000C1F15D9A90910606909321059923E1F111
:1052F0005C9A8F5F80933E018091200591E0892721
:105300008093200581110E94261980913D01C1E002
:10531000C80F85300CF0C0E0823009F4CEC034F5FF
:105320008823D1F1813009F4BDC0C0933D010E94B2
:10533000E1288091B6069091B706009729F0019771
:105340009093B7068093B606DF91CF911F910F918E
:1053500008955D98C7CF90912205891708F05D9850
:1053600090912105891728F25C98C3CF843009F405
:10537000BBC00CF4B5C08530C1F690911F059111EA
:1053800002C080931F0580911F05815080931F05E7
:10539000882359F2C5E0C9CF80913C018F5F8031ED
:1053A0001CF480933C01C1CF10923C018091E80233
:1053B000811113C0809105159091061590930815E1
:1053C000809307158091FE059091FF05909301064B
:1053D0008093000681E08093E802109206151092F7
:1053E00005151092FF051092FE050091071510910A
:1053F000081580910B1590910C15D1E0181619061F
:105400002CF080910D15811101C0D0E080915401E4
:1054100090915501081719073CF440EF50E16DEFEA
:1054200070E180E00E947424DD2371F080915201CC
:1054300090915301801791073CF44FE051E16CE1EA
:1054400071E180E00E947424009104061091050629
:1054500020910006309101068091E4059091E505C8
:10546000281739073CF440EF50E16DEF70E18FEF02
:105470000E947424101611060CF057CF20910006DC
:10548000309101068091500190915101821793074C
:105490000CF04BCF4FE051E16CE171E18FEF0E94D6
:1054A000742443CF10927B0087E480937C0080912A
:1054B0007A00806480937A0038CF80917A0086FDEC
:1054C00026C0209178003091790080910515909147
:1054D0000615820F931F909306158093051525CF0F
:1054E00010927B0086E4E1CF80917A0086FD11C0A6
:1054F00020917800309179008091FE059091FF0510
:10550000820F931F9093FF058093FE050ECFC2E09C
:105510000CCFC4E00ACF0E94B4281092A0061092CB
:10552000A1061092A2061092A30681110C94A477F2
:1055300008950F931F938091B8159091B915891B09
:105540008F7009F449C09091B515992361F08330AB
:1055500040F48FEF890F29F08093B51590E080E03B
:1055600038C01092B5158091B9152BE4829FC00107
:1055700011248854994FFC01208120FDEFCF4091E8
:10558000A0065091A1066091A2067091A306E95B66
:10559000FF4F0081118122813381401B510B620B2F
:1055A000730B4093A0065093A1066093A2067093DC
:1055B000A3062091B9152F5F2F702093B615309157
:1055C000B9152091B715321304C02091B615209358
:1055D000B7151F910F9108950E948B2ABFCF2F926C
:1055E0003F924F925F926F927F928F929F92AF9273
:1055F000BF92CF92DF92EF92FF920F931F93CF93C0
:10560000DF9300D000D0CDB7DEB78FEF9FEF909340
:105610008900809388000AE00983312C212C78943A
:105620008091DC049091DD04A091DE04B091DF0450
:10563000892B8A2B8B2B09F0C4C18091E20488232B
:10564000E1F08091E0049091E1041092E204892B52
:1056500009F4B7C11092E1041092E0041092D3044F
:105660009091B8158091B915981709F4AAC1809145
:10567000B9158F5F8F708093B9158091E004909178
:10568000E104892B09F49DC14091D8045091D904BB
:105690006091DA047091DB048091D4049091D50478
:1056A000A091D604B091D7040091C60410E030E078
:1056B00020E0841B950BA60BB70B081719072A07C8
:1056C0003B0710F4D901C8018A83840F951FA61FD8
:1056D000B71F8093D8049093D904A093DA04B093B1
:1056E000DB04E1E0C0909E04D0909F04E090A00411
:1056F000F090A1048091AE049091AF04A091B00409
:10570000B091B104C80ED91EEA1EFB1EC092AE04B1
:10571000D092AF04E092B004F092B104F7FC33C031
:1057200040919604042E000C550B660B770B80916C
:10573000EF049091F004A091F104B091F204840F71
:10574000951FA61FB71F8093EF049093F004A093BA
:10575000F104B093F20480919A0490919B04A0917B
:105760009C04B0919D04A7019601281B390B4A0B9C
:105770005B0BDA01C9018093AE049093AF04A09350
:10578000B004B093B1040091A2041091A30420913D
:10579000A4043091A5048091B2049091B304A09127
:1057A000B404B091B504080F191F2A1F3B1F0093C2
:1057B000B2041093B3042093B4043093B50437FDBE
:1057C00033C080919704082E000C990BAA0BBB0BD9
:1057D0004091F3045091F4046091F5047091F60443
:1057E000840F951FA61FB71F8093F3049093F404B2
:1057F000A093F504B093F60480919A0490919B04D1
:10580000A0919C04B0919D04B901A801481B590BBB
:105810006A0B7B0BDB01CA018093B2049093B30443
:10582000A093B404B093B5044091A6045091A7048A
:105830006091A8047091A9048091B6049091B70476
:10584000A091B804B091B904480F591F6A1F7B1F7B
:105850004093B6045093B7046093B8047093B904AE
:1058600077FD33C080919804082E000C990BAA0B89
:10587000BB0B8090F7049090F804A090F904B090CE
:10588000FA04880D991DAA1DBB1D8093F7049093FF
:10589000F804A093F904B093FA0480919A049091CB
:1058A0009B04A0919C04B0919D042A013B01481ADD
:1058B000590A6A0A7B0AD301C2018093B604909305
:1058C000B704A093B804B093B9048090AA04909050
:1058D000AB04A090AC04B090AD048091BA04909158
:1058E000BB04A091BC04B091BD04880D991DAA1DF4
:1058F000BB1D8093BA049093BB04A093BC04B093E7
:10590000BD04B7FD33C040909904042C000C550829
:10591000660877088090FB049090FC04A090FD043A
:10592000B090FE04840C951CA61CB71C8092FB044E
:105930009092FC04A092FD04B092FE0480909A0420
:1059400090909B04A0909C04B0909D042C013D017C
:10595000481859086A087B08530142018092BA042A
:105960009092BB04A092BC04B092BD04E11104C0AB
:10597000E0918400F0918500F7FE5F9A37FF469A28
:1059800077FF2B9AB7FF299AE0918400F091850068
:10599000E0918400F0918500F7FE5F9837FF46980C
:1059A00077FF2B98B7FF29985A80552021F08091D6
:1059B0008400909185000A8101500A83E0E0011182
:1059C00091CE8090600190906101A0906201B090B2
:1059D000630181149104A104B10409F047C08091CE
:1059E0004B0690914C06009709F42FC023B1247008
:1059F00015980000000000000000181619060CF0B1
:105A0000D7C02A9A00000000000000002B9A34E062
:105A10003A950000E9F72B98000000000000000014
:105A2000222309F4C7C02A9A0000000000000000E9
:105A3000181619060CF0C0C080914B0690914C06C8
:105A4000019790934C0680934B060E94AA77882377
:105A500009F4B8C080ED97E0A0E0B0E08093600169
:105A600090936101A0936201B09363018091DC0483
:105A70009091DD04A091DE04B091DF04892B8A2B84
:105A80008B2B09F050C4E091E004F091E1043097D1
:105A900009F424C58091D8049091D904A091DA0426
:105AA000B091DB044091D4045091D5046091D604A8
:105AB0007091D70484179507A607B70708F486C026
:105AC0001092E1041092E0041092D3049091B81562
:105AD0008091B915981709F401C58091B9158F5FA8
:105AE0008F708093B91580EDC82E87E0D82EE12CF9
:105AF000F12C8091E0049091E104892B09F00BC412
:105B00000E94992A9093E1048093E004892B09F480
:105B100002C44090E0045090E1045C824B82D201C8
:105B20008C9183FFB3C2F201858D968DA78DB0A1B4
:105B3000418D528D638D748D058916892789308D2D
:105B40000093EF041093F0042093F1043093F204D7
:105B50004093F3045093F4046093F5047093F604B7
:105B60008093F7049093F804A093F904B093FA0497
:105B700081A192A1A3A1B4A18093FB049093FC0402
:105B8000A093FD04B093FE041092E1041092E0048F
:105B90001092D3049091B8158091B915981709F413
:105BA000AFCF8091B9158F5F8F708093B915A8CF53
:105BB0002A9828CF2A9838CF80914B0690914C068E
:105BC00001963FCF8FEF9FEFDC0148CF4091CF048C
:105BD0005091D0046091D1047091D20448175907B4
:105BE0006A077B0708F4DEC08091CB049091CC0457
:105BF000A091CD04B091CE0441A952A963A974A982
:105C00001127859F412C969F9001A69F300DA59F3F
:105C1000200D311D869F400C211D311F959F400C8A
:105C2000211D311FA49F400C211D311F949F410C49
:105C3000211F311F4694211F311F789F200D311DD8
:105C4000799F300D112442AD53AD64AD75AD420F57
:105C5000531F611D711D4093C7045093C804609386
:105C6000C9047093CA0406A917A920AD31AD041761
:105C700015072607370740F40093C7041093C8049C
:105C80002093C9043093CA044090C7045090C804BC
:105C90006090C9047090CA0421ED3FE001E00A83DE
:105CA000F901459155916591749144155505660525
:105CB000770570F476946794579447941A81110F7E
:105CC0001A832C5F3F4F4DEE5FE04217530741F7B9
:105CD0005A815093C60460E246165104610471046F
:105CE00028F410E2412E512C612C712C70E2471ADD
:105CF0005108610871084114E8E05E06610471040E
:105D000008F42EC0F4E05F9E900111242F52344F0E
:105D1000F901329645915491042DEE27059FB0016B
:105D2000049F610D7E1F06946E1F7E1F1124AB0120
:105D300070E060E0F901C590D490F12CE12CC41A18
:105D4000D50AE60AF70A8C0D9D1DAE1DBF1D809376
:105D5000CB049093CC04A093CD04B093CE04C9CED1
:105D6000B301A20176956795579547959A012C7FC7
:105D70002F52384FF901C590D490F90132964591D0
:105D80005491142D1770149F9001159F300D1124FC
:105D9000F3E036952795FA95E1F7C21AD30AF12C6C
:105DA000E12CD1CF4091C2045091C3046091C4044E
:105DB0007091C504481759076A077B0708F0D4C0DB
:105DC0008091BE049091BF04A091C004B091C10421
:105DD00041A952A963A974A92227859F312D969FB5
:105DE0008001A69F100DA59F000D111D869F300DEF
:105DF000011D121F959F300D011D121FA49F300D14
:105E0000011D121F949F310D021F121F3695021F94
:105E1000121F789F000D111D799F100D112430E085
:105E200020E04091C7045091C8046091C90470916A
:105E3000CA04FE9640805180628073800417150763
:105E40002607370758F4401B510B620B730B44169F
:105E500055066606770610F42A013B0121ED3FE066
:105E600041E04A83F901459155916591749144153A
:105E700055056605770570F47694679457944794B2
:105E80005A81550F5A832C5F3F4F6DEE7FE06217AA
:105E9000730741F77A817093C604E0E24E1651040D
:105EA0006104710428F400E2402E512C612C712C05
:105EB000F0E24F1A510861087108411408E05006D9
:105EC0006104710408F42EC014E0519E9001112465
:105ED0002F52344FF901329645915491F42DEE270B
:105EE000F59FB001F49F610D7E1F06946E1F7E1F0B
:105EF0001124AB0170E060E0F901C590D490F12C61
:105F0000E12CC41AD50AE60AF70A8C0D9D1DAE1DB8
:105F1000BF1D8093BE049093BF04A093C004B093B0
:105F2000C104E7CDB301A2017695679557954795D2
:105F30009A012C7F2F52384FF901C590D490F90166
:105F4000329645915491042D0770049F9001059F4E
:105F5000300D112413E0369527951A95E1F7C21AF2
:105F6000D30AF12CE12CD1CF8091380190913901E5
:105F7000A0913A01B0913B01B7FF5DC0C6A8D7A878
:105F8000E0ACF1AC81ED9FE021E0FC014591559141
:105F9000659174914C155D056E057F0558F4F69476
:105FA000E794D794C794220F04964DEE5FE048170C
:105FB000590759F72093C60450E2C516D104E104ED
:105FC000F10428F470E2C72ED12CE12CF12C60E210
:105FD000C61AD108E108F108C11478E0D706E10437
:105FE000F10408F431C0A4E0DA9EC00111248F52FC
:105FF000944FFC01329625913491BC2D6627B39FB6
:10600000A001B29F410D561F0694461F561F112432
:1060100070E060E0FC0185919491B0E0A0E0841B09
:10602000950BA60BB70B8093380190933901A09381
:106030003A01B0933B01C0903801D0903901E09013
:106040003A01F0903B0155CDD701C601B695A79511
:10605000979587958C7F8F52984FFC0125913491AD
:10606000FC01329645915491EC2DE770E49FC001FC
:10607000E59F900D112463E0969587956A95E1F769
:10608000281B390BC901B0E0A0E0CDCFAB81BC81AA
:1060900055960D911D912D913C91589781E00115D8
:1060A00011052105310509F480E0EB81FC81C18CEB
:1060B000D28CE38CF48CC114D104E104F10409F016
:1060C0008260AB81BC815D964D915D916D917C91BB
:1060D0009097411551056105710509F08460809321
:1060E000D3041092BE041092BF041092C004109208
:1060F000C1041092CB041092CC041092CD041092E3
:10610000CE04EB81FC8185A196A1A7A1B0A58093C7
:10611000D4049093D504A093D604B093D704442418
:1061200055243201481A590A6A0A7B0A4092AE0481
:106130005092AF046092B0047092B1044092B204E5
:106140005092B3046092B4047092B5044092B604C5
:106150005092B7046092B8047092B9044092BA04A5
:106160005092BB046092BC047092BD0441A052A046
:1061700063A074A0440C551C661C771C000F111FF3
:10618000221F331F00939E0410939F042093A004AA
:106190003093A104CC0CDD1CEE1CFF1CC092A204A9
:1061A000D092A304E092A404F092A504440F551FDA
:1061B000661F771F4093A6045093A7046093A8041A
:1061C0007093A9044092AA045092AB046092AC046C
:1061D0007092AD04880F991FAA1FBB1F80939A0469
:1061E00090939B04A0939C04B0939D041092D804B8
:1061F0001092D9041092DA041092DB0481A592A5C2
:10620000A3A5B4A58093CF049093D004A093D10408
:10621000B093D20485A596A5A7A5B0A98093C20482
:106220009093C304A093C404B093C50485A990912E
:10623000E805891721F08093E8050E94D8250E947F
:10624000E12844244A94542C32014092380150925F
:10625000390160923A0170923B01AB81BC81DA96C0
:106260004D915D916D917C91DD974093C704509362
:10627000C8046093C9047093CA0481ED9FE0A1E053
:10628000FC010591159125913491041715072607F6
:10629000370758F47695679557954795AA0F049652
:1062A000EDEEFFE0E817F90759F7A093C604403276
:1062B00051056105710520F440E250E060E070E0B6
:1062C00040525109610971094115F8E05F07610504
:1062D000710508F4DAC004E0509FC00111248F5208
:1062E000944FFC01329625913491AA27439FF001E7
:1062F000429FE10DFA1F0694EA1FFA1F1124AF0115
:1063000070E060E0FC01C590D490F12CE12CC41A3F
:10631000D50AE60AF70AC092DC04D092DD04E092C6
:10632000DE04F092DF0489288A288B28C9F4809142
:10633000DC049091DD04A091DE04B091DF048A3F7B
:106340009105A105B10560F42AEF30E040E050E08E
:106350002093DC043093DD044093DE045093DF048B
:1063600040916001509161016091620170916301FF
:106370000091DC041091DD042091DE043091DF04F3
:106380004F3F8FEF58076807780799F0D901C80188
:10639000B695A79597958795481759076A077B077C
:1063A00040F48093600190936101A0936201B093E7
:1063B00063014091600150916101609162017091AF
:1063C00063014F3F9FEF59076105710508F07DC0DC
:1063D0004B835A83F62FE72F8B819A81AF2FBE2FE5
:1063E000081719072A073B0710F4D901C801081B31
:1063F000190B2A0B3B0B0093DC041093DD04209354
:10640000DE043093DF044F3FEFEF5E076E077E0739
:1064100061F0481B590B6A0B7B0B40936001509352
:1064200061016093620170936301F894209184008C
:1064300030918500205F3F4F09810150098300237F
:1064400009F44AC0280E391E2216330610F40C94A3
:106450000F2B309289002092880078940F900F9033
:106460000F900F90DF91CF911F910F91FF90EF90C0
:10647000DF90CF90BF90AF909F908F907F906F9064
:106480005F904F903F902F900895DB01CA01B69521
:10649000A795979587958C7F8F52984FFC01C59053
:1064A000D490FC013296259134914770429FC001EF
:1064B000439F900D1124A3E096958795AA95E1F747
:1064C000C81AD90AF12CE12C26CFAFEFAB83BFEF6E
:1064D000BA83F0E0E0E080CF1901BBCF80EDC82E99
:1064E00087E0D82EE12CF12C0BCBFC0120813181EF
:1064F000428153816091890B70918A0B80918B0B43
:1065000090918C0B0E9413E10E942CE96093C615B8
:106510007093C7158093C8159093C9159091B815BD
:106520008091B91598130C94321D0E948D260E94FB
:10653000B4284091C6155091C7156091C815709147
:10654000C9154093FB045093FC046093FD047093C1
:10655000FE0481110C94A47708954F925F926F927C
:106560007F928F929F92AF92BF92CF92DF92EF92E3
:10657000FF920F931F93CF93DF93EC018B015A018E
:10658000F9012091890B30918A0B40918B0B50912E
:106590008C0B60817181828193810E9413E10E9442
:1065A0002CE96B017C012091850B3091860B409189
:1065B000870B5091880BF5016081718182819381F5
:1065C0000E9413E10E942CE94B015C012091810B98
:1065D0003091820B4091830B5091840BF8016081C4
:1065E0007181828193810E9413E10E942CE92B0129
:1065F0003C0120917D0B30917E0B40917F0B50919F
:10660000800B688179818A819B810E9413E10E94BD
:106610002CE96093BA157093BB158093BC159093C9
:10662000BD154092BE155092BF156092C015709274
:10663000C1158092C2159092C315A092C415B09254
:10664000C515C092C615D092C715E092C815F09234
:10665000C9159091B8158091B915981791F0DF91EF
:10666000CF911F910F91FF90EF90DF90CF90BF904F
:10667000AF909F908F907F906F905F904F900C9411
:10668000321D0E948D260E94B4284091C21550915F
:10669000C3156091C4157091C5150091BE15109178
:1066A000BF152091C0153091C115C090BA15D0907A
:1066B000BB15E090BC15F090BD15C092EF04D092D0
:1066C000F004E092F104F092F2040093F3041093CA
:1066D000F4042093F5043093F6044093F7045093A8
:1066E000F8046093F9047093FA044091C615509130
:1066F000C7156091C8157091C9154093FB0450935C
:10670000FC046093FD047093FE04882391F0DF91F4
:10671000CF911F910F91FF90EF90DF90CF90BF909E
:10672000AF909F908F907F906F905F904F900C9460
:10673000A477DF91CF911F910F91FF90EF90DF90A1
:10674000CF90BF90AF909F908F907F906F905F9011
:106750004F900895CF92DF92EF92FF92CF93DF9305
:10676000C82F0E94B42894E0C99FE0011124FE01C3
:10677000E151FB4FC080D180E280F38081110E9403
:10678000A477CB55D94FC701B6010E94B4E0288148
:1067900039814A815B810E9413E1DF91CF91FF90A3
:1067A000EF90DF90CF900895CF92DF92EF92FF921B
:1067B000CF93DF93C82F0E94B42894E0C99FE001D3
:1067C0001124FE01ED51FB4FC080D180E280F380A7
:1067D00081110E94A477CB55D94FC701B6010E9401
:1067E000B4E0288139814A815B810E9413E1DF9105
:1067F000CF91FF90EF90DF90CF900895CF930E94BC
:10680000B428C82F8091B9158093B8158093B71517
:106810008093B61584E68093B5150E948B2A80ED8F
:1068200093E09093B7068093B606C1110E94A477B7
:1068300081E08093E204CF910895CF93DF9324E029
:10684000829FC0011124EC01C25AD94FFC01E651CC
:10685000FA4F855A9D4FDC012D913D914D915C91F0
:1068600060817181828193810E94A4E7688379832A
:106870008A839B83DF91CF91089580FF04C090911C
:10688000880490FD8E7F81FF05C0909188049695C5
:1068900090FD8D7F82FF06C0909188049695969515
:1068A00090FD8B7F0895EF92FF920F931F93CF93EC
:1068B000DF93CDB7DEB762970FB6F894DEBF0FBE99
:1068C000CDBF0E943D34882309F43FC04FE352E01E
:1068D00082FF02C04CE352E02FE332E081FF02C0AE
:1068E00025E232E080FD2EC08FE392E05F934F936C
:1068F0003F932F939F938F938AE097E09F938F937B
:106900008E010F5F1F4F1F930F930E9444E00E9460
:10691000347BC8010E946A7AC8010E943FB80FB652
:10692000F894DEBF0FBECDBF81E062960FB6F8943B
:10693000DEBF0FBECDBFDF91CF911F910F91FF90B2
:10694000EF90089587E292E0D1CF80E0EECF809182
:10695000840490918504A0918604B091870480936B
:10696000180190931901A0931A01B0931B01809113
:1069700082049091830490931701809316010895E7
:106980008091180190911901A0911A01B0911B01F9
:106990008093840490938504A0938604B093870425
:1069A0008091160190911701909383048093820443
:1069B00084E690E0909317018093160108954F921A
:1069C0005F926F927F928F929F92AF92BF92CF927F
:1069D000DF92EF92FF920F931F93CF93DF93CDB788
:1069E000DEB72C970FB6F894DEBF0FBECDBF2B01DC
:1069F0003C0129873A874B875C8747015801F6019C
:106A0000E080F1800281138120E030E0A901B7012C
:106A1000C8010E94ADE0882309F488C05E2D4F2D87
:106A2000302F212F852F942FA32FB22F89839A8364
:106A3000AB83BC8320E030E0A901B701C8010E940C
:106A4000ADE0811108C0E0905C01F0905D01009123
:106A50005E0110915F01C701D8018D839E83AF83D2
:106A6000B887A501940160917406709175068091B4
:106A70007606909177060E94ADE087FF0CC0809269
:106A8000740690927506A0927606B0927706CE01B3
:106A900001960E946A1D40926C0650926D066092AB
:106AA0006E0670926F0689859A85AB85BC8580934A
:106AB000700690937106A0937206B0937306CE0190
:106AC00005960E946A1DA50194016091740670915B
:106AD000750680917606909177060E9427E9181630
:106AE00064F48092740690927506A0927606B09235
:106AF0007706CE0101960E946A1D0E948D262C9673
:106B00000FB6F894DEBF0FBECDBFDF91CF911F91BE
:106B10000F91FF90EF90DF90CF90BF90AF909F903C
:106B20008F907F906F905F904F90089550E040E07D
:106B300030E820E477CFCF92DF92EF92FF920F936D
:106B40001F936A01E0907406F09075060091760636
:106B500010917706FB012081318142815381FC0134
:106B600060817181828193810E94DF341F910F9136
:106B7000FF90EF90DF90CF900895CF92DF92EF9249
:106B8000FF920F931F936B01FC01E080F180028163
:106B90001381ECE6F6E024813581468157816081DE
:106BA0007181828193810E94DF341F910F91FF9048
:106BB000EF90DF90CF900895AF92BF92CF92DF9287
:106BC000EF92FF920F931F93CF93DF9300D000D0EB
:106BD000CDB7DEB7FC01E080F18002811381611145
:106BE00012C0A0907406B0907506C0907606D09042
:106BF00077069501A601B701C8010E94ADE087FFA5
:106C000002C07501860120E030E04AE753E4B70195
:106C1000C8010E94ADE087FD04C0E12CF12C0AE719
:106C200013E4C701D80189839A83AB83BC8363ECE7
:106C300071E0CE0101960E94BD350F900F900F902C
:106C40000F90DF91CF911F910F91FF90EF90DF9008
:106C5000CF90BF90AF9008958F929F92AF92BF92C6
:106C6000CF92DF92EF92FF921F93CF93DF93CDB736
:106C7000DEB760970FB6F894DEBF0FBECDBF182FFA
:106C800080E00E94AA334B015C01809276049092CE
:106C90007704A0927804B092790481E00E94AA332C
:106CA0006B017C01C0927A04D0927B04E0927C0458
:106CB000F0927D0482E00E94AA3360937E04709378
:106CC0007F0480938004909381041D861E861F8616
:106CD000188A89829A82AB82BC82CD82DE82EF8260
:106CE000F88669877A878B879C8783E00E94AA331E
:106CF0006D877E878F87988BCE0101960E94AE2686
:106D00001E3FD9F480E1FE013196ACE6B6E0019079
:106D10000D928A95E1F760960FB6F894DEBF0FBE2C
:106D2000CDBFDF91CF911F91FF90EF90DF90CF907B
:106D3000BF90AF909F908F90089584E0189FF001CE
:106D40001124DF01A459B94F81E090E08C0F9D1F01
:106D5000E80FF91F40815181628173814D935D93EA
:106D60006D937C931397D7CF0C941CB92F923F92BD
:106D70004F925F926F927F928F929F92AF92BF924B
:106D8000CF92DF92EF92FF920F931F93CF93DF93F7
:106D9000CDB7DEB76C970FB6F894DEBF0FBECDBF90
:106DA0008091E702811151C18091E60281113CC1BD
:106DB0008091E802811119C06C960FB6F894DEBF7D
:106DC0000FBECDBFDF91CF911F910F91FF90EF903C
:106DD000DF90CF90BF90AF909F908F907F906F90FB
:106DE0005F904F903F902F9008950E945C240E94E6
:106DF000B0C14B015C010091091510910A158091F9
:106E0000580190915901801791070CF449C2609183
:106E10000B1570910C15072E000C880B990B0E9416
:106E2000B4E06D837E838F839887B801110F880B40
:106E3000990B0E94B4E069837A838B839C832AE058
:106E4000E22EF12C0CE310E020E0AE014B5F5F4F2F
:106E5000BE016F5F7F4F8DE695E10E94B6240091E1
:106E6000091510910A1580915601909157018017CC
:106E700091070CF4F1C060E060930D15809101154D
:106E800090910215A0910315B09104150097A105EA
:106E9000B10539F1A5019401281B390B4A0B5B0B95
:106EA000DA01C901B7FD1DC08091FF149091001552
:106EB000081719070CF414C280910B1590910C154A
:106EC000009739F00E5F1F4F0497081719070CF44D
:106ED0001DC2109201151092021510920315109206
:106EE00004158091020690910306873991050CF0F4
:106EF000E3C180911B0590911C05A0911D05B091E7
:106F00001E050097A105B10561F1A5019401281B9B
:106F1000390B4A0B5B0BDA01C901B7FD22C0809126
:106F20000206909103062091190530911A058217E7
:106F300093070CF4CDC1209104063091050621156C
:106F4000310539F0029624503109821793070CF469
:106F5000F0C110921B0510921C0510921D05109295
:106F60001E058091150590911605A0911705B09109
:106F70001805A5019401281B390B4A0B5B0BDA019C
:106F8000C901B7FD19CF38E8830E33E1931EA11C68
:106F9000B11C8092150590921605A0921705B0922B
:106FA00018056091040670910506072E000C880BE9
:106FB000990B0E94B4E06D837E838F8398876091E4
:106FC000020670910306072E000C880B990B0E9495
:106FD000B4E069837A838B839C8382E0E82EF12C72
:106FE00002E310E02FEFAE014B5F5F4FBE016F5F1A
:106FF0007F4F86E795E10E94B6248091020690912A
:1070000003069C01255031092239310508F05CC185
:107010002091040630910506821793070CF468C18D
:1070200080E080930606C8CE1092E6020E94FE33EE
:107030000E948D268EEF0E942C360E94B4368091DD
:10704000E802882309F4B8CED0CE41E070E060E0D9
:1070500082E490E10E94B27D8091580190915901A3
:10706000081719070CF007CFE0900B15F0900C15DE
:10707000B801012E000C880B990B0E94B4E01B0193
:107080002C01E114F10409F43CC1B701601B710B40
:10709000072E000C880B990B0E94B4E06B017C0159
:1070A00020E030E040E251EC0E94ADE087FD29C1D4
:1070B00020E030E040E251E4C701B6010E9427E938
:1070C00018160CF449C180911405811149C1209111
:1070D0000C0530910D0540910E0550910F05298743
:1070E0003A874B875C878091100590911105A0919C
:1070F0001205B09113058D879E87AF87B88BA201CB
:1071000091016091000570910105809102059091B7
:1071100003050E94A3E720911615309117154091A1
:107120001815509119150E9413E129853A854B8550
:107130005C850E94A3E720ED3CEC4CE45DE30E94FB
:1071400013E129853A854B855C850E94A4E7698B0C
:107150007A8B8B8B9C8B60930C0570930D058093C1
:107160000E0590930F052091121530911315409143
:107170001415509115152D8B3E8B4F8B588F2D85E7
:107180003E854F855889C701B6010E94A4E7762E37
:10719000672E89879D8720E030E0A9010E94ADE03D
:1071A00087FDE9C02D893E894F89588D60E070E0E8
:1071B0008FE793E40E9427E8698F7A8F8B8F9C8FEB
:1071C000272D362D49855D850E94ADE087FF06C0DD
:1071D000798C6A8C3B8D39874C8D4D87872D962D08
:1071E000A985BD858093100590931105A093120584
:1071F000B093130520910E1530910F154091101585
:1072000050911115C701B6010E9413E16B017C0179
:10721000C0920405D0920505E0920605F09207059C
:10722000272D362D49855D856D897E898F89988DBD
:107230000E9413E19B01AC012093080530930905DE
:1072400040930A0550930B05C701B6010E94A4E7BD
:1072500029893A894B895C890E94A4E720E030E0C3
:10726000A9010E94A4E76B017C0120E030E0A901A4
:107270000E94ADE087FD48C020E030E04FE753E4D6
:10728000C701B6010E9427E91816A4F56FE72092FE
:107290000005309201054092020550920305ECCDA5
:1072A00040EF50E16DEF70E180E00E9474240091A6
:1072B000091510910A15ABCD40EF50E16DEF70E16B
:1072C0008FEF0E94742415CE109206065C9874CD40
:1072D00044E250E163E370E18FEF0E94742441CEF9
:1072E00044E250E163E370E180E00E947424F9CD50
:1072F0008FE797CEC701B6010E9499E8759567950B
:10730000C6CF81E08093140560E0C1CF10930015D3
:107310000093FF140E94B0C1605B7C438F4F9F4F6E
:1073200060930115709302158093031590930415D3
:10733000D8CD90931A05809319050E94B0C1605E64
:1073400070448D4F9F4F60931B0570931C05809375
:107350001D0590931E0505CE81E08093140596CF00
:10736000109214051D861E861F86188A19861A8695
:107370001B861C86C4CE712C612C19861D862ECFCF
:107380002F923F924F925F926F927F928F929F9235
:10739000AF92BF92CF92DF92EF92FF920F931F9323
:1073A000CF93DF93CDB7DEB7A6970FB6F894DEBFC5
:1073B0000FBECDBF80911E01882309F4CDC08091FE
:1073C0008804C82ED12CF12CE12C80FF3CC0809089
:1073D000200190902101A0902201B09023012091E2
:1073E0004B0230914C0240914D0250914E02C5012A
:1073F000B4010E9427E9181644F480924B0290923F
:107400004C02A0924D02B0924E0280902C019090BE
:107410002D01A0902E01B0902F0120914B023091B0
:107420004C0240914D0250914E02C501B4010E94A0
:10743000ADE087FF08C080924B0290924C02A09270
:107440004D02B0924E02D701C601B695A795979509
:10745000879580FF3CC08090240190902501A090EA
:107460002601B090270120914F02309150024091A7
:10747000510250915202C501B4010E9427E9181629
:1074800044F480924F0290925002A0925102B09226
:1074900052028090300190903101A0903201B09062
:1074A000330120914F02309150024091510250918E
:1074B0005202C501B4010E94ADE087FF08C080926E
:1074C0004F0290925002A0925102B092520292E06A
:1074D000F694E794D794C7949A95D1F7C0FE3CC030
:1074E000C0902801D0902901E0902A01F0902B0152
:1074F000209153023091540240915502509156020E
:10750000C701B6010E9427E9181644F4C09253023D
:10751000D0925402E0925502F0925602C09034018B
:10752000D0903501E0903601F09037012091530260
:10753000309154024091550250915602C701B60154
:107540000E94ADE087FF08C0C0925302D09254025F
:10755000E0925502F09256028091680B83FD7EC046
:10756000209178063091790640917A0650917B06F9
:1075700060915702709158028091590290915A027D
:107580000E94ADE0882309F469C01091B50611117D
:1075900061C080916801909169010197209109155E
:1075A00030910A15281739073CF40E94347B8FEE7E
:1075B00096E00E947B7A11E020917806309179065E
:1075C00040917A0650917B06609157027091580263
:1075D0008091590290915A020E94A3E76B017C01AD
:1075E00020E030E0A9010E9427E987FF04C0F7FAF4
:1075F000F094F7F8F0942091640130916501409186
:10760000660150916701C701B6010E9413E120E0B5
:1076100030E84BE354E40E9427E91816ECF40E948A
:10762000347B80ED96E00E947B7A809157029091A6
:107630005802A0915902B0915A0280937806909313
:107640007906A0937A06B0937B0687E592E00E94C4
:10765000753204C010E0B0CF1111E7CF2AE037ED4A
:1076600043E25CE3609118017091190180911A0165
:1076700090911B010E9413E16B017C016091160146
:1076800070911701072E000C880B990B0E94B4E033
:107690009B01AC01C701B6010E9413E1698B7A8B93
:1076A0008B8B9C8B80916B02882309F46CC020919A
:1076B0006C0630916D0640916E0650916F06609198
:1076C0004B0270914C0280914D0290914E020E94AB
:1076D000A3E76D8B7E8B8F8B988F209170063091F6
:1076E0007106409172065091730660914F0270913D
:1076F000500280915102909152020E94A3E7698F3B
:107700007A8F8B8F9C8F20917406309175064091F3
:1077100076065091770660915302709154028091E1
:107720005502909156020E94A3E76D8F7E8F8F8F36
:1077300098A3209178063091790640917A0650916D
:107740007B06609157027091580280915902909186
:107750005A020E94A3E76B017C0120E030E0A901FE
:107760006D897E898F89988D0E94ADE081110FC04F
:1077700020E030E0A901698D7A8D8B8D9C8D0E946F
:10778000ADE0811104C0C12CD12C76012CC12D8912
:107790003E894F89588DCA01B9010E9413E14B01FE
:1077A0005C01298D3A8D4B8D5C8DCA01B9010E9417
:1077B00013E19B01AC01C501B4010E94A4E74B0198
:1077C0005C012D8D3E8D4F8D58A1CA01B9010E94DB
:1077D00013E19B01AC01C501B4010E94A4E74B0178
:1077E0005C01A7019601C701B6010E9413E19B014C
:1077F000AC01C501B4010E94A4E70E9465E94B01F8
:107800005C012DEB37E346E855E30E94ADE087FFCE
:107810000FC020E030E0A901C701B6010E9427E9AE
:107820004601570187FF04C0B7FAB094B7F8B09487
:107830002DEB37E346E855E3C501B4010E94ADE006
:1078400087FDDEC020E030E040EA51E4C501B4012C
:107850000E9427E80E94A0E81B01672B19F422244C
:107860002394312CB10190E080E00E94B2E09B01B2
:10787000AC0160E070E080E89FE30E9427E82B0104
:107880003C01AC019B01C501B4010E9413E14B0115
:107890005C01A30192016D897E898F89988D0E9478
:1078A00013E16D8B7E8B8F8B988FA3019201698D75
:1078B0007A8D8B8D9C8D0E9413E1698F7A8F8B8FCF
:1078C0009C8FA30192016D8D7E8D8F8D98A10E945A
:1078D00013E16D8F7E8F8F8F98A3A3019201C70153
:1078E000B6010E9413E169A37AA38BA39CA380E154
:1078F000ECE6F6E08E010F5F1F4FD80101900D926C
:107900008A95E1F70E94B0C12B013C0128EC420EA0
:10791000511C611C711C0DA31EA381E0281A3108A3
:1079200009F45FC00E94B0C18B019C0104191509C4
:107930002609370937FD86C02B013C0128EC420E91
:10794000511C611C711C0E9440832D893E894F8906
:10795000588D69817A818B819C810E94A4E769831B
:107960007A838B839C83298D3A8D4B8D5C8D6D81C1
:107970007E818F8198850E94A4E76D837E838F83AB
:1079800098872D8D3E8D4F8D58A169857A858B8581
:107990009C850E94A4E769877A878B879C8729A1A9
:1079A0003AA14BA15CA16D857E858F8598890E9447
:1079B000A4E76D877E878F87988B750164018E01A0
:1079C0000F5E1F4F9E01235F3F4FAE01475F5F4F2A
:1079D000BE016B5F7F4F8DA19EA10E94BAB881113D
:1079E0009CCF750164018E010F5E1F4F27E532E0C9
:1079F00043E552E06FE472E08BE492E00E94BAB893
:107A000080E1EBE4F2E0ACE6B6E001900D928A95FD
:107A1000E1F7A6960FB6F894DEBF0FBECDBFDF919B
:107A2000CF911F910F91FF90EF90DF90CF90BF907B
:107A3000AF909F908F907F906F905F904F903F900E
:107A40002F9008950E94B63680CFCF930E94BD3507
:107A50008091F805C82FC47082FD0CC01092F80503
:107A600082E00E942C360E94B43681E0C11180E091
:107A7000CF9108950E94267D882381F3F9CFCF937B
:107A8000DF93CDB7DEB72C970FB6F894DEBF0FBEED
:107A9000CDBF0E9498B90E94B4289CE0EFEEF4E0BC
:107AA000DE01119601900D929A95E1F781110E94E5
:107AB000A477CE0101960E9464252C960FB6F89407
:107AC000DEBF0FBECDBFDF91CF9108952F923F92C1
:107AD0004F925F926F927F928F929F92AF92BF92DE
:107AE000CF92DF92EF92FF920F931F93CF93DF938A
:107AF00000D01F92CDB7DEB780906C0690906D06D7
:107B0000A0906E06B0906F0640907006509071067F
:107B10006090720670907306C0907406D0907506DF
:107B2000E0907606F09077060E9413260E943E149D
:107B300001E717E080E291E09B838A8385E6282EA7
:107B400087E0382E198289810E941D34C8010E9465
:107B50008673EA81FB816193719381939193FB8397
:107B6000EA83C1010E948673EA81FB816087718785
:107B700082879387F981FF5FF9830C5F1F4F84E051
:107B8000280E311CF330F9F60E9447770E946126D7
:107B9000A501940160916C0670916D0680916E064E
:107BA00090916F060E94ADE081111CC0A30192016B
:107BB00060917006709171068091720690917306C3
:107BC0000E94ADE081110EC02091740630917506BF
:107BD0004091760650917706C701B6010E94ADE04C
:107BE0008823B9F00F900F900F90DF91CF911F91E4
:107BF0000F91FF90EF90DF90CF90BF90AF909F904C
:107C00008F907F906F905F904F903F902F900C944B
:107C10003F3D0F900F900F90DF91CF911F910F91EB
:107C2000FF90EF90DF90CF90BF90AF909F908F909C
:107C30007F906F905F904F903F902F9008952F927C
:107C40003F924F925F926F927F928F929F92AF92EC
:107C5000BF92CF92DF92EF92FF920F931F93CF9339
:107C6000DF93CDB7DEB7C358D1090FB6F894DEBFA6
:107C70000FBECDBFCDB6DEB641E064E070E0CE0110
:107C800087589F4F0E9462B941E062E070E0CE01E8
:107C900083589F4F0E9462B943E050E0BE0167588D
:107CA0007F4F8BEC91E00E9406EA892B31F181E055
:107CB000809395049091950481E089270FB6F894FC
:107CC000DEBE0FBECDBECD57DF4F0FB6F894DEBF80
:107CD0000FBECDBFDF91CF911F910F91FF90EF901D
:107CE000DF90CF90BF90AF909F908F907F906F90DC
:107CF0005F904F903F902F900895E9961CAE1DAE77
:107D00001EAE1FAEE99710921B1510921A15CE01E8
:107D10008F579F4F0E940F1DADB6BEB6CF57DF4F96
:107D20000881C158D04010E00D5F1F4F000F111F98
:107D3000000F111F8DB79EB7801B910B0FB6F894E3
:107D40009EBF0FBE8DBFEDB7FEB73196CE57DF4F4A
:107D5000F983E883C258D040801B910B0FB6F8948A
:107D60009EBF0FBE8DBFEDB7FEB731964F01801B92
:107D7000910B0FB6F8949EBF0FBE8DBFEDB7FEB747
:107D800031967F01B801CE57DF4F88819981C25863
:107D9000D0400E94141D4091E50281E0482764E034
:107DA00070E089E79BE00E9462B9B801C4010E94BB
:107DB000141DB801C7010E94141D1091E502111194
:107DC00053C0CF57DF4F8881C158D04090E0029612
:107DD000A9E6BBE070E060E030E020E04DEC57E069
:107DE000821793070CF498C0CE57DF4FE881F981D2
:107DF000C258D040E60FF71F4080518062807380E8
:107E00004D925D926D927D92821793070CF48AC019
:107E1000F401E60FF71F208031800281E381210108
:107E2000602E7E2E50964D925D926D927C9253976D
:107E3000821793070CF480C0F701E60FF71F20802C
:107E400031800281E3812101602E7E2E90964D9239
:107E50005D926D927C9293972F5F3F4F6C5F7F4F47
:107E60002430310509F0BCCF8DE99BE00E94DF1C76
:107E700081EA9BE00E94DF1C85EA9BE00E94DF1CF8
:107E800089EA9BE00E94DF1C8DEA9BE00E94DF1CD8
:107E900041E0412760E170E08CE796E00E9462B922
:107EA000CE018B589F4F0E94DF1C0FB6F894BEBEC8
:107EB0000FBEADBE8AEE95E00E94071DCE0183592C
:107EC0009F4F0E94E71C8E010F5F1F4FC8010E9449
:107ED000DF1CCE018B589F4F0E94DF1CCE018B58B8
:107EE0009F4F0E94DF1CC8010E940F1DCE018359C5
:107EF0009F4F0E940F1DE980AE968FADAE97E89E12
:107F000070011124F1E0EF1AF10800F1CE018B5855
:107F10009F4F0E94DF1CF6CFFA0145905590659067
:107F200074906ECFEDEBF7E04590559065907490AE
:107F30001201062DE72D73CFEDEAF7E0459055903D
:107F4000659074901201062DE72D7DCF87EA95E1AB
:107F50000E94071D8AE0F82EFA94CE01FF2029F036
:107F60008B589F4F0E94DF1CF7CF81589F4F0E9474
:107F70000F1DCE0180589F4F0E940F1DC158DF4F2B
:107F80008881CF57D040853009F049C1C058DF4FB4
:107F90008881C058D040853009F041C18091E50208
:107FA000811102C00E94B5768DED92E00E94FF1C07
:107FB00085ED92E00E94FF1C4091E50281E0482798
:107FC00064E670E081E792E00E9462B9C8010E9415
:107FD000F71CCE0183599F4F0E94E71C4091E50298
:107FE000FF24F3944F2564E070E0C8010E9462B959
:107FF00089EE95E00E94F71C4091E5024F256CE068
:1080000070E087E096E00E9462B94091E5024F255A
:1080100064E170E0C8010E9462B9F090E502F110DD
:1080200038C089809A80AB80BC80A5019401C501CD
:10803000B4010E94A5E981112CC080920E15909286
:108040000F15A0921015B09211152CEA35EC47E2ED
:108050005EE36D817E818F8198850E9413E160933C
:1080600012157093131580931415909315152CEA1F
:1080700035EC47E25EE369857A858B859C850E94B5
:1080800027E8609316157093171580931815909331
:108090001915C8010E94EF1CC8010E94D71CC80115
:1080A0000E94D71CC8010E94E71CC8010E94EF1C57
:1080B00085E0F80111928A95E9F7EE24E3944F2DBB
:1080C0004E2565E070E0C8010E9462B9C8010E94B7
:1080D000F71C4091E5024E2560E270E0C8010E9465
:1080E00062B9CE0183599F4F0E94F71C4091E5026F
:1080F0004E2569E070E0C8010E9462B94091E50236
:1081000041110FC08981809370028A819B81AC816B
:10811000BD8180936C0290936D02A0936E02B09328
:108120006F02FF24F3944F2560E270E0C8010E94C3
:1081300062B94091E5024F2560E470E0C8010E94F9
:1081400062B94091E5024F2560E170E0C8010E94EC
:1081500062B94091E5024F2560E170E0C8010E94DC
:1081600062B9C8010E94DF1C4091E5024F256CE016
:1081700070E0C8010E9462B94091E5024F256CE6AB
:1081800070E0C8010E9462B919821A821B821C82A7
:108190001D821E821F82188619861A861B861C86DF
:1081A000C8010E94D71C4091E5024F2568E070E0AD
:1081B000C8010E9462B94091E5024F256CE070E071
:1081C000C8010E9462B9CE0181589F4F0E94E71CEE
:1081D000CE0183599F4F0E94DF1C80916A069091C7
:1081E0006B068134934069F41092950420911A151E
:1081F00030911B15EF968EAD9FADEF97281739077D
:1082000019F081E0809395048091E502811152CDAF
:108210008091950481114ECD0E94663D4BCDC801E1
:108220000E94FF1CCE0183599F4F0E94FF1CC15822
:10823000DF4FE880CF57D040C058DF4F8881C0580B
:10824000D040E89E7001112481E0E81AF10808F49A
:10825000BDCECE018B589F4F0E94DF1CF5CF84E628
:1082600090E090936B0680936A0610921B15109213
:108270001A150C941F3ECF93DF9300D000D0CDB7DA
:10828000DEB784EF91E0A0E0B0E089839A83AB830E
:10829000BC83BE016F5F7F4F8CE30E94197986EB30
:1082A00096E00E947B7A86B160EB76E082FB8827BD
:1082B00080F90E94BE1C86B16AEA76E083FB8827BB
:1082C00080F90E94BE1C86B164EA76E082958170D6
:1082D0000E94BE1C349909C00E9453790F900F90E0
:1082E0000F900F90DF91CF9108950E9438790F90F1
:1082F0000F900F900F90DF91CF9108958091E70537
:10830000811104C080914606882331F062E070E05C
:1083100080E090E00C94C1770895CF93DF93CDB7C0
:10832000DEB72C970FB6F894DEBF0FBECDBFA9E61F
:10833000BBE090E080E0FC01EF53F84F4591559190
:10834000659174914D935D936D937D93FC01EF5412
:10835000F84F459155916591749150964D935D9369
:108360006D937C935397FC01EF55F84F45915591D0
:108370006591749190964D935D936D937C939397D3
:10838000049680319105B9F680E29EE4A0E0B0E069
:108390008093790B90937A0BA0937B0BB0937C0B1B
:1083A00080E090E8ABE3B4E480939D0B90939E0B48
:1083B000A0939F0BB093A00B80E090E0AAE7B4E4F9
:1083C0008093A10B9093A20BA093A30BB093A40B4B
:1083D00080E090E0A6E9B3E48093A50B9093A60B10
:1083E000A093A70BB093A80B1092A90B1092AA0B05
:1083F0001092AB0B1092AC0B1092AD0B1092AE0B17
:108400001092AF0B1092B00B80E090E0A0E2B1E4CC
:1084100080937C0690937D06A0937E06B0937F06A2
:1084200080E090E0A0EAB0E480938006909381061B
:10843000A0938206B09383064AE959E969E97EE38D
:108440004093840650938506609386067093870652
:108450008093880690938906A0938A06B0938B0632
:108460001092F2051092F3051092F4051092F505A2
:108470001092EE051092EF051092F0051092F105A2
:108480001092EA051092EB051092EC051092ED05A2
:108490000E9403778CE0EAE6F1E0DE01119601909C
:1084A0000D928A95E1F789819A81AB81BC81809395
:1084B000A7159093A815A093A915B093AA158D811F
:1084C0009E81AF81B8858093AB159093AC15A09336
:1084D000AD15B093AE1589859A85AB85BC85809323
:1084E000AF159093B015A093B115B093B21584EB6E
:1084F00090E0909308068093070686E490E09093BE
:108500000A068093090610920C0610920B0680EF63
:1085100090E090930E0680930D068EE690E0909387
:10852000100680930F06109212061092110689E22F
:108530009CE5ABE8B1E480930E1590930F15A093E2
:108540001015B093111585E192E1A5E5BEE3809386
:10855000121590931315A0931415B093151580E57B
:1085600094EEA6EBB3E48093161590931715A093A1
:108570001815B09319151092700280E090E0A0EEEB
:10858000BFE380936C0290936D02A0936E02B09350
:108590006F021092E7051092E6050E947E412C962C
:1085A0000FB6F894DEBF0FBECDBFDF91CF910C9414
:1085B000663D0C948D413F924F925F926F927F92F5
:1085C0008F929F92AF92BF92CF92DF92EF92FF92E3
:1085D0000F931F93CF93DF9300D000D0CDB7DEB7BA
:1085E000382E80E090E0A0E2B1E489839A83AB83E7
:1085F000BC83C090AF15D090B015E090B115F0904D
:10860000B21520E030E0A901C701B6010E94ADE03B
:1086100087FF0CC0A701960160E070E080E291E462
:108620000E94A3E769837A838B839C8360E0CE01F9
:1086300001960E94DC3540906C0650906D0660906B
:108640006E0670906F068090700690907106A090F4
:108650007206B0907306332089F10E94697D1982F9
:108660001A821B821C82E0907406F09075060091BD
:10867000760610917706CE0101966C01A501940152
:10868000C301B2010E94DF34309246060E947E414F
:108690000F900F900F900F90DF91CF911F910F913E
:1086A000FF90EF90DF90CF90BF90AF909F908F9012
:1086B0007F906F905F904F903F9008950E94267D2D
:1086C000CECF2F923F924F925F926F927F928F9276
:1086D0009F92AF92BF92DF92EF92FF920F931F9300
:1086E000CF93DF93CDB7DEB764970FB6F894DEBFB4
:1086F0000FBECDBFD82E282E312CF101EC52FA4DF1
:10870000F49082E0D81234C080914606811103C0F3
:1087100081E00E94DB420E94697D81115AC181E69D
:1087200097E00E94867320E030E0A9010E94ADE04E
:108730008823F1F06F2DFF0C770B880B990B0E94AB
:10874000B4E02B013C0181E697E00E9486734B0167
:108750005C0120E030E040EA50E40E94ADE087FF99
:108760001BC0812C912C90EAA92E90E4B92E14C044
:108770006F2DFF0C770B880B990B0E94B4E02B0137
:108780003C01C101880F991F880F991F875A984F84
:108790000E9486734B015C01A3019201C501B401E3
:1087A0000E9413E14B015C017101EE0CFF1CEE0C09
:1087B000FF1CC701835B984F0E94867320E030E066
:1087C00040EC5FE30E9413E1A30192010E9413E1D8
:1087D000AB01BC0100E010E098018D2D0E9411BC9E
:1087E00092E0D91230C10E94267D20E030E0A9013C
:1087F000C501B4010E94ADE000E010E020E431E4E6
:10880000811118C08091450684608093450680914F
:108810008804846080938804C7018F5B984F0E940E
:1088200086736093740670937506809376069093B2
:1088300077063DC0B501A40170588D2D0E9411BC72
:10884000E2E0DE1609F4C0C0A5019401C501B4013F
:108850000E94A4E7698B7A8B8B8B9C8BF2E0DF12F2
:10886000D0C000E010E020EC30E449895A896B89DF
:108870007C898D2D0E9411BC82E0D812F0C00E942C
:10888000267D80914506846080934506809188040A
:10889000846080938804C7018F5B984F0E94867321
:1088A000F701E459F94F60837183828393832091A8
:1088B000AF153091B0154091B1155091B21560913E
:1088C00074067091750680917606909177060E94E5
:1088D000A3E7609374067093750680937606909371
:1088E0007706F701E55AFD4F10821182128213823A
:1088F0008D2D0E941D340E94B436F701E459F94FC2
:1089000080819181A281B381F701E55BFD4F808376
:108910009183A283B38392E0D91609F48FC08CE0CF
:10892000E6E7F1E0DE01119601900D928A95E1F7FC
:10893000E1E0F0E0EC0FFD1FEE0DFF1D8080918067
:10894000A280B38020E030E0A901C501B4010E94FB
:10895000ADE08823F1F120E030E0A901C501B401C8
:108960000E9427E987FF04C0B7FAB094B7F8B09423
:10897000F701E459F94F7F01A5019401C301B20148
:108980000E9413E19B01AC01F7016081718182813A
:1089900093810E94A3E7F7016083718382839383AD
:1089A000F2E080E090E0A0E4B1E4DF1621F080E0A6
:1089B00090E0A8E4B2E48D879E87AF87B88BCE01A4
:1089C0000D960E946A1D05C00E94697D882309F4E6
:1089D0003BCF64960FB6F894DEBF0FBECDBFDF91DC
:1089E000CF911F910F91FF90EF90DF90BF90AF90CC
:1089F0009F908F907F906F905F904F903F902F90BF
:108A00000895F101E25CF84F6491611107C00E9482
:108A1000347B8CE197E00E947B7A6AE070E090E022
:108A200080E00E94B2E09B01AC0160E070E088E46D
:108A300092E40E9427E88B019C0117CF0E948C735F
:108A40008111C7CF6CCF20E030E0A901C501B4018E
:108A50000E94ADE000E010E098018111EBCE81E0D2
:108A600090E0A0E0B0E00D2C04C0880F991FAA1F71
:108A7000BB1F0A94D2F720914506282B2093450668
:108A800020918804822B80938804C7018F5B984FC4
:108A90000E948673F701E459F94F608371838283E2
:108AA00093831FCF8091F805882319F01092F80561
:108AB000089540E070E060E084E896E00E94B27DB6
:108AC0000F931F9380915D06813019F50E94B0C10C
:108AD0000091710410917204209173043091740418
:108AE000601B710B820B930B28EE33E040E050E0EB
:108AF0000E94F5E660916D0470916E0480916F04A0
:108B000090917004620F731F841F951F1F910F9126
:108B100008956091470270914802809149029091B6
:108B20004A02D6CF10925D06109271041092720420
:108B3000109273041092740410924702109248022B
:108B40001092490210924A0210926D0410926E0423
:108B500010926F0410927004089580915D06813028
:108B6000F1F08230C9F40E94604560936D04709307
:108B70006E0480936F049093700481E080935D068F
:108B80000E94B0C160937104709372048093730467
:108B90009093740481E008950E949245EECF80E0A6
:108BA00008950E94FDB90E94F977882351F08091C1
:108BB000241782FD06C085EB92E09093F705809321
:108BC000F6058EEA92E00E9466B50C94AD45809160
:108BD0005D068150823070F410925D060E94B0C133
:108BE00060934702709348028093490290934A022F
:108BF00081E0089580E008958C3221E0920714F01E
:108C00008CE291E090930C1580930B150C94BCC1F1
:108C1000E0916304E63010F581E08E0F80936304E9
:108C200040913006509131066091320670913306C2
:108C300090912B0680912C0628E0E29FF0011124F0
:108C4000ED5CFB4F2091CA153091CB153183208309
:108C50004283538364837583968387830895CF9378
:108C6000DF93EC010E94084620E040E070E060E005
:108C7000CE01DF91CF910C94051820E040E070E028
:108C800060E08FE292E60C9405181092A4060E9410
:108C9000AF230C943D46E0916304EE2389F0E1504C
:108CA000E093630488E0E89FF0011124ED5CFB4F42
:108CB0006281738127814681808191810C9405189E
:108CC0000C943D467F928F929F92AF92BF92CF922B
:108CD000DF92EF92FF920F931F93CF93DF930E9447
:108CE00087BEC0912B067C2E85E0882E8C0ED6E0A8
:108CF000DC1B85E0D82EDC1AEE24EA94F12C84E00B
:108D0000C82ECC1A83E0B82EBC1A82E0A82EAC1A6A
:108D100081E0982E9C1AC11166C080912E0688238E
:108D200009F445C080915B01882361F0672D61954E
:108D300081E090912E06911180E024E04FE756E00B
:108D40000E9433BD8091A4068093FA05C43009F0D7
:108D5000EBC01092420680912E06843009F4D1C0F7
:108D600080915B018823E1F011E080912E06843030
:108D700009F010E08091FA0524E6829FC0011124D9
:108D800081589F4FB7010E9486E7862F0E94D51514
:108D900000E09C0144E656E06C2D812F0E94BB71DF
:108DA000CF5FC811B8CF87E080932C060EC08091AA
:108DB000280610922806882309F4B4CF0E944B4657
:108DC00080912D06882309F4ADCFDF91CF911F91BB
:108DD0000F91FF90EF90DF90CF90BF90AF909F905A
:108DE0008F907F900895C130C1F580912E0681301B
:108DF000E9F080915B018823A1F011E080912E06BB
:108E0000813009F010E080911601909117010E94C5
:108E1000A01500E09C0149E756E0692D812F0E94D2
:108E2000BB718091A4068093FA05BACF8091280681
:108E3000109228068823E9F210E000E027EE33E0E4
:108E40004AE050E066E171E089E796E00E9496BF53
:108E500080912D06882369F2B8CFC23009F0C0C0D6
:108E600080912E068230C9F080915B018823C9F27F
:108E700011E080912E06823009F010E080910B15F0
:108E800090910C150E94A01500E09C0142E756E06D
:108E90006A2D812F0E94BB7155CF809128061092B8
:108EA0002806882309F30E94E0BD03ED1CE12CE2B3
:108EB00031E050E040E06BE075E182E796E00E942F
:108EC00096BF80912D06882379F27FCF8091280666
:108ED00010922806882309F48BC00E94E0BD08ED9B
:108EE00017E12CE830E050E040E064E076E08EE608
:108EF00096E00E9496BF80912D06882309F478C0E1
:108F000064CF8091280610922806882309F428CF80
:108F10000E94E0BD84E696E00E9454C080912D0638
:108F2000882309F41DCF51CFC53091F580912E06CD
:108F30008530B9F080915B01882309F431CF11E0CD
:108F400080912E06853009F010E080911C019091EF
:108F50001D010E94A01500E09C014FE556E06D2D1B
:108F60001CCF8091280610922806882319F306EF5B
:108F700015E127EE33E04AE050E06CE171E08FE567
:108F800096E00E9496BF80912D06882399F21DCF0E
:108F9000C63009F005CF80912E06863091F0809181
:108FA0005B01882309F4FCCE81E090912E06963077
:108FB00009F080E023E040E556E06D2F0E9433BDCC
:108FC000EFCE8091280610922806882341F386E18F
:108FD00096E50E942F4680912D06882301F3F5CE59
:108FE000C33009F0AFCE80912E06833009F46ECFE6
:108FF00080915B01882309F414CF11E080912E0643
:10900000833009F010E080910406909105060E94DB
:10901000A01500E09C014EE656E06B2D3ACF3F9242
:109020004F925F926F927F928F929F92AF92BF9278
:10903000CF92DF92EF92FF920F931F93CF93DF9324
:10904000FF24F39480910B1590910C15892B09F452
:10905000F12C0E9487BEC0912B065C2E95E0692EF4
:109060006C0EAA24AA94B12C83E0E82EEC1A82E0BC
:10907000982E9C1A81E0882E8C1A4C2E419435E44F
:10908000C32E36E4D32E86E0782E7C1AC11195C00B
:1090900080912E06882309F470C080915B0188239B
:1090A00059F081E090912E06911180E024E04BE48C
:1090B00056E0642D0E9433BD10E000E0D4E03C2E69
:1090C00035180093FA05CD131FC0F801EE0FFF1FEE
:1090D000E15EF94F85919491909344068093430605
:1090E00080912E068C1709F41EC180915B018823A4
:1090F00059F081E090912E069D1380E023E04CE230
:1091000056E0632D0E9433BD8D2F0F5F1F4FD5E0BA
:109110008530B9F68091040690910506892B19F4E3
:10912000FF2009F420C1C630F9F480912E06863064
:1091300009F40AC180915B018823B1F0DF92CF92DC
:1091400083E296E09F938F937F9281E090912E0629
:10915000963009F080E08F930E94A01D0F900F9031
:109160000F900F900F900F9087E0FF24F394CF5F44
:10917000C6118CCF80932C060EC0809128061092C9
:109180002806882309F489CF0E944B4680912D063A
:10919000882309F482CFDF91CF911F910F91FF9027
:1091A000EF90DF90CF90BF90AF909F908F907F9087
:1091B0006F905F904F903F900895C13009F069C063
:1091C00080912E06813009F449C080915B0188238B
:1091D00009F472CFD1E080912E06813009F0D0E001
:1091E00080910B1590910C150E94A01500E09C0138
:1091F00044E456E0682D8D2F0E94BB718091A40637
:109200008093FA05C33009F057CF1092420680913F
:109210002E06833009F474C080915B01882309F421
:109220004BCFD1E080912E06833009F0D0E08091C1
:10923000FA0524E6829FC001112481589F4FB50191
:109240000E9486E7862F0E94D51500E09C0146E328
:1092500056E06E2D8D2F0E94BB712ECF8091280677
:1092600010922806882309F4B0CF0E94E0BD05EDD6
:109270001CE12CE231E050E040E06BE075E184E479
:1092800096E00E9496BF80912D06882309F49DCF19
:1092900082CFC23009F0B2CF80912E068230B9F071
:1092A00080915B01882309F407CFD1E080912E06DD
:1092B000823009F0D0E080910406909105060E946A
:1092C000A01500E09C0140E456E0692D94CF809108
:1092D000280610922806882319F30E94E0BD08EDA5
:1092E00017E12CE830E050E040E064E076E080E414
:1092F00096E00E9496BF80912D06882389F24BCF7D
:109300008091280610922806882309F485CF0E94B0
:10931000E0BD86E396E00E9454C080912D0688232C
:1093200009F47ACF38CF8091280610922806882336
:1093300009F4DBCE85EB99E40E942F4680912D063F
:10934000882309F4D2CE27CF8091280610922806D0
:10935000882309F4EFCE0E94454680912D0688238C
:1093600009F4E8CE18CF86E002CF4F925F926F9259
:109370007F928F929F92AF92BF92CF92DF92EF92A5
:10938000FF920F931F93CF93DF930091FA050E94F2
:1093900087BEC0912B0610E0000F111F015E194F10
:1093A00095E0592E5C0E25E0E22E26E0F22ED3E069
:1093B000DC1B3EEAC32E3DE1D32E47EFA42E45E051
:1093C000B42E82E0782E7C1A5CE2852E56E0952E33
:1093D00081E0682E6C1A4C2E4194C11137C08091E7
:1093E0002E068823B1F080915B01882359F081E03B
:1093F00090912E06911180E024E043E156E0642D27
:109400000E9433BDCF5F5C12E8CF84E080932C06CE
:109410000CC08091280610922806882321F30E9410
:109420004B4680912D068823F1F2DF91CF911F9159
:109430000F91FF90EF90DF90CF90BF90AF909F90F3
:109440008F907F906F905F904F900895C13059F545
:10945000F8018591949190934406809343068091FE
:109460002E06813081F080915B01882359F21F9292
:109470009F928F926F9281E090912E06913009F425
:1094800074C080E072C0809128061092280688235C
:1094900051F38091FA05682F0E944CBF80912D06F0
:1094A000882309F3C2CFC23009F042C0F801859188
:1094B0009491909344068093430680912E068230C7
:1094C000D1F080915B01882309F49CCFDF92CF9289
:1094D000BF92AF927F9281E090912E06923009F078
:1094E00080E08F930E94A01D0F900F900F900F901F
:1094F0000F900F9087CF809128061092280688231E
:1095000001F30E94AE1D80912D068823D1F28DCFEC
:1095100080912806109228068823C1F06091FA05F0
:109520008FEF0E944CBF80912D06882379F07DCF6C
:10953000C33009F067CFF801859194919093440668
:109540008093430680912E06833011F380915B0156
:10955000882309F457CF1F92FF92EF92DF9381E0A7
:1095600090912E06933009F08CCF8F930E94A01D0E
:109570000F900F900F900F900F9044CFAF92BF922B
:10958000CF92DF92EF92FF920F931F93CF93DF93CF
:109590000E9487BEC0912B0685E0B82EBC0E90EECF
:1095A000E92E95E0F92ED3E0DC1B2EEEC22E25E04D
:1095B000D22E12E01C1B01E00C1BAC2EA194C11199
:1095C00031C080912E068823B1F080915B01882301
:1095D00059F081E090912E06911180E024E042EF55
:1095E00055E06A2D0E9433BDCF5FCB11E8CF84E0F8
:1095F00080932C060CC080912806109228068823A0
:1096000021F30E944B4680912D068823F1F2DF91D1
:10961000CF911F910F91FF90EF90DF90CF90BF906F
:10962000AF900895C13011F580912E06813079F008
:1096300080915B018823C1F281E090912E069130E8
:1096400009F080E023E04BE955E2602FCBCF809119
:10965000280610922806882359F38DE79BE40E9480
:109660002F4680912D06882319F3D1CFC23081F582
:1096700090912E06923071F080915B01882309F45D
:10968000B3CF81E0923009F080E020E244EE55E073
:10969000612FA8CF8091280610922806882361F3B5
:1096A000D092F705C092F60580912D06882321F30C
:1096B000AECF8091280610922806882381F0F09280
:1096C000F705E092F60580912D06882341F09FCFA3
:1096D000C33009F089CF90912E06933051F38091D9
:1096E0005B01882309F480CF81E0933009F080E0AA
:1096F00020E24FEC55E06D2F75CFDF92EF92FF9295
:109700000F931F93CF93DF930E9487BEC0912B06C8
:1097100085E0E82EEC0ED4E0DC1B13E01C1B02E01D
:109720000C1B81E0F82EFC1ADC2ED194C1112EC046
:1097300080912E068823B1F080915B01882359F037
:1097400081E090912E06911180E024E048EC55E0F4
:109750006D2D0E9433BDCF5FCE11E8CF85E08093A1
:109760002C060CC08091280610922806882321F32D
:109770000E944B4680912D068823F1F2DF91CF9114
:109780001F910F91FF90EF90DF900895C13011F578
:1097900080912E06813079F080915B018823D9F287
:1097A00081E090912E06913009F080E023E04CEBAF
:1097B00055E26F2DCECF809128061092280688237F
:1097C00059F38DEB9DE10E942F4680912D06882351
:1097D00019F3D4CFC23009F055C080912E068230E3
:1097E00081F080915B01882309F4B5CF81E09091ED
:1097F0002E06923009F080E023E045EB55E2602F21
:10980000A8CF8091280610922806882351F388EB70
:109810009DE10E942F4680912D06882311F3AECF43
:1098200080912E06833081F080915B01882309F4BA
:1098300092CF81E090912E06933009F080E023E0F2
:109840004EEA55E2612F85CF8091280610922806B6
:10985000882351F383EB9DE10E942F4680912D06D2
:10986000882311F38BCF8091280610922806882335
:1098700091F08EE898E10E942F4680912D06882372
:1098800051F07CCFC33061F2C43009F064CF8091D5
:109890002E06843041F380915B01882309F45BCF6D
:1098A00081E090912E06943009F080E023E045EAB3
:1098B00055E26D2F4ECF0C944B462F923F924F9214
:1098C0005F926F927F928F929F92AF92BF92CF9250
:1098D000DF92EF92FF921F93CF93DF93CDB7DEB766
:1098E0002C970FB6F894DEBF0FBECDBF1C01162F0C
:1098F00080912806109228068823E1F010922A060B
:109900000E944B462C960FB6F894DEBF0FBECDBF1B
:10991000DF91CF911F91FF90EF90DF90CF90BF909C
:10992000AF909F908F907F906F905F904F903F90FF
:109930002F9008958091300690913106A0913206C3
:10994000B09133068D839E83AF83B887892B8A2B92
:109950008B2B09F460C080911E01882309F4BDC0DF
:1099600080911F018111B9C0613009F494C0623047
:1099700009F4A2C08090200190902101A0902201C2
:10998000B0902301C0902C01D0902D01E0902E01C9
:10999000F0902F01612E712C6D817E818F819885D1
:1099A0000E94B4E020911201309113014091140102
:1099B000509115010E9413E1D301AA0FBB1FAA0FFA
:1099C000BB1FBC87AB87A459B94FBA87A9872D9114
:1099D0003D914D915C910E94A4E72B013C018D814A
:1099E0009E81AF81B885B7FF8FC0A5019401C301E7
:1099F000B2010E94ADE087FD7FC0EB85FC85E45994
:109A0000F94F4082518262827382812F0E947719BE
:109A100081E080935B011092300610923106109223
:109A200032061092330680915B01882309F46ACFD5
:109A3000F4E01F9FC0011124FC01E459F94F825A40
:109A4000994FDC012D913D914D915C916081718127
:109A5000828193810E94A4E76B017C01C982DA8232
:109A6000EB82FC822DEC3CEC4CEC5DE3609112014E
:109A70007091130180911401909115010E9427E9C2
:109A800087FD52C0CE0101960E94A514BC01C10100
:109A90000E943C7137CF8090240190902501A090C6
:109AA0002601B0902701C0903001D0903101E090A4
:109AB0003201F09033016ECF8090280190902901FF
:109AC000A0902A01B0902B01C0903401D0903501B4
:109AD000E0903601F09037015DCF812C30E5932E78
:109AE00033ECA32E37ECB32EC12C40E5D42E43EC3F
:109AF000E42E47E4F42E4ECFA985BA858D929D922F
:109B0000AD92BC92139781CFA7019601C301B20118
:109B10000E9427E918160CF070CFE985FA85C082FB
:109B2000D182E282F38271CF20E030E040E251E462
:109B3000C701B6010E9413E120E030E04AE754E497
:109B40000E9413E14B015C0120E030E0A901C70154
:109B5000B6010E94ADE020E030E040EA50E487FF2B
:109B600004C020E030E040EA50ECC501B4010E949E
:109B7000A4E720E030E040E251E40E9427E80E94A0
:109B800099E86B017C01F7FC62C020EA36E841E00D
:109B900050E00E9417E7CA01B9012AE030E040E036
:109BA00050E00E9417E7605D60933406C701B6017C
:109BB00020E137E240E050E00E9417E78AE0882E7B
:109BC000912CA12CB12CCA01B901A50194010E94CC
:109BD00017E7605D60933506C701B60128EE33E0F4
:109BE00040E050E00E9417E7CA01B901A5019401C5
:109BF0000E9417E7605D609336068EE28093370619
:109C0000C701B60124E630E040E050E00E9417E7CB
:109C1000CA01B901A50194010E9417E7605D609334
:109C20003806C701B601A50194010E9417E7162F57
:109C3000CA01B901A50194010E9417E7605D609314
:109C40003906105D10933A0684E396E01FCFF09436
:109C5000E094D094C094C11CD11CE11CF11C6DE2B5
:109C6000A3CF62E08EEA95E20C945D4C61E085EB57
:109C700095E20C945D4C60E08CEB95E20C945D4CAD
:109C8000CF93DF9300D000D0CDB7DEB78091280608
:109C900010922806882359F010922A060E944B46FB
:109CA0000F900F900F900F90DF91CF9108956091DA
:109CB000300670913106809132069091330661151D
:109CC00071058105910561F10E94B4E020911201B6
:109CD0003091130140911401509115010E9413E13C
:109CE000209178063091790640917A0650917B0652
:109CF0000E94A4E7609378067093790680937A06B1
:109D000090937B0683E00E94771981E080935B014A
:109D100010923006109231061092320610923306DD
:109D200080915B01882309F4BBCF20911306309109
:109D300014064091150650911606609178067091B0
:109D4000790680917A0690917B060E94A3E7698349
:109D50007A838B839C83CE0101960E94A514BC015B
:109D600085EA95E20E943C719BCF2F923F924F92E1
:109D70005F926F927F928F929F92AF92BF92CF929B
:109D8000DF92EF92FF920F931F93CF93DF93CDB7A4
:109D9000DEB7ED970FB6F894DEBF0FBECDBF809152
:109DA0002F06882369F18091241700E010E083FFDB
:109DB00023C087E395E10E948D1F8BE1E7E3F5E186
:109DC000DE01919601900D928A95E1F710E000E096
:109DD000BE016F5F7F4FCE0181960E9466CE18163E
:109DE0003CF4CE0101960E9449C8080F111DF0CF26
:109DF000CE0181960E94602100936B0410936C0445
:109E00000E9487BE10912B061CAF85E0810F8DAF9D
:109E1000312E319487E7C82E86E1D82E97E9A92EF6
:109E200095E0B92E81E0782E711A2BE9822E25E07B
:109E3000922E111113C080912E06882391F18091EA
:109E40005B01882359F081E090912E06911180E00A
:109E500024E044EA55E0632D0E9433BD809124172D
:109E600085FF55C01130D9F480912E068130F1F173
:109E700080915B01882309F45BC11F929F928F92AE
:109E80007F9281E090912E06913009F080E08F93CF
:109E90000E94A01D0F900F900F900F900F9082E0E6
:109EA00066C08091280610922806882341F20E94FD
:109EB0004B4680912D06882311F2ED960FB6F8944B
:109EC000DEBF0FBECDBFDF91CF911F910F91FF90ED
:109ED000EF90DF90CF90BF90AF909F908F907F904A
:109EE0006F905F904F903F902F900895809128063B
:109EF00010922806882309F4BBCF10922B060E94EB
:109F000005D280912D06882309F4B2CFD6CF83FFE6
:109F10002DC0113021F680912E068130D1F0809134
:109F20005B01882309F404C1DF92CF92BF92AF9204
:109F30007F9281E090912E06913009F080E08F931E
:109F40000E94A01D0F900F900F900F900F900F90F8
:109F5000A6CF8091280610922806882301F30E943C
:109F6000771680912D068823D1F2A7CF81E09091BA
:109F70005B01992309F4DDC0582E082FF12CE12C48
:109F8000412E9CAD491A802F20916B0430916C04B6
:109F9000E216F30608F0CDC00113A5C087E395E1F2
:109FA0000E948D1F202E25188BE1E7E3F5E1DE01ED
:109FB000919601900D928A95E1F7612CBE016F5F39
:109FC0007F4FCE0181960E9466CE18167CF4CE019A
:109FD00001960E9449C8882389F326106BC0BE01F0
:109FE0006F5F7F4F80E596E00E9464C8CE01819646
:109FF0000E9460218091241790912E0684FF78C0E2
:10A00000911366C08091280610922806882309F4CF
:10A010005FC019821C8280913A1562E575E1882340
:10A0200011F067E375E121E040E556E0CE010196CD
:10A030000E946621882309F43FC08BE1FE0131961E
:10A04000A7E3B5E101900D928A95E1F7809124177D
:10A050008F7D80932417A0911917AA3080F481E096
:10A060008A0F809319178BE18A9FD0011124A55F75
:10A07000B94EE7E3F5E101900D928A95E1F7CE0143
:10A0800001960E94602110922B0682E090E0A0E0F1
:10A09000B0E08093300690933106A0933206B093DF
:10A0A000330681E080932D0610926A0483E080934A
:10A0B0005B0103CF639482CF0E94347B60E576E03E
:10A0C00081E895E00E9436838AE00E94637AD7CFC8
:10A0D00080915B01882339F081E0911380E041E0B9
:10A0E000642D0E9474BD8FEFE81AF80A0F5F4BCF02
:10A0F000911759F080915B018823A9F381E0909139
:10A100002E06911380E040E0EBCF8091280610925C
:10A110002806882379F380E596E00E94EBC70E9429
:10A120003D460E94FDB980912D06882319F3C5CEC6
:10A1300082E01F5F9DAD91137CCE80932C06BDCE37
:10A140003F924F925F926F927F928F929F92AF92C7
:10A15000BF92CF92DF92EF92FF920F931F93CF9314
:10A16000DF930E9487BEC0912B063C2E85E0482ECF
:10A170004C0E9DE8C92E94E0D92E09EB14E0D4E0F2
:10A18000DC1B2CE5A22E24E0B22E37EAE32E34E0CD
:10A19000F32E83E0782E7C1A4DE2842E44E0942E38
:10A1A00082E0682E6C1A81E0582E5C1AC11139C009
:10A1B00080912E068823B9F080915B01882361F09D
:10A1C000632D619581E090912E06911180E024E04D
:10A1D00047ED54E00E9433BDCF5FC411E7CF85E067
:10A1E00080932C060CC080912806109228068823A4
:10A1F00019F30E944B4680912D068823E9F2DF91E6
:10A20000CF911F910F91FF90EF90DF90CF90BF9073
:10A21000AF909F908F907F906F905F904F903F9006
:10A220000895C13041F580912E06813089F08091EA
:10A230005B01882389F21F9281ED94E09F938F93B5
:10A240005F9281E090912E06913061F180E02AC00A
:10A250008091280610922806882349F38FEC93E01A
:10A260009093F7058093F6050E943D4680912D0658
:10A270008823E9F2C4CFC23009F064C080912E0671
:10A280008230C9F080915B01882309F4A5CF1F9229
:10A2900088EC94E09F938F936F9281E090912E06CB
:10A2A0009230A1F68F930E94A01D0F900F900F90F7
:10A2B0000F900F9091CF8091280610922806882346
:10A2C00009F39092F7058092F6050E943D46809131
:10A2D0002D068823B9F293CF80912E06833081F02A
:10A2E00080915B01882309F477CF1F92FF92EF9250
:10A2F0007F9281E090912E06933009F0A7CFD2CFC4
:10A300008091280610922806882351F3B092F70511
:10A31000A092F6050E943D4680912D06882301F308
:10A320006ECF80912806109228068823A1F0D09243
:10A33000F705C092F6050E943D4680912D068823C0
:10A3400051F05DCFC33041F2C43009F045CF809168
:10A350002E06843031F380915B01882309F43CCFD1
:10A360001F921F930F93DF9381E090912E069430FC
:10A3700009F06CCF97CFDF92EF92FF920F931F936C
:10A38000CF93DF930E94BF17082F0E9487BEC09112
:10A390002B06FC2E85E0E82EEC0E11E01C1BDC2EBB
:10A3A000D194C11114C080912E068823F9F08091B8
:10A3B0005B01882309F477C081E090912E0691110A
:10A3C00080E024E043E353E06D2D0E9433BD011192
:10A3D0003DC0D2E0C130D9F580912E068130D1F058
:10A3E00080915B01811125C0D2E047C08091280691
:10A3F000109228068823D9F20E944B4680912D06A0
:10A400008823A9F2DF91CF911F910F91FF90EF90D8
:10A41000DF9008958091280610922806882301F382
:10A420008AE893E50E942F4680912D068823C1F289
:10A43000E9CF81E090912E06913009F080E023E091
:10A440004AE253E0612F0E9433BDCECFD1E0DC134E
:10A4500014C080912E068D17B9F080915B0188237E
:10A4600061F06C2F6F1981E090912E069C1380E0B3
:10A4700023E041E253E00E9433BDCF5FCE1191CF84
:10A48000DF5FD0932C06BECF80912806109228065D
:10A49000882319F389EB94E50E942F4680912D06BD
:10A4A0008823D9F2AFCFD1E0002309F49DCFE5CFC7
:10A4B0006F927F928F929F92AF92BF92CF92DF92D4
:10A4C000EF92FF920F931F93CF93DF930E9487BE6B
:10A4D000C0912B066C2E85E0782E7C0E9EE6E92E30
:10A4E00099E7F92E2DE4C22E23E0D22ED5E0DC1B15
:10A4F00038E3A32E39E7B32E14E01C1B03E00C1B3A
:10A5000082E0982E9C1A81E0882E8C1AC11136C0E8
:10A5100080912E068823B9F080915B01882361F039
:10A52000662D619581E090912E06911180E024E0E6
:10A5300045E653E00E9433BDCF5FC711E7CF86E009
:10A5400080932C060CC08091280610922806882340
:10A5500019F30E944B4680912D068823E9F2DF9182
:10A56000CF911F910F91FF90EF90DF90CF90BF9010
:10A57000AF909F908F907F906F900895C13029F594
:10A5800080912E068130A1F080915B018823A1F299
:10A5900089E899E79F938F938FE593E09F938F933B
:10A5A0008F9281E090912E06913049F180E027C092
:10A5B0008091280610922806882331F30E94897919
:10A5C00080912D06882301F3CACFC23009F085C0DF
:10A5D00080912E068230E9F080915B01882309F496
:10A5E000ABCF85E89DE19F938F9385E593E09F93A3
:10A5F0008F939F9281E090912E069230B9F68F93BF
:10A600000E94A01D0F900F900F900F900F900F9031
:10A6100093CF80912806109228068823E9F20E94A1
:10A62000851D80912D068823B9F299CF80912E0641
:10A630008330A9F080915B01882309F47DCF83E505
:10A6400099E79F938F9386E493E09F938F930F9363
:10A6500081E090912E06933009F0A8CFD0CF809161
:10A66000280610922806882329F30E9453798091A6
:10A670002D068823F9F273CF80912E06843099F04D
:10A6800080915B01882309F457CFBF92AF9281E498
:10A6900093E09F938F931F9381E090912E069430C7
:10A6A00009F084CFACCF8091280610922806882329
:10A6B00039F30E94387980912D06882309F34FCF12
:10A6C0008091280610922806882399F00E946E79BE
:10A6D00080912D06882369F042CFC33009F4A6CFBC
:10A6E000C43051F2C53009F027CF80912E06853055
:10A6F00039F380915B01882309F41ECFFF92EF921A
:10A70000DF92CF92DF9381E090912E06953009F091
:10A710004DCF75CFBF92CF92DF92EF92FF920F9302
:10A720001F93CF93DF930E9487BEC0912B0685E0D5
:10A73000C82ECC0ED4E0DC1B13E01C1B82E0F82EEC
:10A74000FC1A81E0E82EEC1ABC2EB194C11130C085
:10A7500080912E068823B1F080915B01882359F007
:10A7600081E090912E06911180E024E04FE053E0CB
:10A770006B2D0E9433BDCF5FCC11E8CF85E0809375
:10A780002C060CC08091280610922806882321F3FD
:10A790000E944B4680912D068823F1F2DF91CF91E4
:10A7A0001F910F91FF90EF90DF90CF90BF90089591
:10A7B000C130B9F580912E068130F1F080915B01B6
:10A7C0008823C9F2DD24D39480912E06813009F0CC
:10A7D000D12C60917D0B70917E0B80917F0B9091BD
:10A7E000800B0E94B61600E09C0144E053E06E2D01
:10A7F0008D2D0E94BB71BFCF809128061092280634
:10A800008823E1F20E94E0BD4BE856E26DE77BE071
:10A8100084E093E00E94DDBE80912D06882371F2D2
:10A82000BDCFC23009F07FC080912E068230E1F0AA
:10A8300080915B01882309F49ECFDD24D39480911D
:10A840002E06823009F0D12C6091810B7091820B21
:10A850008091830B9091840B0E94B61600E09C01BE
:10A8600049EF52E06F2DC4CF809128061092280640
:10A870008823F1F20E94E0BD49E856E261E87BE0FE
:10A8800089EF92E00E94DDBE80912D06882381F23F
:10A8900085CF80912E068330E1F080915B01882383
:10A8A00009F469CFDD24D39480912E06833009F01A
:10A8B000D12C6091850B7091860B8091870B9091C4
:10A8C000880B0E94B61600E09C014EEE52E0612F0C
:10A8D0008FCF80912806109228068823F1F20E94DB
:10A8E000E0BD47E856E265E87BE08EEE92E00E942C
:10A8F000DDBE80912D06882381F250CF80912806FD
:10A90000109228068823C9F00E94E0BD45E856E26F
:10A9100069E87BE083EE92E00E94DDBE80912D0627
:10A92000882359F03BCFC33009F4B3CFC43009F0CA
:10A9300022CF80912E06843009F380915B01882319
:10A9400009F419CFDD24D39480912E06843009F0C8
:10A95000D12C6091890B70918A0B80918B0B909117
:10A960008C0B0E94B61600E09C0143EE52E06D2F66
:10A970003FCF2F923F924F925F926F927F928F9232
:10A980009F92AF92BF92CF92DF92EF92FF920F937E
:10A990001F93CF93DF93CDB7DEB729970FB6F89407
:10A9A000DEBF0FBECDBF0E9487BE10912B0685E093
:10A9B000810F8E8391E0911B9F83812F81958887E2
:10A9C0008CE6282E82E0382E9CED892E95E0992E7B
:10A9D000A12CB12C26ED422E26E0522E612C712C9A
:10A9E00082E0811B8987111148C080912E0688233F
:10A9F000F9F080915B01882359F081E090912E0657
:10AA0000911180E024E04FE053E068850E9433BD5F
:10AA100080917002882309F407C1123009F461C0E3
:10AA200083E01F5F9E819113DECF80932C060CC0C4
:10AA300080912806109228068823D9F20E944B465E
:10AA400080912D068823A9F229960FB6F894DEBFCF
:10AA50000FBECDBFDF91CF911F910F91FF90EF906F
:10AA6000DF90CF90BF90AF909F908F907F906F902E
:10AA70005F904F903F902F900895113049F680914C
:10AA80002E068130C9F080915B01882309F281E0B4
:10AA900090912E06913009F080E09091700226EDA1
:10AAA00032E0911102C022ED32E001E049ED52E0C6
:10AAB0006F810E94BB71ACCF80917002909128068B
:10AAC000109228069923F9F281278093700283E07F
:10AAD00080935B010E943E1480912D06882399F299
:10AAE000B3CF80912E068230D1F180915B01882313
:10AAF00009F496CF81E08D8380912E06823009F093
:10AB00001D82C0906C02D0906D02E0906E02F090B9
:10AB10006F0220E030E0A901C701B6010E94ADE05C
:10AB20002DEB37E346E055EB87FD04C02DEB37E313
:10AB300046E055E3C701B6010E94A4E769837A8322
:10AB40008B839C83CE0101960E94ECBD00E09C01AA
:10AB500048EC52E069858D810E94BB7161CF809184
:10AB6000280610922806882309F4BFCF0E94E0BD72
:10AB700020E030E04AE754E460916C0270916D028D
:10AB800080916E0290916F020E9413E120E030E00C
:10AB9000A9010E94A4E720E030E84BEB54E40E94B6
:10ABA000A3E70E94A0E86B0191E090932D060E941C
:10ABB000084683E080935B0188EC92E0909327063F
:10ABC0008093260630922506209224068092200645
:10ABD00090922106A0922206B092230640921C0673
:10ABE00050921D0660921E0670921F06F12CE12CF9
:10ABF000C0923006D0923106E0923206F0923306CF
:10AC00008FE497E59093CB158093CA158EE394E17A
:10AC100090931B0680931A061092190680912D06B8
:10AC2000882309F462CF10CF82E0FBCECF92DF926F
:10AC3000EF92FF92CF93DF9380912806109228061F
:10AC4000882351F010922A06DF91CF91FF90EF9068
:10AC5000DF90CF900C944B4681E080932A06809140
:10AC6000300690913106A0913206B09133060097DC
:10AC7000A105B10509F44BC02AE0289FE001299FF6
:10AC8000D00D112410923006109231061092320627
:10AC900010923306BE010D2E000C880B990B0E94FA
:10ACA000B4E02091AD063091AE064091AF065091D0
:10ACB000B0060E9413E12091AF153091B01540917C
:10ACC000B1155091B2150E94A4E76B017C0120E000
:10ACD00030E040E151EC0E9427E987FD18C020E0F8
:10ACE00030E040E151E4C701B6010E94ADE0181622
:10ACF00074F0CE010E94E9C1C092AF15D092B01598
:10AD0000E092B115F092B21582E080935B018091E0
:10AD10005B01882379F08FEA95E10E94ECBDBC01CC
:10AD200089EB92E0DF91CF91FF90EF90DF90CF9091
:10AD30000C943C71DF91CF91FF90EF90DF90CF901A
:10AD400008950F931F93CF93DF93FC01EB01809144
:10AD5000300690913106A0913206B0913306B7FFCC
:10AD600008C01092300610923106109232061092EE
:10AD7000330680911C0690911D06A0911E06B0918D
:10AD80001F06409130065091310660913206709155
:10AD9000330684179507A607B70744F48093300657
:10ADA00090933106A0933206B093330680915B01F5
:10ADB0008823E1F06091300670913106809132066F
:10ADC00090913306009120061091210620912206D1
:10ADD00030912306600F711F821F931F0995BC01DC
:10ADE00080912606909127060E943C71809128064A
:10ADF000811108C0809119068823D1F180915B01EF
:10AE00008823B1F180912406909125060097B1F036
:10AE100040913006509131066091320670913306B0
:10AE200000912006109121062091220630912306E0
:10AE3000400F511F621F731FFE010995E0911A0612
:10AE4000F0911B06309741F080911906811103C0E3
:10AE50008091280681110995809128061092280674
:10AE6000882331F0DF91CF911F910F910C944B46C5
:10AE7000DF91CF911F910F91089569E176E182E30F
:10AE800096E10C94A1566FE476E182E696E10C948B
:10AE9000A1566EE777E187E997E10C94A15666EA3F
:10AEA00077E189EE9DE10C94A156CF93DF93CDB766
:10AEB000DEB78D819091F312891768F08093F312B9
:10AEC0009E01285F3F4F4E815F816AE270E088EC0F
:10AED00092E10E9474E0DF91CF9108950F931F9348
:10AEE000CF93DF938C016F3F19F41092F31260E05F
:10AEF0002091F312862F062E000C990B28171906A5
:10AF000009F0F4F46093F312C8010E94FADF800F95
:10AF1000911FEC01C01BD10BCB32D1053CF0019746
:10AF2000FC012491207C2038D1F3F3CFDD27AE0142
:10AF3000B80188EC92E10E941BE0C853DD4E1882F4
:10AF4000DF91CF911F910F910895DF92EF92FF92C1
:10AF50000F931F93CF93DF93CDB7DEB7C658D109B8
:10AF60000FB6F894DEBF0FBECDBFC358DF4F1882B7
:10AF700019821A821B82CD57D0408091290290916C
:10AF80002A02A0912B02B0912C02CF57DF4F888369
:10AF90009983AA83BB83C158D04084E690E0909304
:10AFA0006B0680936A0610921B1510921A15109268
:10AFB000950464E070E0CE018F579F4F0E9448C116
:10AFC00080916A0690916B06029690936B0680932F
:10AFD0006A0610921B1510921A1581E0CA57DF4FAE
:10AFE0008883C658D040CE018A579F4F0E942A1DA1
:10AFF00068E470E089E69BE00E9448C160E170E08F
:10B000008CE796E00E9448C18AE097EDA3EABCE392
:10B01000C358DF4F88839983AA83BB83CD57D04021
:10B02000CE0183589F4F0E94221D8AEE95E00E9418
:10B030002E1D7E018DE6E80EF11C8FEFD7018C935B
:10B04000C7010E942A1D19821A821B821C828E014E
:10B050000F5F1F4FC8010E94221D19821A821B8296
:10B060001C82C8010E94221DC358DF4F188219821A
:10B070001A821B82CD57D04083E0F70180838983F9
:10B08000CE0183589F4F0E94221DC7010E942A1D96
:10B09000C8010E942A1D4AE0D42EDA94DD2031F046
:10B0A000CE0183589F4F0E94221DF7CF87EA95E17A
:10B0B0000E942E1DC358DF4F188219821A821B82EC
:10B0C000CD57D0403AE0D32EDA94DD2031F0CE01D6
:10B0D00083589F4F0E94221DF7CF85E0D82ED9823A
:10B0E000D701DC92C8010E942A1DC7010E942A1DB7
:10B0F00068E070E08DED92E00E9448C168E070E089
:10B1000085ED92E00E9448C164E670E081E792E03C
:10B110000E9448C119828FEFF7018083C8010E9405
:10B12000261DC7010E942A1D64E070E087EC91E0B3
:10B130000E9448C18091E9058983C8010E94261DAB
:10B140006CE070E087E096E00E9448C1198A1A8A94
:10B150001B8A1C8A80E090E0A0E8BFE38D879E8771
:10B16000AF87B88B80910E1590910F15A091101597
:10B17000B091111589839A83AB83BC832CEA35EC9B
:10B1800047E25EE3609112157091131580911415DA
:10B19000909115150E9427E86D837E838F83988791
:10B1A0002CEA35EC47E25EE36091161570911715B5
:10B1B00080911815909119150E9413E169877A877B
:10B1C0008B879C8764E170E0C8010E9448C184E1DC
:10B1D00090E09A838983C8010E941A1D8CE0E2E8FE
:10B1E000F1E0D80101900D928A95E1F7C8010E9423
:10B1F0001E1D8CE0E2E8F1E0D80101900D928A95E5
:10B20000E1F7C8010E941E1D1982C8010E942A1D73
:10B210008FE790E09A838983C8010E941A1DEEE8A7
:10B22000F1E0D80101900D92DA94E1F765E070E069
:10B23000C8010E9448C11982C8010E94261D80E2EF
:10B24000E3E9F1E0D80101900D928A95E1F760E21F
:10B2500070E0C8010E9448C1D7011C92C7010E943A
:10B26000261D80E792E00E94261D8CE692E00E9457
:10B27000221DC358DF4F188219821A821B82CD57B4
:10B28000D040CE0183589F4F0E94221D80E2F801DA
:10B2900011928A95E9F760E270E0C8010E9448C106
:10B2A000FE01F99688E0DF011D928A95E9F744E6F0
:10B2B00050E060E070E049835A836B837C834D8368
:10B2C0005E836F83788783E090E0A0E0B0E08987B9
:10B2D0009A87AB87BC874D875E876F87788B498B52
:10B2E0005A8B6B8B7C8B8D8B9E8BAF8BB88F898FA2
:10B2F0009A8FAB8FBC8F8D8F9E8FAF8FB8A38EE14F
:10B3000090E0A0E0B0E089A39AA3ABA3BCA38DA377
:10B310009EA3AFA3B8A789A79AA7ABA7BCA78DA7E1
:10B320009EA7AFA7B8AB89AB9AABABABBCAB8DABB1
:10B330009EABAFABB8AF60E470E0C8010E9448C1FB
:10B3400090E1D92EF8018D2D11928A95E9F760E1EF
:10B3500070E0C8010E9448C1D8011D92DA94E9F753
:10B3600060E170E0C8010E9448C1C358DF4F1882F5
:10B3700019821A821B82CD57D040CE0183589F4F2D
:10B380000E94221D2CE0D22EF8018D2D11928A955B
:10B39000E9F76CE070E0C8010E9448C18CE6D80172
:10B3A0001D928A95E9F76CE670E0C8010E9448C1D9
:10B3B00089E894E00E941E1DF7011082118212821A
:10B3C0001382148215821682178268E070E0C7012A
:10B3D0000E9448C1F7011192DA94E9F7CB57DF4F89
:10B3E0001882C558D04080E090E0A0E4B0E4ED962B
:10B3F0008CAF9DAFAEAFBFAFED97C7010E942E1DC2
:10B40000CE018B579F4F0E942A1DCE0187589F4F18
:10B410000E94221D80919504811124C000916A062A
:10B4200010916B0680911A1590911B15D7018D9381
:10B430009C9384E690E090936B0680936A0664E0A8
:10B4400070E08BEC91E00E9448C1C7010E941A1D78
:10B4500091E00134134009F490E080919504892B28
:10B460008093950480919504811105C060E08DE77B
:10B4700097E00E946E579091950481E08927CA5702
:10B48000DF4F0FB6F894DEBF0FBECDBFDF91CF9177
:10B490001F910F91FF90EF90DF90089581E08093CE
:10B4A000E5020E942F411092E50281110C942F4178
:10B4B0000E948D410E94A5570E94347B8DE897E041
:10B4C0000E947B7A80E008950C944E5A0C94A55704
:10B4D0002F923F924F925F926F927F928F929F92A4
:10B4E000AF92BF92CF92DF92EF92FF920F931F9392
:10B4F000CF93DF9300D01F92CDB7DEB70E94BF1766
:10B50000582E0E9487BE20912B062A83422E2B5F45
:10B510002B8383E0782E741803E713E024E6E22EF1
:10B520002AE5F22E34E8C32E33E0D32E46E6A42ECD
:10B530004AE5B42E52E9852E53E0952E82E0841917
:10B54000898381E0382E3418242C21948A8181113A
:10B55000A0C080912E06882309F477C080915B01FA
:10B56000882359F081E090912E06911180E024E02B
:10B570004AEC53E0622D0E9433BD511050C18A81C4
:10B58000833009F03CC180912E06833009F4D5C088
:10B5900080915B018111E2C084E0682E81E0860D1C
:10B5A00051104AC09A8189131FC080912E068917B5
:10B5B00009F407C180915B018823B1F0FF92EF92FB
:10B5C000DF92CF928A8184198F9381E090912E0629
:10B5D0002A81921380E08F930E94A01D0F900F90FC
:10B5E0000F900F900F900F9082E0860D9A81891333
:10B5F00021C080912E06891709F4F2C080915B0169
:10B600008823C1F089ED92E49F938F931F930F934A
:10B610008A8184198F9381E090912E062A8192135A
:10B6200080E08F930E94A01D0F900F900F900F90BD
:10B630000F900F9083E0860D9A819F5F9A832B81F4
:10B64000921384CF80932C060EC08091280610920E
:10B650002806882309F482CF0E944B4680912D064C
:10B66000882309F47BCF0F900F900F90DF91CF913B
:10B670001F910F91FF90EF90DF90CF90BF90AF9010
:10B680009F908F907F906F905F904F903F902F9002
:10B6900008959A81913051F580912E068130B9F04C
:10B6A00080915B01882309F468CF81E090912E0698
:10B6B000913009F080E023E048EB53E0632D0E94D5
:10B6C00033BD5110ACC085E094E0692E6BCF809102
:10B6D000280610922806882319F38BEB91E50E9427
:10B6E0002F4680912D068823D9F2BDCF2A812230A2
:10B6F00009F043CF80912E06823081F080915B016A
:10B70000882309F43ACF81E090912E06923009F017
:10B7100080E023E049EA53E06981D1CF8091280697
:10B7200010922806882351F386E196E50E942F4661
:10B7300080912D06882311F396CF809128061092D0
:10B740002806882309F424CF88E592E50E942F4635
:10B7500080912D06882309F41BCF85CF81E090913D
:10B760002E06933009F080E023E041EA53E0672D94
:10B770000E9433BD11CF809128061092280688239D
:10B7800009F447C00E94A55780912D06882309F42B
:10B7900040C069CFBF92AF929F928F928A818419E5
:10B7A0008F9381E090912E062A81921380E08F93EF
:10B7B0000E94A01D0F900F900F900F900F900F9070
:10B7C0002CC08091280610922806882309F4F2CE16
:10B7D0000E944E5A80912D06882309F4EBCE43CF68
:10B7E0008091280610922806882309F407CF0E942A
:10B7F0008D4180912D06882309F400CF34CF8A81B2
:10B80000843009F060CF80912E069A81891709F45F
:10B81000B2CF80915B018111BDCF8A81BECE9A816A
:10B8200084E0933009F008CFEECFCF9380912B04C2
:10B83000811109C083EA92E09093690480936804BF
:10B8400081E080932B040E94084620E040E070E0F5
:10B8500060E088E29EE10E940518C1E0C0932A06DC
:10B860000E948D2610922A060E944B46C0932A06FB
:10B8700060E08DE396E20E946E578FE992E090932C
:10B88000F7058093F605CF9108952F923F924F923E
:10B890005F926F927F928F929F92AF92BF92CF9260
:10B8A000DF92EF92FF920F931F93CF93DF9300D01D
:10B8B00000D000D0CDB7DEB790915D0680912417FF
:10B8C00082FB442440F8913011F44424439483FBD8
:10B8D000222720F92983212C83FF03C00E94F977B6
:10B8E000282E0E9487BE80912B068D83582E8B5F59
:10B8F0008A830FE315E081E0382E351883E0782E37
:10B90000751882E085198B8335E1E32E3CE5F32E33
:10B9100049E6C42E45E0D42E952D91959C8358EE92
:10B92000A52E54E0B52E6BE0862E65E0962E2D8177
:10B9300021113EC080912E068823A9F080915B01E1
:10B94000882359F081E090912E06911180E024E047
:10B9500045E755E06C810E9433BD442009F4ABC03B
:10B9600024E0622EC2C08091280610922806882307
:10B9700029F30E944B4680912D068823F9F22696E2
:10B980000FB6F894DEBF0FBECDBFDF91CF911F91F0
:10B990000F91FF90EF90DF90CF90BF90AF909F906E
:10B9A0008F907F906F905F904F903F902F90089571
:10B9B000442009F480C08D81813061F580912E068C
:10B9C0008130D9F080915B018823A1F0FF92EF9242
:10B9D000DF92CF923F9281E090912E06913009F054
:10B9E00080E08F930E94A01D0F900F900F900F90FA
:10B9F0000F900F9094E0692E91C0809128061092CC
:10BA000028068823F9F20E94155C80912D06882370
:10BA1000C9F2B5CF9D81923031F580912E068230EA
:10BA200099F080915B01882361F081E090912E066E
:10BA3000923009F080E023E04EE555E06B810E94F2
:10BA400033BD84E0682E85C08091280610922806B8
:10BA5000882339F388ED9DE10E942F4680912D06C1
:10BA60008823F9F28CCF2D81233009F079CF809192
:10BA70002E06833089F080915B01882311F381E0E9
:10BA800090912E06933009F080E023E049E555E0DF
:10BA9000672D0E9433BDAECF8091280610922806F4
:10BAA000882349F382E696E40E942F4680912D0672
:10BAB000882309F364CF80915D06823029F00E94CB
:10BAC0000778882309F4CFC08D81813009F0E9C05F
:10BAD00080912E06813009F49EC080915B01811116
:10BAE000A9C092E09E836E8063948D81681216C017
:10BAF00080912E06861509F4E6C080915B018823AB
:10BB000069F06D81651981E090912E062D81921367
:10BB100080E023E04CE255E00E9433BD81E0860DD9
:10BB20009D81891316C080912E06891709F4DCC007
:10BB300080915B01882369F06D81651981E09091A6
:10BB40002E062D81921380E023E04EE155E00E9405
:10BB500033BD82E0860D411055C09D81891316C00A
:10BB600080912E06891709F4D0C080915B0188234B
:10BB700069F06D81651981E090912E062D819213F7
:10BB800080E023E04FE055E00E9433BD83E0860D66
:10BB90009981992309F4ECC0211034C02D818213BE
:10BBA00014C090912E06921709F4C0C080915B01D9
:10BBB000882359F06D81651981E02D81921380E011
:10BBC00020E24DEF54E00E9433BD84E0860D9D815C
:10BBD000891316C080912E06891709F4B8C0809188
:10BBE0005B01882369F06D81651981E090912E06D3
:10BBF0002D81921380E023E04CEE54E00E9433BD8F
:10BC000085E0860D9D819F5F9D832A8192138FCE53
:10BC100080932C06B4CE80912806109228068823A3
:10BC200009F45BCF0E94D14580912D06882309F449
:10BC300054CFA5CE81ED95E49F938F931F930F93DF
:10BC40003F9281E090912E06913009F080E08F9331
:10BC50000E94A01D0F900F900F900F900F900F90CB
:10BC600082E08E8340CF91E09E838E819D818913F7
:10BC70003ACF80912E062E818217B1F080915B0120
:10BC8000882309F430CF6D81651981E090912E06EB
:10BC90002D81921380E023E048E355E00E9433BDFC
:10BCA00022CF22E02E83E1CF809128061092280631
:10BCB000882321F38EEB9AE40E942F4680912D0673
:10BCC0008823E1F25CCE8091280610922806882312
:10BCD00009F413CF8FE098E40E942F4680912D063F
:10BCE000882309F40ACF4BCE8091280610922806AB
:10BCF000882309F41DCF88E69AE50E942F4680919B
:10BD00002D06882309F414CF3ACE8091280610928C
:10BD10002806882309F429CF80EA90E50E942F465F
:10BD200080912D06882309F420CF29CE8091280602
:10BD300010922806882309F439CF9092F705809253
:10BD4000F60580912D06882309F430CF18CE809116
:10BD5000280610922806882309F441CF85EB9EE43B
:10BD60000E942F4680912D06882309F438CF07CEF4
:10BD70009D81891314C090912E062D81921789F010
:10BD800080915B01882359F06D81651981E02D81D7
:10BD9000921380E020E24CE455E00E9433BD84E041
:10BDA00030CF8091280610922806882349F3B0925C
:10BDB000F705A092F60580912D06882309F3DFCDC3
:10BDC0001092450210925A0180912417806480934A
:10BDD00024178AE892E00E9466B560E081E992E06B
:10BDE0000E946E570C943D464F925F926F927F92E5
:10BDF0008F929F92AF92BF92CF92DF92EF92FF927B
:10BE00000F931F93CF93DF9300D000D0CDB7DEB751
:10BE10000E94B0C14B015C01809110018F3FF1F194
:10BE20000E94B0C1C0901804D0901904E0901A0488
:10BE3000F0901B046C197D098E099F0997FD2EC097
:10BE40008091B8159091B9158F5F8F70891731F176
:10BE5000E0911001E43008F0E2C024E0E29FF0013C
:10BE60001124ED54FE4F80819181A281B381898399
:10BE70009A83AB83BC83C12CD12C76018E010F5FDA
:10BE80001F4F28E736E044E756E060E776E08CE6AF
:10BE900096E00E94BAB88FEF809310010E94261995
:10BEA0008091260482FFC4C08091230481111DC0AB
:10BEB00091E090932304809145028927809328067E
:10BEC0001092450283E080935B01109226040E9449
:10BED000B0C16C507E4F8F4F9F4F6093270470937B
:10BEE00028048093290490932A0480914102909120
:10BEF0004202A0914302B0914402A5019401281B83
:10BF0000390B4A0B5B0BDA01C901B7FF05C0809101
:10BF10006A04882309F4D2C1D501C4018C599F4F0A
:10BF2000AF4FBF4F8093410290934202A0934302D0
:10BF3000B093440260912404062E000C770B77FF27
:10BF400003C0719561957109909124048091220438
:10BF5000981371C0633008F06EC010922404809171
:10BF6000240480932204643008F075C08091280670
:10BF70008111F3C08091CA159091CB158F529246D2
:10BF800041F480911101882309F4F9C08150809314
:10BF900011010E94B428C090A006D090A106E090A4
:10BFA000A206F090A30681110E94A477D701C601D2
:10BFB0003AE0B695A795979587953A95D1F700976A
:10BFC00041E0A407B10520F08FEF9FEFA0E0B0E0C3
:10BFD0009695879520915B012111E3C030916A0409
:10BFE00031119AC18091CA159091CB158F5292460A
:10BFF00009F479C180912A06811175C180911E04CE
:10C0000090911F04A0912004B0912104881A990AEC
:10C01000AA0ABB0AB7FC75C10E943D4672C1809155
:10C020005C0190915D01A0915E01B0915F011FCF15
:10C03000109223045ACF633009F091CF80912404E9
:10C0400087FD07C081E0880F880F8093240464E097
:10C0500086CF8FEFF8CF8091400621E030E040E0BE
:10C0600050E0882309F456C0C0903C06D0903D06AD
:10C07000E0903E06F0903F06C114D104E104F104C3
:10C08000E9F170E090E080E00E94B2E020E030E072
:10C0900040E85EE30E9413E12B013C01C501B401BD
:10C0A0006C197D098E099F090E94B2E09B01AC01C9
:10C0B000C301B2010E9427E820E030E04AE754E4DF
:10C0C0000E9413E16B017C0120E030E042E053E488
:10C0D0000E9427E924E630E040E050E087FF12C0EC
:10C0E00020E030E040EA52E4C701B6010E9427E9AF
:10C0F0002AE030E040E050E087FF04C021E030E07B
:10C1000040E050E080923C0690923D06A0923E06B0
:10C11000B0923F06A09124040A2E000CBB0B0E9493
:10C1200041E724E030E040E050E00E9417E78091D2
:10C13000300690913106A0913206B0913306820FFD
:10C14000931FA41FB51F8093300690933106A093D0
:10C150003206B093330610922404D501C4018856E8
:10C16000954CAF4FBF4F80931E0490931F04A09334
:10C170002004B093210481E080935B01FBCE8CE02E
:10C180008093110180911C0490911D04009729F067
:10C19000019790931D0480931C0481E080935B01C0
:10C1A000F8CE009741F040911C0450911D044817AF
:10C1B000590708F017CF80916A0481111DC0223001
:10C1C00038F0243008F44CC0243011F410925B0194
:10C1D00080910916811105C081E0809309160E94A3
:10C1E000F9C28091D2159091D3150E94D2C281E0FC
:10C1F00080932F0680936A0483E00E94F66F81E0AB
:10C200008093F015E091CA15F091CB150995109225
:10C210002F0680916A04811127C010922806809110
:10C22000CA159091CB158F52924609F0E3CE0E9429
:10C23000B0C1DC01CB0188199909AA09BB09C090DA
:10C240001C04D0901D04F12CE12CC816D906EA0676
:10C25000FB0608F0C7CE90931D0480931C04C2CE49
:10C2600081E080935B01B4CF80ED95E10E9443C6ED
:10C2700091E0811101C090E090936A04882369F2F3
:10C280008091CA159091CB158F529246B9F40E94B5
:10C29000B0C1DC01CB0188199909AA09BB09C0907A
:10C2A0001C04D0901D04F12CE12CC816D906EA0616
:10C2B000FB0620F490931D0480931C040F900F90B4
:10C2C0000F900F90DF91CF911F910F91FF90EF9002
:10C2D000DF90CF90BF90AF909F908F907F906F90A6
:10C2E0005F904F90089548E9840E4AE3941EA11C84
:10C2F000B11C80921E0490921F04A0922004B09260
:10C30000210480916A048111D9CF80915B01813031
:10C31000A9F610925B01D2CF009709F46DCF43CFFD
:10C32000CF938091E903811154C0109207161092A7
:10C330000816109209161092D5151092D415109265
:10C34000D7151092D6151092D91581E08093D81583
:10C3500082E28093DA151092DF151092DE15E3EF7A
:10C36000F5E121E036E18FEF81932E173F07E1F7EA
:10C37000C1E0C093F01524EF36EA3093E615209320
:10C38000E515C093E7151092E8151092E91590E4B1
:10C390009093EA151092EB1522EC36EA30930216D0
:10C3A0002093011628E031E03093D3152093D21565
:10C3B0009EE19093F71591E19093F8159CE190938D
:10C3C000F5158093F4158093F3150E94F9C2C0937C
:10C3D000E90381E08093400287ED91E09093FC14A3
:10C3E0008093FB141092FE141092FD1453985B9AE4
:10C3F00052985A9A3898409A0E942619109224040A
:10C40000CF910895FC01A081B1811C92A281B381DA
:10C410008C918F5F8C930280F381E02D90818CE072
:10C42000989F800D1124ECECF5E113AE84AF0895D4
:10C43000FC0180E09491992331F0907C903809F0D0
:10C440008F5F3196F7CF0895FC0180E09191992399
:10C4500029F0907C9038D1F38F5FF8CF08954F92F8
:10C460005F926F927F928F929F92AF92BF92CF9284
:10C47000DF92EF92FF920F931F93CF93DF9300D041
:10C4800000D01F92CDB7DEB71092400680912806EB
:10C49000109228068823E9F020E040E070E060E098
:10C4A00085E49CE50F900F900F900F900F90DF9117
:10C4B000CF911F910F91FF90EF90DF90CF90BF90A1
:10C4C000AF909F908F907F906F905F904F900C9463
:10C4D00005182091160130911701409130065091B6
:10C4E0003106CA01820F931F2436310509F015C4A5
:10C4F0004730510544F006978A3091050CF01CC472
:10C500008AE090E023C406964A3F5F4FACF38091E7
:10C510002F06882309F4C0C120915E0630915F0682
:10C52000409160065091610660916C0670916D06B5
:10C5300080916E0690916F060E94A4E74B015C010A
:10C540002091620630916306409164065091650621
:10C5500060917006709171068091720690917306D9
:10C560000E94A4E769837A838B839C83209166066B
:10C570003091670640916806509169066091740693
:10C580007091750680917606909177060E94A4E7D7
:10C590002B013C0120E030E040E251E40E9413E135
:10C5A00020E030E048EC52E40E9413E16B017C0192
:10C5B00020E030E0A901C301B2010E94ADE020E01B
:10C5C00030E040EA50EC87FD04C020E030E040EA73
:10C5D00050E4C701B6010E94A4E720E030E040E249
:10C5E00051E40E9427E80E9499E82B013C0180E277
:10C5F00077FE09C07094609450944094411C511C83
:10C60000611C711C8DE28093340660E2F0E14F16EC
:10C61000F7E25F06610471048CF0C301B20120E10E
:10C6200037E240E050E00E9417E7CA01B9012AE072
:10C6300030E040E050E00E9417E7605D609335060F
:10C6400060E228EE421623E05206610471048CF089
:10C65000C301B20128EE33E040E050E00E9417E74A
:10C66000CA01B9012AE030E040E050E00E9417E73B
:10C67000605D60933606C301B20124E630E040E01D
:10C6800050E00E9417E76AE0C62ED12CE12CF12C75
:10C69000CA01B901A70196010E9417E7605D609386
:10C6A0003706C301B201A70196010E9417E76D8307
:10C6B000CA01B901A70196010E9417E7CD80CC20DD
:10C6C00009F454C38EE280933806605D60933906A6
:10C6D0002C2D205D20933A0664E376E080E194E01F
:10C6E0000E94FFE920E030E0A901C501B4010E94E9
:10C6F000ADE020E030E040E05FEB87FD04C020E0EB
:10C7000030E040E05FE3C501B4010E94A4E70E946D
:10C7100099E8CB010E942115BC018BE094E00E94B6
:10C72000FFE920E030E0A90169817A818B819C8159
:10C730000E94ADE020E030E040E05FEB87FD04C008
:10C7400020E030E040E05FE369817A818B819C8169
:10C750000E94A4E70E9499E8CB010E942115BC0128
:10C7600086E094E00E94FFE9409146024F774983BA
:10C77000411127C00E94F977882319F180911C1775
:10C7800090911D17A0911E17B0911F170097A1053A
:10C79000B105B9F0BC01CD016D597F4F8F4F9F4F4F
:10C7A00024E630E040E050E00E94F5E6609120177A
:10C7B0007091211780912217909123170E94F5E61E
:10C7C00029830E946045B62E872E982EA92E6D8350
:10C7D00080910F01C9808C15C1F0C0920F0128E42F
:10C7E000C29EB001112490E080E00E94B2E02AE0F5
:10C7F00037ED43E25CE30E9413E10E94A0E86093FE
:10C800000504C110C5C21092000480910E01CD80B4
:10C81000C81609F441C0B0920E016B2D782D892DF8
:10C820009A2D20E13EE040E050E00E94F5E66901EB
:10C830002CE3422E512C612C712C6B2D782D892DDF
:10C840009A2DA30192010E94F5E6CA01B901A30144
:10C8500092010E94F5E624E6C216D10408F0BFC298
:10C860007F936F93DF92CF9281EE91E09F938F93AE
:10C8700080EF93E09F938F930E9444E00FB6F8946B
:10C88000DEBF0FBECDBF85E0982F990F990F891B92
:10C89000880F80588093EF030E94B0C10091EB0392
:10C8A0001091EC032091ED033091EE036B017C01BC
:10C8B000C01AD10AE20AF30A9701860137FD11C0B6
:10C8C0002091EA0320952093EA036A547C4F8F4F0E
:10C8D0009F4F6093EB037093EC038093ED03909371
:10C8E000EE03D090EA03D98281E00E94F66F809136
:10C8F0000416843158F480910616883038F026E604
:10C9000032E04CE068E080E50E9471C3809104163B
:10C910008431A0F480910616823080F0E980EE2008
:10C9200031F08091A40620E332E0811102C02AEFA9
:10C9300031E042E162E088E60E9471C38091041612
:10C940008C3108F0D0C0E0900915F0900A158830BD
:10C9500028F580910B1590910C150E94A015FC01F3
:10C96000808193E0803229F4818192E0803209F461
:10C9700091E043E050E0491B51094E0F5F1F892FA2
:10C98000880F880F981B892F67E0815F0E9479725A
:10C9900069E070E080E090E00E94077080910416EA
:10C9A0008C3130F580910616843110F1C7010E9458
:10C9B000A015FC01808193E0803229F4818192E00E
:10C9C000803209F491E043E050E0491B51094E0FD9
:10C9D0005F1F892F880F880F981B892F6CE1815F5B
:10C9E0000E94797269E070E080E090E00E94077038
:10C9F000E0900206F090030680910416883028F536
:10CA000080910406909105060E94A015FC0180818A
:10CA100093E0803229F4818192E0803209F491E040
:10CA200043E050E0491B51094E0F5F1F892F880FCB
:10CA3000880F981B892F67E0865A0E94797269E0F7
:10CA400070E080E090E00E940770809104168C31C5
:10CA500030F580910616843110F1C7010E94A015AF
:10CA6000FC01808193E0803229F4818192E0803260
:10CA700009F491E043E050E0491B51094E0F5F1F5C
:10CA8000892F880F880F981B892F6CE1865A0E9486
:10CA9000797269E070E080E090E00E940770809118
:10CAA00004168C3100F5809106168431E0F08091F7
:10CAB000A4068823C1F024E6829FC0011124815876
:10CAC0009F4F6FEF70E00E9486E7CB010E94A01598
:10CAD000AC016CE187E60E94797265E270E080E06B
:10CAE00090E00E9407700E94F977882369F1809195
:10CAF0000416843348F5809106168A3228F107E03F
:10CB000028E04AE26AE280ED95E10E947AC405E0FD
:10CB100022E04CE262E380ED95E10E947AC46AE093
:10CB20008AE20E9433C46091D2157091D31582E3DA
:10CB30008093EC158BE28093ED152CEE35E142E30A
:10CB400080ED95E10E94CEC280910416853340F4B9
:10CB500080910616813320F06AE486E30E9433C494
:10CB600080910416843368F480910616823348F06D
:10CB700002E02091050442E367E380ED95E10E9425
:10CB80007AC4809104168033D8F4809106168832D6
:10CB9000B8F080910004882361F040E054E060E345
:10CBA00087E30E94797265E270E080E090E00E9485
:10CBB000077040EF53E060E38091EF030E947972C9
:10CBC00080910416873208F055C0809106168F3187
:10CBD00008F450C083E08093071646E2409308169D
:10CBE00068E570E080E090E00E9407708BE0809341
:10CBF000071666E260930816C980CC2009F404C1C8
:10CC00008BE094E00E94387188E280930716F6E288
:10CC1000F093081669E570E080E090E00E940770EC
:10CC200080E38093071696E2C92EC0920816D98039
:10CC3000DD2009F40AC186E094E00E9438718DE499
:10CC400080930716F6E2F09308166AE570E080E03C
:10CC500090E00E94077085E58093071686E2C82E53
:10CC6000C0920816D980DD2009F412C180E194E059
:10CC70000E94387180910416833338F5809106162E
:10CC80008B3218F183E00E94F66F83E080930716E1
:10CC900083E38093081666E070E080E090E00E94F5
:10CCA000077081E00E94F66F809116019091170144
:10CCB0000E94A015AC0163E38CE00E94797265E2EA
:10CCC00070E080E090E00E9407708091041681344B
:10CCD00008F007C180910616863308F402C110924D
:10CCE00007168EE38093081688EC92E10E94246276
:10CCF000898360E870E088EC92E10E94DA70F98143
:10CD0000F53108F0EEC060E270E080E090E00E9453
:10CD1000077029812F5F2983F2CF243631054CF427
:10CD20008536910504F58A30910534F48AE090E067
:10CD300009C084369105BCF0883EE3E09E0714F0FC
:10CD400087EE93E02817390709F4E1CB9093170198
:10CD5000809316011092300610923106109232061E
:10CD600010923306D4CB84E690E0F0CF662351F0E6
:10CD70008EE280933806605D6093390680E280938E
:10CD80003A06AACC80E28093390680933806F6CF23
:10CD9000498180E2443628F0842F64E60E9458E7F7
:10CDA000805D80933806698190E26A3040F02AE025
:10CDB000862F622F0E9458E70E9458E7905D90935B
:10CDC000390689816AE00E9458E7905D90933A069F
:10CDD00068E376E080E094E00E94FFE916CD7F935F
:10CDE0006F93DF92CF9287ED91E09F938F9380EFC7
:10CDF00093E09F938F930E9444E00FB6F894DEBFB8
:10CE00000FBECDBF86E040CD87E00E943D3480FF5D
:10CE100013C00BE014E0F80161918F01662309F45F
:10CE2000F3CE6F320CF06FE3062E000C770B880BFD
:10CE3000990B0E940770EFCF8091450680FDE0CEF0
:10CE400085EF91E00E94D670DFCE87E00E943D34EE
:10CE5000869580FF13C006E014E0F80161918F0110
:10CE6000662309F4ECCE6F320CF06FE3062E000C53
:10CE7000770B880B990B0E940770EFCF80914506C6
:10CE8000869580FDD8CE85EF91E00E94D670D7CEF2
:10CE900087E00E943D348695869580FF17C080E12B
:10CEA00094E09A838983E981FA816191FA83E98325
:10CEB000662309F4DFCE6F320CF06FE3062E000C10
:10CEC000770B880B990B0E940770EDCF8091450678
:10CED0008695869580FDCACE8DEE91E00E94D67033
:10CEE000C9CE0F900F900F900F900F90DF91CF91C0
:10CEF0001F910F91FF90EF90DF90CF90BF90AF9078
:10CF00009F908F907F906F905F904F900895AF9219
:10CF1000BF92CF92DF92EF92FF920F931F93CF9326
:10CF2000DF93EC015B018A01FB01099587FD16C0C7
:10CF3000C82ED12CF12CE12C2196F801C082D1828F
:10CF4000E282F382CE01DF91CF911F910F91FF908A
:10CF5000EF90DF90CF90BF90AF900895982F907E84
:10CF6000903CA9F48F7190E0B0E0A0E06C017D01ED
:10CF700056E0CC0CDD1CEE1CFF1C5A95D1F7CE01FF
:10CF80000196F50109958F73C82A2296D6CF982F5E
:10CF9000907F903E11F58F7090E0B0E0A0E06C01C2
:10CFA0007D0136E0CC0CDD1CEE1CFF1C3A95D1F760
:10CFB000CE010196F50109958F73C82A46E0CC0C85
:10CFC000DD1CEE1CFF1C4A95D1F7CE010296F5013F
:10CFD00009958F73C82A2396B0CF982F987F903FDA
:10CFE00079F5877090E0B0E0A0E06C017D0186E00B
:10CFF000CC0CDD1CEE1CFF1C8A95D1F7CE010196EE
:10D00000F50109958F73C82A96E0CC0CDD1CEE1C47
:10D01000FF1C9A95D1F7CE010296F50109958F7301
:10D02000C82A26E0CC0CDD1CEE1CFF1C2A95D1F78B
:10D03000CE010396F50109958F73C82A24967DCFFA
:10D04000982F907C903841F4807C803869F4219648
:10D05000CE01F5010995F8CF8E7F8D3F28F02196FE
:10D06000CE01F5010995F8CFC12CD12C760165CF01
:10D07000AF92BF92CF92DF92EF92FF920F931F93E6
:10D08000CF93DF9300D000D0CDB7DEB77C01062F61
:10D090006A01122F86E0A82EB12C11160CF040C0A8
:10D0A000AE014F5F5F4F62ED77E1C7010E94876776
:10D0B0007C0169817A818B819C8161157105810573
:10D0C000910571F16D3371058105910509F450C029
:10D0D0006E3771058105910509F44AC06A32710500
:10D0E0008105910569F507FF12C08DEC91E00E3FB7
:10D0F00011F089EC91E026E01202B00111240E94A7
:10D10000787066E070E00E9486E7161B61C065E4F7
:10D1100070E080E090E00E940770115059F510E037
:10D12000812F0F900F900F900F90DF91CF911F9153
:10D130000F91FF90EF90DF90CF90BF90AF90089548
:10D14000643271058105910579F4C114D10461F04F
:10D1500026E01202B0011124C6010E947870B501C8
:10D160000E9486E7161B99CF0E940770115095CF39
:10D1700007FDBBCF61E089819A81AB81BC81CD97EE
:10D18000A105B10509F460E0600F6A30ACF0115000
:10D19000862F6AE00E9464E7092F682F880F770BBB
:10D1A000605D7F4F072E000C880B990B0E94077063
:10D1B000112309F4B4CF602F062E000C770B605DAD
:10D1C0007F4F072E000C880B990B0E94077011509F
:10D1D000112309F4A4CF86E01802B0011124C7017D
:10D1E0000E94787066E070E00E9486E7161B98CF78
:10D1F00011980000000087FD52C041980000000017
:10D20000119A0000000011980000000086FD53C034
:10D21000419800000000119A0000000011980000E1
:10D22000000085FD46C0419800000000119A0000F2
:10D23000000011980000000084FD39C041980000F2
:10D240000000119A0000000011980000000083FD0A
:10D250002CC0419800000000119A000000001198B5
:10D260000000000082FD1FC0419800000000119ADC
:10D270000000000011980000000081FD12C04198DC
:10D2800000000000119A000000001198000000004A
:10D29000419800000000119A000000000895419A92
:10D2A000ADCF419AEDCF419AE0CF419AD3CF419A89
:10D2B000C6CF419AB9CF419AACCF90E080E00895B3
:10D2C000CF93DF93DB01F9019C919130C1F0943051
:10D2D00080F094509C938830D1F4808191810097A4
:10D2E00071F0019791838083480F591FEA011882DA
:10D2F00006C08C3539F49C5F9C93943041F4DF91E7
:10D30000CF9108958B3339F781E08C93F8CF20814A
:10D310003181B9016F5F7F4F71836083420F531F6B
:10D32000EA018883808191818F3591056CF7E7CF81
:10D330000F931F9381E000912017109121172091E6
:10D3400022173091231740911C1750911D1760919F
:10D350001E1770911F17041715072607370708F4C3
:10D3600080E01F910F910895282F90916C058330D4
:10D3700021F495FD0FC094FD0FC0892F90E0B0E01F
:10D38000A0E004C0B695A795979587952A95D2F702
:10D390008170089581E0089580E008952F923F9272
:10D3A0004F925F926F927F928F929F92AF92BF92B5
:10D3B000CF92DF92EF92FF920F931F93CF93DF9361
:10D3C000CDB7DEB72E970FB6F894DEBF0FBECDBF38
:10D3D000E82ED62E042F122F282F30E03C872B87E3
:10D3E000462F50E05A87498765E0F62EF29EC0012D
:10D3F000F39E900D11249E878D87FA01E80FF91F87
:10D40000EE0FFF1FEE0FFF1FEF58FD4F6081718180
:10D41000828193819B01AC010E94A5E9882309F4D4
:10D4200034C1E00E612F6D0DFE9CF0011124A98521
:10D43000BA85AE0FBF1FAA0FBB1FAA0FBB1FAF58E5
:10D44000BD4FAC901196BC9011971296CC9012974C
:10D450001396DC90E00EFE9CA0011124A985BA85EC
:10D46000A40FB51FAA0FBB1FAA0FBB1FAF58BD4FFC
:10D47000EC901196FC90119712960C9112971396BE
:10D480009C90862F90E0AD85BE85A80FB91FAA0F8E
:10D49000BB1FAA0FBB1FAF58BD4F8C9011967C903D
:10D4A000119712966C90129713965C90610F70E032
:10D4B000AD85BE85A60FB71FAA0FBB1FAA0FBB1F46
:10D4C000AF58BD4F4C9011963C90119712961C91FD
:10D4D000129713962C90E80FF91FEE0FFF1FEE0F17
:10D4E000FF1FEF58FD4FB081B98321812A8332811C
:10D4F0003B8383818C83FA01E60FF71FEE0FFF1F3A
:10D50000EE0FFF1FEF58FD4F90819D83A181AE83E9
:10D51000B281BF83238128879701402F592DB701FE
:10D52000802F992D0E94A5E9882321F0E12CF12C70
:10D5300000E0912C9501A601B501C6010E94A5E964
:10D54000882319F05701C02ED92C242D332D412FBB
:10D55000522D642D732D812F922D0E94A5E98823D1
:10D5600021F0412C312C10E0212C282D372D462D77
:10D57000552D682D772D862D952D0E94A5E98823A0
:10D5800021F0842C732C612E522C2D813E814F81F1
:10D5900058856D817E818F8198850E94A5E98823B9
:10D5A00021F01D821E821F82188629813A814B81BB
:10D5B0005C8169817A818B819C810E94A5E98823A5
:10D5C00041F03D8139834E814A835F815B83888549
:10D5D0008C8385E0EB85FC858E9FD0018F9FB00DFD
:10D5E000112429853A85A20FB31FAA0FBB1FAA0FCA
:10D5F000BB1FAF58BD4FBA87A9879501A601B501DA
:10D60000C6010E94A4E79701402F592D0E94A3E76D
:10D610006B017C01282D372D462D552D682D772D3A
:10D62000862D952D0E94A4E7242D332D412F522DB8
:10D630000E94A3E79B01AC01C701B6010E94A4E7C9
:10D640006B017C0129813A814B815C8169817A81FE
:10D650008B819C810E94A4E72D813E814F8158855A
:10D660000E94A3E79B01AC01C701B6010E94A4E799
:10D6700020E030E040E450E40E9427E8A985BA8524
:10D680006D937D938D939C9313972E960FB6F8947C
:10D69000DEBF0FBECDBFDF91CF911F910F91FF90E5
:10D6A000EF90DF90CF90BF90AF909F908F907F9042
:10D6B0006F905F904F903F902F900895AF92BF92E0
:10D6C000CF92DF92EF92FF920F931F93CF93DF934E
:10D6D0006B01E9014A3009F4B8C0453109F06AC06C
:10D6E000DB011296ED91FC91F280C681D781139AED
:10D6F00088E28A950000E9F7BF2CB29420EFB222AD
:10D7000030E1A32EAF0C48E2E42E88EF0E94F868C7
:10D710008E2D8A950000E9F7BFE1BF1508F481C09E
:10D720008F2D807780680E94F8688B2D0E94F868A2
:10D730008E2D8A950000E9F780E80E94F86880E065
:10D740000E94F8688E2D8A950000E9F78AEF0E9402
:10D75000F8688E2D8A950000E9F78E01005F1F4F53
:10D760008881807F0E94F86889918295807F0E94DD
:10D77000F868C017D107A1F78E2D8A950000E9F748
:10D78000F394E0E1BE0EFA10C0CF1398D6011296C2
:10D79000CD91DC91CE010E949BC28111EEC1DF913F
:10D7A000CF911F910F91FF90EF90DF90CF90BF909E
:10D7B000AF900895FB0102811381423309F498C1AF
:10D7C00008F49CC1463409F489C1473409F48CC17A
:10D7D0004B3329F589812B81D80112966C911297D0
:10D7E00013964C91213009F4DFC1233009F0A9C10F
:10D7F00038EF380F582F91E0431708F490E041E0DC
:10D80000531708F040E031E0561708F430E0592F84
:10D81000542B352309F0BDC1942309F0BAC181E02E
:10D82000BECF80EE8F0D8068807F0E94F8688F2DBC
:10D830008295807F0E94F8688E2D8A950000E9F716
:10D8400080E80E94F86880E87BCF0B9A1398399A99
:10D850004198099A119A139A88E28A950000E9F78B
:10D8600088E790E0CEE9DFE0FE013197F1F701971C
:10D87000D9F788EF0E94F86818E2812F8A95000096
:10D88000E9F780E20E94F86880E00E94F868812F42
:10D890008A950000E9F780E00E94F86880E80E941D
:10D8A000F868812F8A950000E9F780E00E94F86807
:10D8B00080E10E94F868812F8A950000E9F7CE0187
:10D8C0000197F1F7CE010197F1F7CE010197F1F73A
:10D8D000CE010197F1F7CE010197F1F7CE01019743
:10D8E000F1F7CE010197F1F7CE010197F1F7CE01E3
:10D8F0000197F1F7CE010197F1F7CE010197F1F70A
:10D90000CE010197F1F7CE010197F1F7CE01019712
:10D91000F1F72197F1F780E20E94F86880E40E9415
:10D92000F868812F8A950000E9F780E20E94F86884
:10D9300080E60E94F8681A950000E9F710E0D0E050
:10D94000C8E28D2F807780680E94F868812F0E943E
:10D95000F8688C2F8A950000E9F780E80E94F86843
:10D9600080E00E94F8688C2F8A950000E9F78AEF22
:10D970000E94F8688C2F8A950000E9F780E21198E0
:10D9800000000000419800000000119A0000000013
:10D99000119800000000419800000000119A00005A
:10D9A0000000119800000000419800000000119A4A
:10D9B00000000000119800000000419800000000E5
:10D9C000119A00000000119800000000419800002A
:10D9D0000000119A0000000011980000000041981A
:10D9E00000000000119A00000000119800000000E3
:10D9F000419800000000119A0000000011980000FA
:10DA00000000419800000000119A000000001198E9
:10DA100000000000419800000000119A0000000082
:10DA2000119800000000419800000000119A0000C9
:10DA30000000119800000000419800000000119AB9
:10DA40000000000011980000000041980000000054
:10DA5000119A000000001198000000004198000099
:10DA60000000119A00000000119800000000419889
:10DA700000000000119A0000000011980000000052
:10DA8000419800000000119A000000001198000069
:10DA90000000419800000000119A000000009C2F37
:10DAA0009A950000E9F7815009F069CF88EF0E944C
:10DAB000F8688C2F8A950000E9F7DF5F105FD0329D
:10DAC00009F03FCF80E00E94F86880EC0E94F8687F
:10DAD000CA950000E9F7139881E061CED801159648
:10DAE0008C91888381E05BCEF80181818883FACFB5
:10DAF000B901C8010E94B8C281E051CE443171F031
:10DB0000473109F08CCE1882F801828189838581A2
:10DB100081508A8383818B8381E041CED801159621
:10DB20004C91159750E0440F551F70E060E0169639
:10DB30008D919C910E94CFE9C8010E94B1C281E001
:10DB40002ECE481708F46BCE861708F468CEFA80FC
:10DB5000E12CD12C243070F41DC0BE01C8010E94FC
:10DB6000B8C2898198819D0D98838E0D8983FF0CA1
:10DB700009F455CEF7FEF6CFF0CF4D8150E0440FBB
:10DB8000551F70E060E08E819F810E94CFE981E0A7
:10DB900006CEFA8030E0F901E151FE4FD0802551E8
:10DBA0003E4FF901E080E6CF58E0580F382F23CEE2
:10DBB000EF92FF920F931F93CF93DF93EC018B01B2
:10DBC0007A018A859B858617970731F0888199812C
:10DBD0000E9475C61B870A87B701888199810E94B8
:10DBE000ACBD2E813F81820F932F911D9F838E8329
:10DBF00090E080E0DF91CF911F910F91FF90EF9027
:10DC000008959F92AF92BF92CF92DF92EF92FF92D0
:10DC10000F931F93CF93DF93EC018B01942EA52ECE
:10DC20008A859B858617970731F0888199810E94A4
:10DC300075C61B870A8788859985019649F5BC803A
:10DC40000A818E81080FC880D980D6015596ED9142
:10DC5000FC91C6010995B80EE92CFA2C10E0F701E9
:10DC600021917F01211127C08E819F81810F911DFC
:10DC70009F838E8390E080E0DF91CF911F910F9181
:10DC8000FF90EF90DF90CF90BF90AF909F9008955E
:10DC90000E811F81692D7A2D888199810E94ACBDEA
:10DCA000800F912F911D288539852817390738F65F
:10DCB00081E090E0E1CF4B2D602FC6010E94CDC6E0
:10DCC000080F180FCCCFDF92EF92FF920F931F93A4
:10DCD000CF93DF93EC01D62E1CAD0BAD7C0184E01D
:10DCE000E80EF11CE98DFA8DC7010995412F480F07
:10DCF0002D2D602FC7010E94CDC69BAD890F8BAF24
:10DD000081E090E0DF91CF911F910F91FF90EF9014
:10DD1000DF900895EF92FF920F931F93CF937C01B2
:10DD200000916F0510917005C0E0F701EC0FF11D37
:10DD30006081662351F0062E000C770BC8010E940B
:10DD4000F4E9892B49F4CF5FF0CF80E0CF911F91A8
:10DD50000F91FF90EF90089581E0F8CF682F880F22
:10DD6000770B80916F05909170050E94F4E9FC019A
:10DD700081E0309709F480E0309781F0918120EDC7
:10DD8000290F2A3030F09E3251F4928190539A300C
:10DD900098F43196F0936705E093660508959D32F7
:10DDA00011F09B3249F4928120ED290F2A3088F33B
:10DDB0009E3211F49381EACFF0E0E0E0EBCF0E94D5
:10DDC000AE6E882341F081E02091660530916705B1
:10DDD000232B09F480E00895CF93DF9300D000D087
:10DDE000CDB7DEB780E090E0A0EAB0E489839A8303
:10DDF000AB83BC8361E0CE0101960E94DC350F90BD
:10DE00000F900F900F90DF91CF910895809166054C
:10DE100090916705009731F04AE050E070E060E0D3
:10DE20000C94CFDE60E070E0CB0108958091660530
:10DE300090916705009731F04AE050E070E060E0B3
:10DE40000C94A1DD60E070E0CB0108950E94166F94
:10DE500097FD0CC00E94166F6F3F710581059105FB
:10DE600009F034F40E94166F862F089580E008951B
:10DE70008FEF0895CF93C62F0E94DF6E882319F08D
:10DE8000CF910C94266F8C2FCF91089580916605C9
:10DE900090916705892B41F00E94266F91E08111D6
:10DEA00001C090E0892F089591E0FCCFCF93DF93DC
:10DEB000C82FD62F0E94DF6E882321F0DF91CF91EB
:10DEC0000C94466F8C2F0E94AE6E811101C08D2F75
:10DED000DF91CF9108950E94166FCB010895CF93E3
:10DEE000DF93EB010E94DF6E882321F0DF91CF9159
:10DEF0000C946B6FCE01DF91CF9108950F931F9318
:10DF0000CF9380916605909167050097E9F0FC0139
:10DF10008F01C1912C2F2F7D81F0C53411F0C536B2
:10DF2000B9F7F801108270E060E00E9443DCF8016C
:10DF3000C083CF911F910F91089570E060E0CF9161
:10DF40001F910F910C9443DC60E070E0CB01F1CFA6
:10DF5000CF92DF92EF92FF926A017B010E94DF6E07
:10DF6000882331F0FF90EF90DF90CF900C947E6F7C
:10DF7000C701B601FF90EF90DF90CF9008959CE02D
:10DF8000899F802D112491E0980F909375052CE0C6
:10DF9000280F2093410630E02E5F3F4F409104163A
:10DFA0004217130619F014F080E008952091061628
:10DFB0009217D0F7662341F08E5F0E941AC48091B9
:10DFC00041068E5F0E941AC480914106909104160A
:10DFD000891750F32091061690917505291720F3A3
:10DFE000109207168093081681E008952091740519
:10DFF000022E000C330B8217130641F08093740538
:10E0000064EA7CE180ED95E10C9475C60895CF92A9
:10E01000DF92EF92FF920F931F93CF93DF93CDB7D1
:10E02000DEB72C970FB6F894DEBF0FBECDBF6F3FA3
:10E0300071058105910509F0D0F48CEC95E10E9401
:10E04000636EE091D415F091D5153196849190E0EE
:10E050002C960FB6F894DEBF0FBECDBFDF91CF91E7
:10E060001F910F91FF90EF90DF90CF900895F09067
:10E070000716E09008162091400221110FC044E8D5
:10E080005CE16E2D8F2D0E9439C790E080E0F80E84
:10E09000F0920716E09208169927DACFC090D415AF
:10E0A000D090D51520ED35E13A8329832F2D30E02E
:10E0B0003C832B832E2D30E03E832D8318861F82D8
:10E0C0002FEF3FEF3A8729871C861B8601E01EE66B
:10E0D0009E012F5F3F4FAB01BC01C6010E9475B589
:10E0E000B60180ED95E10E9475C68F819885CFCFEE
:10E0F000CF92DF92EF92FF920F931F93CF93DF9314
:10E10000CDB7DEB72C970FB6F894DEBF0FBECDBFEC
:10E11000F0900716E09008162091400221111DC0D2
:10E1200044E65CE16E2D8F2D0E9439C790E080E0BF
:10E13000F80EF0920716E092081699272C960FB663
:10E14000F894DEBF0FBECDBFDF91CF911F910F912D
:10E15000FF90EF90DF90CF900895C090D415D090AD
:10E16000D51520ED35E13A8329832F2D30E03C830E
:10E170002B832E2D30E03E832D8318861F827A87D5
:10E1800069871C861B8601E01EE69E012F5F3F4FBC
:10E1900042ED57E1BC01C6010E9439B6B60180EDDF
:10E1A00095E10E9475C68F819885C2CF6FEF7FEF92
:10E1B0000C947870CF92DF92EF92FF920F931F939F
:10E1C000CF93DF93CDB7DEB72C970FB6F894DEBFB1
:10E1D0000FBECDBFF0900716E090081620914002C8
:10E1E00021111DC044E45CE16E2D8F2D0E9439C7C2
:10E1F00090E080E0F80EF0920716E092081699275A
:10E200002C960FB6F894DEBF0FBECDBFDF91CF9135
:10E210001F910F91FF90EF90DF90CF900895C090E5
:10E22000D415D090D51520ED35E13A8329832F2DD3
:10E2300030E03C832B832E2D30E03E832D831886E7
:10E240001F827A8769871C861B8601E01EE69E0175
:10E250002F5F3F4F45ED57E1BC01C6010E9439B623
:10E26000B60180ED95E10E9475C68F819885C2CF79
:10E270006FEF7FEF0C94DA70AF92BF92CF92DF9284
:10E28000EF92FF920F931F93CF93DF935C016B018B
:10E290000E941862E82EC6010E942462F12C03E15C
:10E2A00010E0081B1109C5E20E151F050CF4CFE1A3
:10E2B0008C2F90E09C012E5F3F4F40910416421737
:10E2C000130609F0CCF509972091061628171906B0
:10E2D0009CF1409143065091440660914206109291
:10E2E0000716C093081625E1C5010E943868D1E0E1
:10E2F000C114D104B1F06AE370E080E090E00E94C4
:10E3000007700E151F05D4F4C45F80910416C8175A
:10E3100040F0209106164C2F4950550B2417150636
:10E320007CF4DF91CF911F910F91FF90EF90DF90E0
:10E33000CF90BF90AF900895D0E0DACFDD2389F37E
:10E34000802F880F080F000F00930716C093081640
:10E3500060E270E080E090E00E940770C601DF910B
:10E36000CF911F910F91FF90EF90DF90CF90BF90D2
:10E37000AF900C9438718F929F92AF92BF92CF92D0
:10E38000DF92EF92FF920F931F93CF93DF93CDB75E
:10E39000DEB72C970FB6F894DEBF0FBECDBF982F17
:10E3A000862F5A017901D02E692F0E94BF6F8823D2
:10E3B00009F489C0C701002391F10E941862C82E98
:10E3C0008090D4159090D51580914002811145C060
:10E3D0001FEF23E12C1940914306509144066091B0
:10E3E0004206C5010E943868CC2009F46CC0B6E032
:10E3F0008B9F500111246AE370E080E090E00E945E
:10E40000077057E0A516B10408F444C060E270E05C
:10E4100080E090E00E940770A81AB90AF2CF0E942B
:10E420002462C82E8090D4159090D515809140021A
:10E43000882371F2FE0133968AE0DF011D928A95EE
:10E44000E9F780ED95E19A83898308ED1DE69E0149
:10E450002F5F3F4F45ED57E112C0FE0133968AE032
:10E46000DF011D928A95E9F780ED95E19A83898312
:10E4700008ED1DE69E012F5F3F4F42ED57E1B701CA
:10E48000C4010E9439B6B40180ED95E10E9475C6C1
:10E490001F819FCF40914106212F30E0A6E0CA9E08
:10E4A000C00111242E5F3F4F281739070CF49C013F
:10E4B00080E8821B8093071640930816C701DD2071
:10E4C000A9F00E94D6702C960FB6F894DEBF0FBE4E
:10E4D000CDBFDF91CF911F910F91FF90EF90DF9013
:10E4E000CF90BF90AF909F908F9008950E94387109
:10E4F000EACFECECF5E183AF64AFCA010C9438715C
:10E500000F931F93CF9310926E0510926D052FE31A
:10E510002093730510927205109271059C01F90108
:10E5200090812F5F3F4F9032D1F39E34C9F48181A7
:10E5300090ED980F9A3020F08D3211F08B3281F4EB
:10E5400032969F012F5F3F4F808180538A3008F4BD
:10E5500068C09F012F5F3F4F8081803209F463C004
:10E56000F0934F06E0934E068F010F5F1F4FC0815F
:10E570006AE270E0C8010E94F4E9009731F0FC0102
:10E58000319780818032E1F31182CD3429F0C43596
:10E5900019F0C73409F041C0F80180810F5F1F4FA7
:10E5A0008032D1F380538A30C0F5C093730530E0D8
:10E5B00020E06AE0AF014F5F5F4F629FC001639F41
:10E5C000900D11249C01205331098081280F311DA9
:10E5D00087FD3A95FA01808180538A3058F3309351
:10E5E000720520937105CA01FC01019640814032F9
:10E5F000D9F3F0937005E0936F05CD3401F52E311A
:10E60000310539F090F42731310519F02C313105FD
:10E61000B1F4F0936E05E0936D05CF911F910F91CA
:10E620000895F9018ECFF90194CF2537310538F0DF
:10E630002737310570F3203A83E0380751F350E073
:10E6400040E0CF0101966081662309F45AC061322F
:10E6500091F4CD3481F42032310569F490936E0544
:10E6600080936D0563E270E00E94F4E90097A9F2DF
:10E67000FC011082D2CFFC01DF018D91803271F05C
:10E6800090ED980F9A3008F18E3251F491819053A9
:10E690009A30D8F041155105E1F414C0FD01ECCFDA
:10E6A0008D3211F08B3259F4918160ED690F6A302F
:10E6B00060F09E3221F4928190539A3030F04115EF
:10E6C000510519F4AF014150510981548A3108F4C0
:10E6D000B8CFDF01FD018D91882309F4B2CF90ED11
:10E6E000980F9A30B8F393ED980F923098F38B32DD
:10E6F00089F3CF0101966081603209F0A2CFFC015D
:10E70000F8CF50936E0540936D0587CFFC0165915E
:10E71000759185919491089580914606882319F00A
:10E7200080E00E94DB4280E008954F925F926F92FA
:10E730007F928F929F92AF92BF92CF92DF92EF9291
:10E74000FF92CF93DF93CDB7DEB728970FB6F8943B
:10E75000DEBF0FBECDBF5C01DB01CD90DD90ED9043
:10E76000FC90E091B315F091B415FE83ED838481A4
:10E770009581A681B78189839A83AB83BC839C01F1
:10E78000AD01C701B6010E94A3E72B013C01F501D1
:10E7900080809180A280B380AD81BE818D919D915A
:10E7A0000D90BC91A02D8D839E83AF83B88727E108
:10E7B00037EB41ED58EBC301B2010E9427E987FD19
:10E7C000D0C027E030E04AE753E4C301B2010E9421
:10E7D000ADE018160CF4C5C02D813E814F815885DF
:10E7E000C501B4010E94A3E72B013C0127E137EBEF
:10E7F00041ED58EB0E9427E987FDB3C027E030E0E8
:10E800004AE753E4C301B2010E94ADE018160CF4CC
:10E81000A8C020E030E0A9016D817E818F819885BC
:10E820000E94A4E72B013C0120E030E040E450E4EA
:10E830000E94ADE087FF05C0412C512C30E4632ECF
:10E84000762C27E137EB41ED58E3C301B2010E947A
:10E85000A3E79B01AC01C501B4010E9427E987FD34
:10E8600080C020E030E04AE753E46D817E818F81F3
:10E8700098850E94A4E72B013C0120E030E043E6AC
:10E8800053E40E9427E9181634F4412C512C23E656
:10E89000622E23E4722E27E137EB41ED58E3C301EA
:10E8A000B2010E94A4E79B01AC01C501B4010E9422
:10E8B000ADE018160CF455C020E030E0A9016981E4
:10E8C0007A818B819C810E94A4E74B015C0120E04E
:10E8D00030E040E951E40E94ADE087FF06C0812CA2
:10E8E000912C90E9A92E91E4B92E27E137EB41ED67
:10E8F00058E3C501B4010E94A3E79B01AC01C70125
:10E90000B6010E9427E987FD2CC020E030E04AE7ED
:10E9100053E469817A818B819C810E94A4E74B0139
:10E920005C0120E030E044E553E40E9427E918163A
:10E9300034F4812C912C84E5A82E83E4B82E27E1B1
:10E9400037EB41ED58E3C501B4010E94A4E79B01F8
:10E95000AC01B1E0B983C701B6010E94ADE0181661
:10E960000CF41982898128960FB6F894DEBF0FBE89
:10E97000CDBFDF91CF91FF90EF90DF90CF90BF9010
:10E98000AF909F908F907F906F905F904F90089581
:10E990004F925F926F927F928F929F92AF92BF92AF
:10E9A000CF92DF92EF92FF920F931F93CF93DF935B
:10E9B000EC012091D5023091D6024091D7025091BE
:10E9C000D802688179818A819B810E94A3E76B01CB
:10E9D0007C012091D9023091DA024091DB02509102
:10E9E000DC026C817D818E819F810E94A3E74B01B7
:10E9F0005C01A701960160914201709143018091F1
:10EA00004401909145010E94ADE0882309F450C073
:10EA1000C0924201D0924301E0924401F09245013C
:10EA200020915E0530915F05409160055091610530
:10EA3000C701B6010E9413E12B013C010E94CFE8FF
:10EA40006B017C0120E030E0A9010E94ADE087FD70
:10EA500070C020E030E040E450E4C701B6010E94FD
:10EA600027E918162CF4C12CD12CC0E4EC2EFE2C76
:10EA7000A7019601C301B2010E94A3E76093560566
:10EA8000709357058093580590935905C701B601B7
:10EA90000E9499E860935405062E000C770B6F5F77
:10EAA0007F4F6430710514F064E070E060935205AC
:10EAB000D091400110915405A50194016091460147
:10EAC0007091470180914801909149010E94ADE009
:10EAD000811133C0D11381C020913A0530913B059B
:10EAE00040913C0550913D05609156057091570548
:10EAF00080915805909159050E9413E120913E059F
:10EB000030913F0540914005509141050E94A4E796
:10EB1000DF91CF911F910F91FF90EF90DF90CF90F9
:10EB2000BF90AF909F908F907F906F905F904F902D
:10EB30000895C12CD12C76019BCF809246019092F2
:10EB40004701A0924801B09249012091620530919D
:10EB500063054091640550916505C501B4010E94AB
:10EB600013E14B015C010E94CFE86B017C0120E0C6
:10EB700030E0A9010E94ADE087FDF3C020E030E065
:10EB800040E450E4C701B6010E9427E918162CF4AE
:10EB9000C12CD12CB0E4EB2EFE2CA7019601C501AF
:10EBA000B4010E94A3E760935A0570935B058093BC
:10EBB0005C0590935D05C701B6010E9499E86093DA
:10EBC0005505062E000C770B6F5F7F4F6430710583
:10EBD00014F064E070E060935305C0915505D113C3
:10EBE00005C0809141018C1709F470C080915405D3
:10EBF0009091550590934101809340010C2E000C9B
:10EC0000DD0B25E01203C0011124FC01EC0FFD1FF8
:10EC1000EE0FFF1FEE0FFF1FEF58FD4F20813181D8
:10EC20004281538120934E0530934F054093500508
:10EC30005093510500915305002E000C110BFC015F
:10EC4000E00FF11FEE0FFF1FEE0FFF1FEF58FD4FFC
:10EC500060817181828193810E94A3E760934A055C
:10EC600070934B0580934C0590934D052091520570
:10EC700035E02303F0011124CE0FDF1FCC0FDD1F81
:10EC8000CC0FDD1FCF58DD4F288139814A815B8150
:10EC90002093460530934705409348055093490516
:10ECA000E00FF11FEE0FFF1FEE0FFF1FEF58FD4F9C
:10ECB00060817181828193810E94A3E76093420504
:10ECC00070934305809344059093450580905A05C1
:10ECD00090905B05A0905C05B0905D0520914A0581
:10ECE00030914B0540914C0550914D05C501B40143
:10ECF0000E9413E120914E0530914F05409150053F
:10ED0000509151050E94A4E76B017C01C0923E0521
:10ED1000D0923F05E0924005F092410520914205D6
:10ED2000309143054091440550914505C501B4011A
:10ED30000E9413E120914605309147054091480516
:10ED4000509149050E94A4E7A70196010E94A3E7FC
:10ED500060933A0570933B0580933C0590933D0585
:10ED6000BBCEC12CD12C760118CF1F93CF93DF934C
:10ED7000CDB7DEB72C970FB6F894DEBF0FBECDBF70
:10ED8000182F882379F020E030E0A9016091DD029E
:10ED90007091DE028091DF029091E0020E94ADE06E
:10EDA0008823F9F080916B028117D9F00E948D269B
:10EDB0008CE0EFECF1E0DE01119601900D928A9566
:10EDC000E1F7CE0101960E94C87480916B028823FE
:10EDD00091F08CE696E00E94C62610926B020E948B
:10EDE000B4362C960FB6F894DEBF0FBECDBFDF91C0
:10EDF000CF911F91089581E080936B028CE696E09D
:10EE00000E94AE26ECCF80E00E94B5761092D90227
:10EE10001092DA021092DB021092DC021092D502FC
:10EE20001092D6021092D7021092D8021092E102EC
:10EE30001092E2021092E3021092E4021092DD02BC
:10EE40001092DE021092DF021092E002E1E7F2E09F
:10EE500025ED32E080E090E0A0ECBFE78083918375
:10EE6000A283B38384839583A683B78380879187A6
:10EE7000A287B38784879587A687B787808B918B76
:10EE8000A28BB38B74962E173F0741F708958F928C
:10EE90009F92AF92BF92CF92DF92EF92FF92C0907B
:10EEA000DD02D090DE02E090DF02F090E00220E090
:10EEB00030E0A901C701B6010E94ADE08823E1F16D
:10EEC000A701960160E070E080E89FE30E9427E8D8
:10EED0006B017C018090E1029090E202A090E3023D
:10EEE000B090E40220E030E0A901C501B4010E9425
:10EEF000ADE0882329F1A501940160E070E080E88D
:10EF00009FE30E9427E8C0925E05D0925F05E092E1
:10EF10006005F092610560936205709363058093CC
:10EF2000640590936505FF90EF90DF90CF90BF90C0
:10EF3000AF909F908F900895C12CD12C7601CACFAD
:10EF400060E070E0CB01DFCFEFE6F0E0808182602F
:10EF50008083089580914B0690914C06892B79F41B
:10EF600080914B0690914C06892B49F420914B06D9
:10EF700030914C0681E0232B19F480E0089581E064
:10EF80000895CF92DF92EF92FF926B017C0183E3B1
:10EF9000C816D104E104F10470F082E3C81AD10864
:10EFA000E108F10862E370E080E090E00E9415C1A2
:10EFB0000E94B636ECCFC701B6010E9415C1FF9082
:10EFC000EF90DF90CF900C94B6365E9A8091450614
:10EFD0008E7F809345065E9A809145068D7F809353
:10EFE0004506159A809145068B7F809345065E9A6B
:10EFF00008959091241793FB882780F993FF06C00A
:10F0000081E090911F15911101C080E008950E9448
:10F01000F977882339F08091241782FB882780F9BB
:10F0200091E08927089581E00895DC01EC918E2F0D
:10F0300090E0FC01EE0FFF1FE80FF91FE158FA4EB8
:10F0400080818F77808308951092900082E0809372
:10F0500091001092950010929400C19AE1E7F0E0BF
:10F0600080818260808308957F928F929F92AF9279
:10F07000BF92CF92DF92EF92FF920F931F93CF93A5
:10F08000DF93EC017B0188818C3008F0C4C090E0F4
:10F09000FC01EE0FFF1FE80FF91FE158FA4E8081C7
:10F0A0008F770E9420B819821A8288812CE0622F03
:10F0B0000E9458E7829FB001112430E020E0AB01AC
:10F0C000420F531FFA01EE0FFF1FE40FF51FE15827
:10F0D000FA4E908197FD09C02F5F3F4F2C303105CC
:10F0E00071F7811102C00E9424787880072D10E00A
:10F0F0006801CC0CDD1CF601E00FF11FE158FA4E5F
:10F1000080818068808377FC86C080E2E81682E098
:10F11000F8060CF03FC08A8128E532E0281B31094F
:10F1200087FD3395220F331F220F331F032E000C50
:10F13000440B550B898178E8872E912C881A910809
:10F1400087FD9394880C991C880C991C092C000C41
:10F15000AA08BB0860E070E0CB01F7FC0AC0B70169
:10F16000653B710514F064EB70E0072E000C880B12
:10F17000990B281939094A095B090E94E5E624EB35
:10F1800030E040E050E00E9417E7820E931EA41E7C
:10F19000B51E74018BE08715D8F0298188E890E0CE
:10F1A000821B910927FD9395880F991F880F991F3E
:10F1B000E816F90604F502972FB7F894E601C00F98
:10F1C000D11FC158DA4E880F991F9A8389832FBFA8
:10F1D00062E370E080E090E0DF91CF911F910F91AA
:10F1E000FF90EF90DF90CF90BF90AF909F908F9067
:10F1F0007F900C94C1772A8188E592E0821B910967
:10F2000027FD9395880F991F880F991FE816F90617
:10F2100094F6C701D0CFDF91CF911F910F91FF904E
:10F22000EF90DF90CF90BF90AF909F908F907F90A6
:10F230000895CF93DF93EB01682F70E084EA95E1A6
:10F240000E943478688179818A819B81643F21E0C2
:10F2500072078105910520F464EF71E080E090E091
:10F260000E94C17786B182958170DF91CF91089518
:10F27000CF93DF9300D000D0CDB7DEB78EEE92E013
:10F28000A0E0B0E089839A83AB83BC83BE016F5F4B
:10F290007F4F8AE50E9419790F900F900F900F9081
:10F2A000DF91CF910895CF93DF9300D000D0CDB7F9
:10F2B000DEB78EEE92E0A0E0B0E089839A83AB8364
:10F2C000BC83BE016F5F7F4F8AE00E9419790F9067
:10F2D0000F900F900F90DF91CF910895CF93DF9310
:10F2E00000D000D0CDB7DEB784EF91E0A0E0B0E071
:10F2F00089839A83AB83BC83BE016F5F7F4F8CE3AE
:10F300000E9419790F900F900F900F90DF91CF917D
:10F310000895CF93DF9300D000D0CDB7DEB784EF50
:10F3200091E0A0E0B0E089839A83AB83BC83BE0107
:10F330006F5F7F4F80EA0E9419790F900F900F90B6
:10F340000F90DF91CF9108951F920F920FB60F92F9
:10F3500011240BB60F922F933F934F935F936F93AC
:10F360007F938F939F93AF93BF93EF93FF9380917E
:10F37000270587FF27C01092950010929400809176
:10F3800027058F5F8093270580912705082E000CA5
:10F39000990B2091A3152817190629F024F08091C4
:10F3A00027058C30DCF180919400909195000496B3
:10F3B00080349C4908F47DC0809194009091950020
:10F3C000049679C080912705082E000C990B209196
:10F3D000A3152817190699F294F2E09127058E2FAC
:10F3E000EE0F990BFC01EE0FFF1FE80FF91FE1581C
:10F3F000FA4E808187FFC3CFE09127058E2FEE0F55
:10F40000990BFC01EE0FFF1FE80FF91FE158FA4EB0
:10F41000808160E08F770E94B9C0B1CF20919400C5
:10F4200030919500E09127058E2FEE0F990BFC018E
:10F43000EE0FFF1FE80FF91FE158FA4E818192810C
:10F44000820F931F9093990080939800E091270575
:10F450008E2FEE0F990BFC01EE0FFF1FE80FF91F27
:10F46000E158FA4E808187FF11C0E09127058E2F69
:10F47000EE0F990BFC01EE0FFF1FE80FF91FE1588B
:10F48000FA4E808161E08F770E94B9C0FF91EF91C1
:10F49000BF91AF919F918F917F916F915F914F91AC
:10F4A0003F912F910F900BBE0F900FBE0F901F90AA
:10F4B000189580E49CE990939900809398008FEFD1
:10F4C00080932705E3CF9091C00095FFFCCF8093F8
:10F4D000C6000895CF93DF93EC018991882319F03A
:10F4E0000E94637AFACF8DE00E94637A8AE0DF910E
:10F4F000CF910C94637ACF93DF93EC01FE0184915A
:10F500002196882319F00E94637AF8CFDF91CF917A
:10F510000895E0919B0C81E6E89FF0011124E350EF
:10F52000F34F8081811107C08EEE94E20E947B7AB6
:10F530008AE00C94637A0895AF92BF92CF92DF92E3
:10F54000EF92FF920F931F93CF93DF938BE194E1A0
:10F550000E947B7AC0E0D7E0D15021F080E20E9487
:10F56000637AFACF8C2F0E94C7C7CF5FC53099F757
:10F570008AE00E94637A01E712E0C0E080E20E9424
:10F58000637A8C2F0E94C7C75801D5E080E20E94A1
:10F59000637AF501C080D180E280F380A7019601F3
:10F5A000C701B6010E94A5E9882369F180E20E94A3
:10F5B000637A8DE30E94637A8DE30E94637A8DE320
:10F5C0000E94637A8DE30E94637A8DE30E94637ADE
:10F5D000D150F4E1AF0EB11CD111D8CF8AE00E9416
:10F5E000637ACF5F0C5F1F4FC53041F68AE0DF9131
:10F5F000CF911F910F91FF90EF90DF90CF90BF9030
:10F60000AF900C94637A20E030E0A901C701B60105
:10F610000E9427E987FD03C08BE20E94637A43E0E2
:10F62000C701B6010E945E22D3CFCF92DF92EF9244
:10F63000FF926A017B010E947B7A42E0C701B6011A
:10F64000FF90EF90DF90CF900C945E22CF93DF93EA
:10F65000EB010E947B7ACE01DF91CF910C9416B71B
:10F6600084E194E10C947B7A8EE094E10C947B7AB3
:10F67000CF9384E50E94DF6EC0E08823D9F00E941A
:10F68000266FC82F1816B4F40E94347B8DE40E94B4
:10F69000637A80917105909172050E94CEC76C2F9C
:10F6A000CC0F770B8AE995E10E94267B8AE00E94C5
:10F6B000637ACFEF8C2FCF9108952F923F924F9284
:10F6C0005F926F927F928F929F92AF92BF92CF92F2
:10F6D000DF92EF92FF920F931F93CF93DF93CDB7FB
:10F6E000DEB766970FB6F894DEBF0FBECDBF83E5D9
:10F6F0000E94AE6E8A83882309F4FCC00E94466F84
:10F70000898380906C0690906D06A0906E06B090F4
:10F710006F0640907006509071066090720670906F
:10F7200073068091740690917506A0917606B0914B
:10F730007706898B9A8BAB8BBC8B9A81992331F09E
:10F74000A981A11103C080E00E94B57686E50E94E0
:10F75000AE6E8A8720E030E0A9016091DD027091F1
:10F76000DE028091DF029091E0020E94ADE08823EA
:10F7700009F4C3C083E40E94AE6E882309F4A3C0D9
:10F780000E947E6F6D877E878F87988BE1E7F2E01E
:10F79000FD83EC83FB83EA8305E0312C212C18ECFC
:10F7A00092EC9E8B1E821F82A8ECA887B2E4B987D8
:10F7B000EA81FB81FC87EB87F5E0FD8BAB85BC859F
:10F7C000CD90DD90ED90FD90BC87AB872E813F8181
:10F7D00048855985C701B6010E94ADE087FF04C086
:10F7E000CE82DF82E886F986232D322D412F5E8975
:10F7F000C701B6010E9427E9181624F43C2C2D2CD1
:10F800001E2DFE8ABD89B150BD8BB111D7CF0150DD
:10F81000EA81FB817496FB83EA830111C9CF232D12
:10F82000322D412F5E896E817F81888599850E9466
:10F83000A4E720E030E040E05FE30E9413E12D8583
:10F840003E854F8558890E94A4E76B017C012DEB12
:10F8500037E346E855EB0E9427E987FD0AC02DEB08
:10F8600037E346E855E3C701B6010E94ADE018163C
:10F8700054F580E00E94B57695E0392E8C819D810B
:10F880009B838A8385E0282EAA81BB816D917D911F
:10F890008D919D91BB83AA838D0104501109A7010D
:10F8A00096010E94A3E7F8016083718382839383AA
:10F8B0002A942110E9CF3A948C819D8144969D83AE
:10F8C0008C833110DBCFBA85BB2381F020E030E0A0
:10F8D000A9016091DD027091DE028091DF029091BA
:10F8E000E0020E94ADE081110E949C7A89810E9411
:10F8F000B5760FC080916B0203CF9981911103C03F
:10F90000AA85AA2399F30E94347B8BED94E10E948F
:10F910007B7AE981EE2351F080916B02811106C060
:10F920000E94307B8CEB94E10E947B7A0E94347BB6
:10F930008EEA94E10E947B7A80916B0281114DC026
:10F940008DEA98E10E947B7A8AE00E94637AA501A1
:10F95000940160916C0670916D0680916E06909195
:10F960006F060E94ADE081111EC0A301920160915B
:10F9700070067091710680917206909173060E94D4
:10F98000ADE0811110C029893A894B895C89609169
:10F9900074067091750680917606909177060E94A4
:10F9A000ADE08823E9F066960FB6F894DEBF0FBE8F
:10F9B000CDBFDF91CF911F910F91FF90EF90DF901E
:10F9C000CF90BF90AF909F908F907F906F905F90FF
:10F9D0004F903F902F900C943F3D81EB98E1B2CF38
:10F9E00066960FB6F894DEBF0FBECDBFDF91CF9104
:10F9F0001F910F91FF90EF90DF90CF90BF90AF904D
:10FA00009F908F907F906F905F904F903F902F903E
:10FA100008950E94AF230E94E7458091F905813047
:10FA2000A1F40E94307B87E993E10E947B7A60E039
:10FA30008DE893E10E946E576EE571E080E090E002
:10FA40000E94C17788E08093F9050895CF92DF92F4
:10FA5000EF92FF921F93CF93DF9300D000D0CDB7EA
:10FA6000DEB78EEEC82E82E0D82EE12CF12CC982B2
:10FA7000DA82EB82FC82BE016F5F7F4F8AE50E94D3
:10FA8000197981110EC010E0812F0F900F900F9007
:10FA90000F90DF91CF911F91FF90EF90DF90CF906B
:10FAA00008950E948979C982DA82EB82FC82BE01C4
:10FAB0006F5F7F4F8AE50E941979182F882319F309
:10FAC0000E94307B81E794E10E947B7A0E94097D4D
:10FAD000DBCFCF92DF92EF92FF921F93CF93DF9312
:10FAE00000D000D0CDB7DEB78EEEC82E82E0D82E83
:10FAF000E12CF12CC982DA82EB82FC82BE016F5FBD
:10FB00007F4F8AE00E94197981110EC010E0812F89
:10FB10000F900F900F900F90DF91CF911F91FF905A
:10FB2000EF90DF90CF9008950E9489790E943879F4
:10FB30000E9453790E943879C982DA82EB82FC8272
:10FB4000BE016F5F7F4F8AE00E941979182F8823CA
:10FB5000E9F20E94307B84E394E10E947B7A0E9468
:10FB6000097DD5CFEC018B01F42E0E94AF230E94BA
:10FB7000307B8DE693E10E947B7A0115110511F42B
:10FB800002E715E2209711F4C4E6D3E10E949061E8
:10FB90001F930F93DF93CF9384E593E19F938F930C
:10FBA000D1E0DF930E9455570E943D46C091D11588
:10FBB000C695C6958DB79EB707960FB6F8949EBFAB
:10FBC0000FBE8DBF80910916811104C0D093091614
:10FBD0000E94F9C28091D2159091D3150E94D2C291
:10FBE000DC2FDD0F1D2F1C0F83E00E94F66F48EC09
:10FBF00052E16C2F80E00E94797210920716D09328
:10FC0000081685E493E10E94D670109207161093AF
:10FC1000081688E393E10E94D67080ED95E10E947A
:10FC200043C68111E1CF8BE593E10E9466B589EE71
:10FC300093E030E6019729F0232F2A950000E9F799
:10FC4000F9CFF89489EE93E038EE019729F0232F4D
:10FC50002A950000E9F7F9CF0E94AF23FF2021F099
:10FC60000E94E577A895FECF5E9AFCCF8091B10BFC
:10FC70009091B20B2FEF3FEF981751F0E92FF0E082
:10FC8000EF54F44F228130E09F5F9F779093B20B47
:10FC9000C90108951F920F920FB60F9211240F9071
:10FCA0000FBE0F901F9018951F920F920FB60F92D4
:10FCB00011240BB60F922F933F934F935F938F9323
:10FCC0009F93EF93FF938091C6004091B20B909168
:10FCD000B10B31E0390F3F77209126052C3008F029
:10FCE00072C0E22FF0E0E958F1480C949AE7837E65
:10FCF000AA7EB97EC47ECB7EE37ECF7EE37ED37EBA
:10FD0000D77EE37EDB7E803229F0E8F48A3011F082
:10FD10008D30F1F4431731F0E92FF0E0EF54F44F58
:10FD20008283932F9093B10BFF91EF919F918F91CD
:10FD30005F914F913F912F910F900BBE0F900FBE8F
:10FD40000F901F9018958D3481F021E08E3471F062
:10FD50002BE00CC08A3338F48033E0F68032D1F2E5
:10FD60008D32B1F7D7CF8D3499F722E02093260555
:10FD7000D1CF813329F0843329F0803249F7CACFBB
:10FD800023E0F4CF28E0F2CF24E0803379F326E0BB
:10FD9000813361F3DDCF25E08833D1F6E7CF27E06B
:10FDA0008233B1F6E3CF29E0813391F6DFCF2AE049
:10FDB000803371F6DBCF8A3019F08D3009F0AACF8D
:10FDC00010922605A7CF8A3019F08D3009F0A2CF06
:10FDD00050910A165523A1F3273049F02A3059F0E3
:10FDE000253071F710925A0110924502E9CF21E0B7
:10FDF0002093E702E5CF21E02093E602E1CF8EBD1C
:10FE00000DB407FEFDCF08958FEF8EBD0DB407FE34
:10FE1000FDCF8EB50895909164009B7F9093640010
:10FE2000982F906A96959CBD80FD03C091E0863026
:10FE300009F490E09DBD0895CF92DF92EF92FF927A
:10FE4000CF936B017C01C42F4A3069F4F7FE0BC0DD
:10FE5000F094E094D094C094C11CD11CE11CF11C1E
:10FE60008DE20E94637A4C2FC701B601CF91FF90BB
:10FE7000EF90DF90CF900C9460C7CF92DF92EF921B
:10FE8000FF926A017B010E947B7A4AE0C701B601BA
:10FE9000FF90EF90DF90CF900C941C7F2F923F92B9
:10FEA0004F925F926F927F928F929F92AF92BF928A
:10FEB000CF92DF92EF92FF920F931F93CF93DF9336
:10FEC000CDB7DEB7EB970FB6F894DEBF0FBECDBF50
:10FED00070E060E085E40E946F6F811171C283E57C
:10FEE0000E94DF6E882309F458C00E946B6F9A83CA
:10FEF000898365E070E083E40E946F6FB82E60E054
:10FF000085E50E94566F8FAB60E087E39CE10E941D
:10FF10006E5749815A81BA01550F880B990B0E947F
:10FF2000B4E06D837E831C010E94B0C16B877C8727
:10FF30008D879E8760915801709159016F507109AA
:10FF4000072E000C880B990B0E94B4E09B01AC01BA
:10FF50006D817E81C1010E9427E918161CF588EE8B
:10FF60009BE10E947B7AEB960FB6F894DEBF0FBE42
:10FF7000CDBFDF91CF911F910F91FF90EF90DF9058
:10FF8000CF90BF90AF909F908F907F906F905F9039
:10FF90004F903F902F900C94FDB924EB30E03A83C2
:10FFA0002983A7CF8B859C85AD85BE85805B9C43CF
:10FFB000AF4FBF4F8BAB9CABADABBEAB84ED9BE10A
:10FFC0000E947B7A0E94AF238FE780930D1581E01A
:10FFD00080935A014B845C846D847E844AA65BA620
:10FFE0006CA67DA61C8E1D8E1E8E1F8E18A219A2B9
:10FFF0001AA21BA219821A821B821C822FE730E0F0
:020000021000EC
:1000000040E050E02F87388B498B5A8B1F8230E4B9
:100010003D8B4CE14E8B56E45F8B188E198E1A8EF9
:100020001B8EFFE7CF2ED12CE12CF12C1EA61FA694
:1000300018AA19AA1AAA1DA21EA21FA218A68CA34A
:100040001C8A1B8A00E010E01AAE1BAEAB2DBB0C65
:10005000BB0BB9AFA8AF80915A01882309F485C0C2
:100060000E94B0C14B015C01B091E802B9A7BB236B
:1000700009F467C00E945C246091091570910A150B
:10008000072E000C880B990B0E94B4E08B018AAFFD
:100090009BAF288D398D4A8D5B8D0E9427E91816FC
:1000A00034F4088F198F2AAD2A8F3BAD3B8F2F81F7
:1000B0003D894E895F89B8018AAD9BAD0E94ADE054
:1000C00087FF06C00F831D8B4AAD4E8B5BAD5F8BE8
:1000D0008CA198014AAD5BAD6D817E81882309F4C6
:1000E0008BC1C1010E94ADE087FF2BC0B501A40107
:1000F0004419550966097709DB01CA0188589341FB
:10010000A109B109B7FD1DC08F859889A989BA8950
:100110008C199D09AE09BF09B595A7959795879547
:1001200080930D154DA35EA36FA378A79D81988F33
:10013000AE81A98F2A8E3B8E8B869C86AD86BE862D
:100140001CA220E030E040EF51E46D817E81C101CE
:100150000E94A4E798014AAD5BAD0E94ADE087FF25
:1001600022C081E69BE10E947B7A10925A010E9494
:10017000AF23F9CE4BEEC42ED12CE12CF12C8EC145
:1001800084E190E0A0E0B0E08F87988BA98BBA8BD8
:1001900034E1C32ED12CE12CF12C8EC1CF86D88A2C
:1001A000E98AFA8A89C1D501C4012AA53BA54CA5D3
:1001B0005DA5821B930BA40BB50BB7FD48C080E077
:1001C0000E9402238AE00E94637AD501C401805311
:1001D000984FAF4FBF4F8AA79BA7ACA7BDA79EA5BF
:1001E000911163C02FA538A949A95AA9B8018AADB0
:1001F0009BAD0E9427E918160CF043C020E030E0C8
:1002000040E050E4B8018AAD9BAD0E94A4E76FA71F
:1002100078AB89AB9AABA5019401205B3C434F4F6F
:100220005F4F2BAB3CAB4DAB5EAB20E030E040EC26
:1002300050E46D817E81C1010E94A3E798014AAD1F
:100240005BAD0E94ADE0881F8827881F8EA78B8535
:100250009C85AD85BE85481659066A067B0610F456
:10026000D301C201881A990AAA0ABB0A31E8831687
:100270003FE4930632E1A306B10470F183E49BE10D
:1002800072CFD501C4012BA93CA94DA95EA9821B3F
:10029000930BA40BB50B44E250E163E370E1B7FDAF
:1002A000D6CF80E00E947424D2CF20E030E040EF2F
:1002B00051E46D817E81C1010E94A3E79B01AC01E5
:1002C000B8018AAD9BAD0E94ADE087FFC0CF40ED85
:1002D00050E160EE70E1E5CF48AD59AD8B899C8966
:1002E000481759070CF069C003970CF466C086EEF6
:1002F0009AE10E947B7A89EC9AE10E947B7A49819B
:100300005A816B817C8182EE9AE10E94157B8AE0A2
:100310000E94637A89EC9AE10E947B7A48A159A1F4
:100320006AA17BA18EED9AE10E94157B8AE00E9472
:10033000637A89EC9AE10E947B7A4C8D5D8D6E8D9B
:100340007F8D8AED9AE10E94157B8AE00E94637A94
:100350009FA9992309F407CE29813A814B815C81B9
:1003600020930E1530930F154093101550931115CF
:100370002CEA35EC47E25EE368A179A18AA19BA152
:100380000E9413E160931215709313158093141556
:10039000909315152CEA35EC47E25EE36C8D7D8D6C
:1003A0008E8D9F8D0E9427E8609316157093171508
:1003B0008093181590931915D6CD0E94F45E4BCEFC
:1003C00083E19CE1EB960FB6F894DEBF0FBECDBF84
:1003D000DF91CF911F910F91FF90EF90DF90CF9021
:1003E000BF90AF909F908F907F906F905F904F9055
:1003F0003F902F900C947B7AC1010E9427E9181638
:100400000CF09FCED501C4012B853C854D855E85C2
:10041000821B930BA40BB50BAC01BD014858534193
:100420006109710977FD8DCE4B895C89452B09F4F3
:10043000FEC04DA05EA06FA078A4480E591E6A1E93
:100440007B1E2DA13EA14FA158A5281B390B4A0B9D
:100450005B0BC701B6010E94E5E6A30192010E9471
:1004600017E7CF84D888E988FA88C20ED31EE41E25
:10047000F51E54E1C516D104E104F1040CF480CE5C
:100480008CEEC816D104E104F1040CF073CE90E8B0
:10049000C916D104E104F1040CF480CECF86D88AC9
:1004A000E98AFA8A2EEF30E040E050E02C193D094D
:1004B0004E095F0969017A014F85588969897A89EE
:1004C0008CEC9BE10E943D7FB701A60187EC9BE18C
:1004D0000E943D7F4F815D896E897F8980EC9BE121
:1004E0000E94157B488D598D6A8D7B8D89EB9BE130
:1004F0000E94157BAB89BC8913970CF498C0C70187
:10050000B6010E94B4E020E030E040E850E40E94F0
:1005100013E169837A838B839C832F813D894E8984
:100520005F89688D798D8A8D9B8D0E94A3E72BED65
:100530003FE049E450E40E9413E120E030E040E075
:100540005FE30E9413E19B01AC0169817A818B8199
:100550009C810E9427E86F83788789879A87C301E7
:10056000B2010E94B4E02FE632E143E85AE30E9470
:1005700013E12B013C012AE939E949E15FE36F818D
:10058000788589859A850E9413E169837A838B83B4
:100590009C839B01AC010E94A4E7A30192010E94ED
:1005A00027E868A379A38AA39BA329813A814B8179
:1005B0005C81C301B2010E9413E120E030E040E021
:1005C0005EE30E9413E16C8F7D8F8E8F9F8F4F8132
:1005D000588569857A8583EB9BE10E94157BB30181
:1005E000A2018DEA9BE10E94157B8AE00E94637A5A
:1005F0008EE99BE10E947B7A49815A816B817C81E3
:1006000088E99BE10E94157B48A159A16AA17BA1C1
:1006100082E99BE10E94157B4C8D5D8D6E8D7F8DF7
:100620008CE89BE10E94157B8AE00E94637A8F85AB
:100630009889A989BA898C0D9D1DAE1DBF1DB595E0
:10064000A7959795879580930D152B893C892F5FEA
:100650003F4F3C8B2B8B3D813F834E814D8B2E8AB0
:100660003F8A2401350159A55CA36BCDCF93DF935D
:10067000EB010E947B7ACE01DF91CF910C94EACB03
:100680004F925F926F927F928F929F92AF92BF92A2
:10069000CF92DF92EF92FF920F931F93CF93DF934E
:1006A00000D01F92CDB7DEB780919A0C803108F050
:1006B000C7C131E6E32E80919A0C803108F0F8C072
:1006C0008091B10B9091B20B891B8F7709F4F0C028
:1006D0000E94367E97FF0BC00E94307B82E093E140
:1006E0000E947B7A8091B10B8093B20BE4CF8A3069
:1006F00019F08D3009F0D3C01092990C8091370C0D
:100700009091380CFC01ED5CF34F1682892B19F4A3
:100710000E94B636D0CF1092380C1092370C09E3F5
:100720001CE0F8018191803209F446C08E3409F052
:10073000A1C06DEF72E1C8010E942AE06C01892B13
:1007400041F06EE470E0C80104960E94F4E900975D
:1007500009F4C8014AE050E070E060E001960E94B0
:10076000A1DD4B015C018091330C9091340CA09180
:10077000350CB091360C0196A11DB11D8816990655
:10078000AA06BB0629F060E08AEC92E1CD2851F17F
:100790006AE270E0C8010E9423EA9C01009729F1F7
:1007A000982F901BF12C992349F09150F801E90FF3
:1007B000F11D8081F826F7CF8F01B3CF4AE050E0DA
:1007C00070E060E0C90101960E94A1DD4F2C512C20
:1007D000712C612C641575058605970551F060E054
:1007E0008BEA92E10E9496B866CF60E081E892E1E0
:1007F000F9CF8092330C9092340CA092350CB092C9
:10080000360C8091F9058130E1F067E470E0C801B1
:100810000E94F4E90097A9F04AE050E070E060E03F
:1008200001960E94A1DD623071058105910548F4B1
:1008300080EE91E10E947B7A60E086ED91E10E947A
:100840006E578091390C8B3309F435CF80919A0C17
:10085000803108F030CF80919C0C8E9DC001112416
:1008600069E37CE08356934F0E94FFE980E00E9499
:1008700062B821CF8091241780FFC3CF6BE175E26E
:10088000C8010E942AE0009731F0FC018381805367
:100890008A3008F0B6CF60E087E592E1A3CF27E386
:1008A0003CE049E35CE069E97CE00E94606903CFD9
:1008B0008091241782FFC4C01A82198281E6F82E23
:1008C00090E1B92E29E6A22E80919A0C803108F091
:1008D000B7C00E9498698111B3C041E050E0BE01E9
:1008E0006D5F7F4F8CE195E10E946DCD0B8110E033
:1008F000019711F00FEF1FEF8091241590912515AE
:10090000A0912615B0912715809320179093211759
:10091000A0932217B09323170E9498690F3F1007E6
:1009200049F4811107C00E94307B8AE193E10E9463
:100930007B7ACACF40919C0C242F30E00A3061F0C2
:100940000D3051F0882309F46DC089819A81009798
:1009500019F001969A8389831092340589819A81CE
:10096000F29EF001F39EF00D1124E656F34FDF01E5
:10097000A80FB91F13961C92892BB9F50E94B636A1
:100980000E949869882309F49FCF0E948D268CE1EC
:1009900095E10E94351E80911B178823F1F181504B
:1009A00080931B178A9DC001112462E086589A4FDC
:1009B0000E94A4CFE0911B1724E0E29FF0011124D4
:1009C000EA58FA4F40815181628173814093201728
:1009D0005093211760932217709323178CE195E1B0
:1009E0000E9445CC0E94E3C76FCF1A82198283818F
:1009F0008D3479F48481823361F48581853349F4BF
:100A0000868180538A3028F0809124178B7F8093D1
:100A1000241781E00E9462B8B3CF0E94D4C7B0927D
:100A2000F90552CF4F9DA00111244356534F9E010B
:100A30002F5F3F4F64E375E0802F0E94606944CFD1
:100A40000E94B0C14B015C018091680590916905DD
:100A5000A0916A05B0916B050097A105B10551F110
:100A600040914706509148066091490670914A06A8
:100A7000840F951FA61FB71FA5019401281B390BD2
:100A80004A0B5B0BDA01C901B7FD14C00E94307B31
:100A900060914E0670914F0689E991E10E9436837C
:100AA0008AE00E94637A40E070E060E090E080E0DD
:100AB0000E94B27D80914A0190914B01A0914C011E
:100AC000B0914D01892B8A2B8B2B79F09091B81521
:100AD0008091B915981709F4FCC08092470690924E
:100AE0004806A0924906B0924A060E94B0C16B0126
:100AF0007C0180914502811108C02091B815909128
:100B0000B91581E0291301C080E0209109153091C9
:100B10000A1591E089272A3A31050CF480E091E02A
:100B20004091300550913105609132057091330547
:100B3000452B462B472B09F490E0981789F0882322
:100B400009F401C1D701C60180569444A24FBF4F9A
:100B50008093300590933105A0933205B09333050F
:100B6000409078065090790660907A0670907B06E7
:100B700020912C0530912D0540912E0550912F0587
:100B8000C301B2010E94ADE0882319F180913005C4
:100B900090913105A0913205B091330540922C051A
:100BA00050922D0560922E0570922F05892B8A2B6D
:100BB0008B2B09F449C0D701C60180569444A24F3B
:100BC000BF4F8093300590933105A0933205B093C9
:100BD00033058091300590913105A0913205B09197
:100BE00033050097A105B10579F1C81AD90AEA0AB7
:100BF000FB0AF7FC29C010923005109231051092C3
:100C000032051092330584E891E10E947B7A60E01E
:100C100080E791E10E946E5780910B1590910C1521
:100C20001816190624F490E080E00E94FC4580919B
:100C30000406909105061816190634F4109205065C
:100C4000109204060E94D8178091350590913605C0
:100C5000A0913705B0913805A5019401281B390BE7
:100C60004A0B5B0BDA01C901B7FD8FC09091B81533
:100C70008091B915F090A406981749F0E091B91544
:100C80003BE4E39FF0011124E250F94FF0800E9411
:100C9000B0C1FF2009F4CFC00091280510912905AB
:100CA00020912A0530912B050115110521053105EB
:100CB00009F04DC06C597F4F8F4F9F4F60932805AF
:100CC0007093290580932A0590932B05FF24FA94AD
:100CD00044C00E94B0C1009147061091480620917F
:100CE000490630914A06C0904A01D0904B01E090ED
:100CF0004C01F0904D010C0D1D1D2E1D3F1D601B64
:100D0000710B820B930B97FF03C010923905EDCE48
:100D1000809139058111E9CE81E0809339055E9A91
:100D2000809145068E7F809345065E9A80914506A8
:100D30008D7F80934506159A809145068B7F809321
:100D400045065E9AD2CE80E090E0DC0101CF601BC8
:100D5000710B820B930B97FDB9CF0F2D10E084E040
:100D60000E9420B8F11070C060E084E00E94B9C019
:100D700044E6840E911CA11CB11C80923505909212
:100D80003605A0923705B09238050E94B63680919C
:100D9000F9058823E1F110913F011130B1F1809103
:100DA000241780628093241781E080933F0164EFD1
:100DB00071E080E090E00E94C1770E9405D28091AE
:100DC000241783FFA3C0123028F460E089E293E186
:100DD0000E946E5701E083E080935B010E94B0C1E6
:100DE0006C597F4F8F4F9F4F609341027093420227
:100DF0008093430290934402002339F0123029F487
:100E000081E080931A170E9460D20E94F45E0F90D6
:100E10000F900F90DF91CF911F910F91FF90EF9066
:100E2000DF90CF90BF90AF909F908F907F906F900A
:100E30005F904F9008951092280510922905109206
:100E40002A0510922B0589CF0F3F110511F461E09F
:100E50008CCFE6E5F5E2E491E150EA3008F051C0CC
:100E6000F0E0EB5CF8470C949AE73F8744874987AA
:100E70005387818781875D8765876D87778784B58D
:100E8000806884BDF7BC74CF84B5806284BDF8BC33
:100E90006FCF8091800080688093800010938900DC
:100EA0000093880065CF80918000806280938000ED
:100EB00010938B0000938A005BCF8091B000806814
:100EC0008093B000F092B30053CF8091B000806265
:100ED0008093B000F092B4004BCF80919000806876
:100EE00080939000109399000093980041CF8091D7
:100EF000900080628093900010939B0000939A0072
:100F000037CF003811050CF0A2CF2ECF00E011230F
:100F100009F47BCF60CF2F923F924F925F926F92F6
:100F20007F928F929F92AF92BF92CF92DF92EF9279
:100F3000FF920F931F93CF93DF93CDB7DEB76397E5
:100F40000FB6F894DEBF0FBECDBF8091680B83FD56
:100F50009FC189E40E94DF6E882309F48BC10E943F
:100F6000266F90E01816190614F481E090E026E050
:100F7000289FF001299FF00D1124E95FF94F82812C
:100F800093811A828C38910514F08CE890E090934C
:100F90000506809304060E94D8172091040630911C
:100FA00005068091020690910306821793070CF4C0
:100FB00022C18BEA9AE160E00E946E5781E0809343
:100FC0005A011B821C821D821E8219861A861B866C
:100FD0001C861E862CE32F873CE1388B46E4498B28
:100FE000312C212C50E859838FEB8A8B1B8A91E09E
:100FF0009D87812C912C54010091040610910506C7
:10100000B801012E000C880B990B0E94B4E06B0113
:101010007C01232D322D49815A890E94ADE088231D
:1010200089F08091020690910306AA81A111E6C081
:10103000B1E0BB8B081719070CF01B8A3C2C2D2C38
:10104000E982FA8A0E94B0C16B017C01DC01CB010C
:1010500029853A854B855C85821B930BA40BB50BC8
:10106000B7FD2FC0D701C60188519C4FAF4FBF4F6E
:1010700089879A87AB87BC8780E00E94022387EA32
:101080009AE10E947B7A81149104A104B10409F4CD
:10109000DFC0C501B40168577C4E8F4F9F4F6C195C
:1010A0007D098E099F0928EE33E040E050E00E9460
:1010B000F5E6CA01B9014AE00E941C7F8AE00E945D
:1010C000637A0E9440830E94B0C160934706709388
:1010D00048068093490690934A06609102067091F3
:1010E0000306072E000C880B990B0E94B4E06F8357
:1010F00078878C019B01AC01632D722D89819A89BF
:101100000E94A3E72B013C0120E030E0A9010E94EE
:1011100027E987FF04C077FA709477F870948114F8
:101120009104A104B10409F097C020E030E040E848
:101130005FE3C301B2010E94ADE087FF10C09D854F
:10114000812C912C5401992331F082E8882E86E07D
:10115000982EA12CB12C8C0C9D1CAE1CBF1CAB89F5
:10116000AA2391F12B813C814D815E8121153105AE
:101170004105510541F0D701C601821B930BA40B19
:10118000B50BB7FD21C02F813885A8016E857F85FD
:10119000888999890E94A3E720E030E040E85FE376
:1011A0000E94ADE087FD2DC0D701C601805A954150
:1011B000AF4FBF4F8B839C83AD83BE839F819E8740
:1011C000A885AF87088B198B80915A018823C9F0B5
:1011D00081149104A104B10461F0B8E8CB1AB3E121
:1011E000DB0AE108F108C818D908EA08FB08F7FE8D
:1011F00008C01D8601CF8AEB9AE1DDCE08171907DA
:101200000CF580915A01882309F442C010925A01CA
:1012100063960FB6F894DEBF0FBECDBFDF91CF91BE
:101220001F910F91FF90EF90DF90CF90BF90AF9004
:101230009F908F907F906F905F904F903F902F90F6
:101240000C94FDB93C2C2D2CE982FA8A1B8AFACE2B
:101250008FE30E94637A32CF20E030E040E450E434
:10126000C301B2010E9427E918160CF078CF46019D
:10127000570175CF83E50E94DF6E8A83811105C017
:1012800082E50E94DF6E882319F00E946B6F7ACE90
:1012900063960FB6F894DEBF0FBECDBFDF91CF913E
:1012A0001F910F91FF90EF90DF90CF90BF90AF9084
:1012B0009F908F907F906F905F904F903F902F9076
:1012C00008952F923F924F925F926F927F928F92EA
:1012D0009F92AF92BF92CF92DF92EF92FF920F93C5
:1012E0001F93CF93DF93CDB7DEB764970FB6F89413
:1012F000DEBF0FBECDBF8091680B83FDB0C10E94E1
:10130000387B898787FDABC189E40E94DF6E882323
:1013100009F497C10E94266F90E01816190614F47C
:1013200081E090E026E0289FF001299FF00D112434
:10133000E95FF94F808191811B8A0E94FC452091D1
:101340000B1530910C158091091590910A15821793
:1013500093078CF487E99AE19F938F9382EA9AE14D
:101360009F938F931F920E9455570F900F900F904D
:101370000F900F9005C02B898CE89AE1222361F32E
:1013800081E080935A011C821D821E821F821A8670
:101390001B861C861D861F862CE3288B3CE1398B1F
:1013A00046E44A8B212C312C50E85A838FEB8B83F7
:1013B000198291E09E87812C912C540101C01E86D8
:1013C00000910B1510910C15B801012E000C880B23
:1013D000990B0E94B4E0D62EE72EF82E9887910143
:1013E0004A815B810E94ADE0882391F080910915CC
:1013F00090910A153B893111E7C041E049830817F4
:1014000019070CF019822D2C3E2CFA8258855B832B
:101410000E94B0C16B017C01DC01CB012A853B85B8
:101420004C855D85821B930BA40BB50BB7FD2FC0BC
:10143000D701C60188519C4FAF4FBF4F8A879B870A
:10144000AC87BD8789850E94022388E89AE10E94C3
:101450007B7A81149104A104B10409F4E0C0C501B0
:10146000B4016053784F8F4F9F4F6C197D098E09DF
:101470009F0928EE33E040E050E00E94F5E6CA0103
:10148000B9014AE00E941C7F8AE00E94637A0E94B0
:1014900040830E94B0C160934706709348068093D2
:1014A000490690934A066091091570910A15072E16
:1014B000000C880B990B0E94B4E06887072F182F47
:1014C0009C8B262F372F482F592FB1018A819B8162
:1014D0000E94A3E72B013C0120E030E0A9010E941B
:1014E00027E987FF04C077FA709477F87094811425
:1014F0009104A104B10409F096C020E030E040E876
:101500005FE3C301B2010E94ADE087FF10C09E857A
:10151000812C912C5401992331F08AE9882E82E0A4
:10152000982EA12CB12C8C0C9D1CAE1CBF1CA9812B
:10153000AA2399F12C813D814E815F8121153105CE
:101540004105510541F0D701C601821B930BA40B45
:10155000B50BB7FD22C02885302F412F5C896F85E0
:10156000788989899A890E94A3E720E030E040ECDD
:101570005FE30E94ADE087FD2AC0D701C601805A13
:101580009541AF4FBF4F8C839D83AE83BF839885BA
:101590009F87088B198BAC89AA8B80915A0188236D
:1015A000B1F081149104A104B10409F408CFB0EDA5
:1015B000CB1AB7E0DB0AE108F108C818D908EA0835
:1015C000FB08F7FCFCCE03C0081719070CF5809147
:1015D0005A01882309F443C010925A0164960FB649
:1015E000F894DEBF0FBECDBFDF91CF911F910F9159
:1015F000FF90EF90DF90CF90BF90AF909F908F9033
:101600007F906F905F904F903F902F900C94FDB91A
:101610002D2C3E2CFA8288858B831982F9CE8FE39C
:101620000E94637A31CF20E030E040E450E4C3010F
:10163000B2010E9427E918160CF079CF4601570134
:1016400076CF83E50E94DF6E8B8B811105C082E52A
:101650000E94DF6E882319F00E946B6F6ECE649635
:101660000FB6F894DEBF0FBECDBFDF91CF911F91B3
:101670000F91FF90EF90DF90CF90BF90AF909F9031
:101680008F907F906F905F904F903F902F90089534
:101690002F923F924F925F926F927F928F929F9282
:1016A000AF92BF92CF92DF92EF92FF920F931F9370
:1016B000CF93DF93CDB7DEB7ED970FB6F894DEBFCB
:1016C0000FBECDBF80916B02888B87E50E94AE6E06
:1016D000882309F41BC120E030E0A9016091DD02FC
:1016E0007091DE028091DF029091E0020E94ADE0F5
:1016F000811107C00E94307B88E895E10E947B7AC7
:1017000018C18AE50E94DF6E882339F10E947E6F3E
:1017100020916606309167064091680650916906EF
:101720000E94A3E76B017C0120E030E040E251EC35
:10173000C701B6010E9427E987FD0AC020E030E01A
:1017400040E251E4C701B6010E94ADE0181674F4FE
:101750000E94307B8BE795E1D1CFC0907406D0908A
:101760007506E0907606F0907706DECF40E050E018
:1017700060EC7FE788E50E94A86F20915E063091BB
:101780005F0640916006509161060E94A3E72B011D
:101790003C0140E050E060EC7FE789E50E94A86FE3
:1017A000209162063091630640916406509165066F
:1017B0000E94A3E74B015C016FEF89E40E943A6F3E
:1017C000182F6FEF8AE40E943A6F082FA30192014D
:1017D000C301B2010E94A5E981116EC0A501940167
:1017E000C501B4010E94A5E9811166C08BA19CA12D
:1017F000ADA1BEA18BAB9CABADABBEAB2091D50276
:101800003091D6024091D7025091D802C301B20163
:101810000E94A3E72B013C0120E030E040E05FE3C1
:101820006BA97CA98DA99EA90E9413E19B01AC0123
:10183000C301B2010E94A4E72BA93CA94DA95EA94E
:101840000E9427E80E9499E8162F4FA058A469A487
:101850007AA42091D9023091DA024091DB025091B2
:10186000DC02C501B4010E94A3E74B015C0120E04A
:1018700030E040E05FE3C301B2010E9413E19B014D
:10188000AC01C501B4010E94A4E7A30192010E942A
:1018900027E80E9499E8062F812F012E000C990B52
:1018A00097FD2CC0059764F5802F002E000C990B36
:1018B00097FD28C0059744F51530D8F50530C8F5D3
:1018C00080E00E94B57695E01902F0011124E00F46
:1018D000F11D07FDFA95EE0FFF1FEE0FFF1FEF58EA
:1018E000FD4FC082D182E282F38288890E94B57660
:1018F00088898823F1F00E943F3D1BC010E0D4CFBF
:1019000014E0D2CF00E0D8CF04E0D6CF8AE40E9422
:10191000AE6E81110CC070E060E086E50E946F6FD2
:101920009A8389830597F0F086E595E1E7CE0E94DA
:101930000377ED960FB6F894DEBF0FBECDBFDF91F3
:10194000CF911F910F91FF90EF90DF90CF90BF90BC
:10195000AF909F908F907F906F905F904F903F904F
:101960002F90089560E084E40E94566F8F8740E0D6
:1019700050E0BA018AE50E94A86F6BA77CA78DA7EB
:101980009EA740E050E86BE376E483E50E94A86FF1
:1019900020E030E040E752E40E9427E860935C01D9
:1019A00070935D0180935E0190935F010091B31588
:1019B0001091B415D801CD90DD90ED90FC9020E011
:1019C00030E0A901C701B6010E94A4E76AAF7BAF6E
:1019D0008CAF9DAF20E030E040E450E40E94ADE0E9
:1019E00087FF06C01AAE1BAEB0E4BCAFE0E4EDAFBB
:1019F00020E030E04AE753E4C701B6010E94A4E7C3
:101A00006BAB672E8FAB98AF20E030E043E653E43A
:101A10000E9427E9181634F41BAA612CF3E6FFABE9
:101A200023E428AFD80114968D909D90AD90BC9082
:101A3000179720E030E0A901C501B4010E94A4E796
:101A40007B018C0120E030E040E951E40E94ADE0F0
:101A500087FF04C0E12CF12C00E911E420E030E024
:101A60004AE753E4C501B4010E94A4E7B62EC72E8D
:101A7000D82E99AF20E030E044E553E40E9427E9F6
:101A8000181634F4B12CC12CF4E5DF2EB3E4B9AF51
:101A900088E40E94AE6E882309F40DC20E947E6F16
:101AA0000E9499E81B0177FF02C06F5F7F4F759519
:101AB00067957195619571096D587F4F072E000CE0
:101AC000880B990B0E94B4E0762E872E982EA92EB3
:101AD0009701A8010E9427E9181624F4E72CF82C96
:101AE000092D1A2D2AAD3BAD4CAD5DAD672D782D7E
:101AF000892D9A2D0E9427E9181624F07AAC8BAC18
:101B00009CACADAC872D982DA92DBA2D8B8B9C8BC1
:101B1000AD8BBE8BC701D8018F8B988FA98FBA8FE1
:101B2000B101330C880B990B0E94B4E01B012C010E
:101B3000AC019B01B701C8010E94A4E77B018C01A5
:101B40002B2D3C2D4D2D59AD0E94ADE087FF04C0DB
:101B5000BE2CCF2CD02E19AFA2019101672D782D6C
:101B6000892D9A2D0E94A4E77B018C012BA9362D8B
:101B70004FA958AD0E94ADE087FF04C0EBAA6F2CBF
:101B80000FAB18AF8BA9962DAFA9B8AD8B8F9C8FDB
:101B9000AD8FBE8F8B2D9C2DAD2DB9AD8F8F98A3A2
:101BA000A9A3BAA3BE01695E7F4FCE0143960E94EE
:101BB0009573882309F4AEC1BE01615E7F4FCE01EB
:101BC0004B960E949573E82E882309F4A3C12F89B0
:101BD000388D498D5A8D6F8D78A189A19AA10E9467
:101BE000A3E720E030E040E85EE30E9413E14B0110
:101BF0005C012B893C894D895E896B8D7C8D8D8D37
:101C00009E8D0E94A3E720E030E040E85EE30E9462
